:100000005446495312720105000008000000000028
:10001000000000800100000058479D2700001000EC
:100020000000000000000000400000000000000090
:1000300000000000010000000000000000000000BF
:10004000544643530000100000D50100FCF0A1F21B
:10005000000001200101100007011000090110003B
:100060000B0110000D0110000F0110001F01100006
:100070001F0110001F0110001F01100011011000CE
:10008000130110001F01100015011000372E100081
:10009000212F10001901100019011000F595110011
:1000A00019011000B9101000BD1010001901100046
:1000B00019011000D12C100019011000C1101000FE
:1000C0001D301000E9021000251B1000190110005E
:1000D0000000000000000000000000000000000020
:1000E0000000000000000000000000000000000010
:1000F0000000000000000000000000000000000000
:1001000000000000000000000000000000000000EF
:1001100000000000000000000000000000000000DF
:1001200000000000000000000000000000000000CF
:1001300000000000000000000000000000000000BF
:1001400000000000000000000000000000000000AF
:1001500000F010F8FEE7FEE7FEE7FEE7FEE7FEE749
:10016000FEE7FEE7FEE7FEE701480047FEE7FEE7A1
:100170001F01100000F002F800F04AF80AA090E811
:10018000000C82448344AAF10107DA4501D100F052
:100190003FF8AFF2090EBAE80F0013F0010F18BFD5
:1001A000FB1A43F0010318473CB201005CB20100A6
:1001B0000A4410F8014B14F00F0508BF10F8015B5A
:1001C000240908BF10F8014B6D1E05D010F8013B43
:1001D0006D1E01F8013BF9D1641E03D0641E01F8C5
:1001E000015BFBD19142E4D370470000002300245F
:1001F00000250026103A28BF78C1FBD8520728BF37
:1002000030C148BF0B6070471FB51FBD10B510BD92
:10021000DFF80CD0FFF7F8FF03F062FE19F0FEF9EB
:100220000000012003B4FFF7F1FF03BC19F0FEF951
:10023000002101E000BF491C8142FBDB7047704791
:100240007047704770477047704700E0401C017866
:100250000029FBD170470CB5010F8DF80010C0F3D9
:1002600003618DF80110C0F303518DF80210C0F343
:1002700003418DF80310C0F303318DF80410C0F36F
:1002800003218DF80510C0F303118DF8061000F05E
:100290000F008DF8070000206A46115C0A2901D280
:1002A000303100E037311154401CC0B20828F4D37B
:1002B0000020401CC0B20828FBD30CBD0CB50109BE
:1002C0008DF8001000F00F008DF8010000206A4644
:1002D000115C0A2901D2303100E037311154401C41
:1002E000C0B20228F4D30020401CC0B20228FBD3C5
:1002F0000CBD0CB5010B8DF80010C0F303218DF877
:100300000110C0F303118DF8021000F00F008DF8FA
:10031000030000206A46115C0A2901D2303100E056
:1003200037311154401CC0B20428F4D30020401CC3
:10033000C0B20428FBD30CBD10484FF6FF7101601A
:1003400070470E480E4A002101601268102050616B
:100350000C48012203685A6003684022DA6003688F
:100360004FF40C621A6102685161026840F6FF7135
:1003700011620068EA21016303A066E700700020B3
:100380000CA911003CA9110055415254204F504571
:100390004E21210D0D0000000B0ACAB2F94910B51B
:1003A0000C68E06143F4FE400B685861086800681F
:1003B0000B6840F0010018600868C068C007FBD0F7
:1003C000086880680B6840F00100986002F07F02C6
:1003D0004FF4004040EA0222086842610868006861
:1003E0000B6840F0010018600868C068C007FBD0C7
:1003F000086880680B6840F00100986008684261F6
:10040000086800680A6840F0010010600868C06869
:10041000C007FBD0086880680A6840F0010090605F
:1004200008688069C0B210BD00F07F0041EA002179
:10043000D4480268516101680968026841F001010D
:1004400011600168C968C907FBD001688968006844
:1004500041F001018160704700F07F014FF40040DE
:1004600040EA0122C74801684A61016809680368D7
:1004700041F0010119600168C968C907FBD0016832
:100480008968036841F00101996001684A61016867
:100490000968026841F0010111600168C968C90773
:1004A000FBD001688968026841F001019160006831
:1004B0008069C0B2704730B50D460446FFF7CCFFE7
:1004C00020EA0501E0B2BDE83040ADE77047F0B585
:1004D000AC48002401210268C2F8141302686FF0CE
:1004E000FE21C2F8201302689921C2F83013006877
:1004F0000321C161A448A54DA54E00684FF4A6771D
:100500004FF0010390F8800188B935F82300C0F35B
:1005100007217F20FFF788FFF01890F8C01615F824
:100520002300FFF781FF5B1CBB42EEDBF0BD35F81B
:100530002300C0F30720844205D0044600F00F01D9
:100540007F20FFF771FFF01890F8C01615F8230010
:10055000FFF76AFF5B1CBB42E9DBF0BD10B503F09F
:10056000C7FC884B04464FF00430196808621968CC
:1005700000144862196801200861196888601968C8
:10058000486000217F20FFF74FFF40210120FFF747
:100590004BFF052C03D119680020C1F8100310BDD2
:1005A000784A00B512680321D16100284FF000019C
:1005B0004FF07F0007D0FFF737FF03210020FFF740
:1005C00033FF002102E0FFF72FFF012100205DF83B
:1005D00004EB29E76B4A00B512680321D1610028BA
:1005E0004FF000014FF07F0003D0FFF71DFF012106
:1005F00006E0FFF719FF03210020FFF715FF002198
:1006000000205DF804EB0FE75E4900B509680320A0
:10061000C86100217F20FFF707FF00205DF804EB91
:100620001AE7584900B509680320C86100217F20F6
:10063000FFF7FAFE082102205DF804EBF4E65149C9
:100640000A68926C0123834008681A4382647047E9
:1006500070474C490968896D80F001000122801CB7
:10066000824001EA0200704746480168496C02680E
:1006700041F4006151640168496C006821F4006133
:10068000416470473F4B012282401868006C09B1F9
:10069000104300E090431968086470473949002806
:1006A0000868C06D0AD00A6840F00200D06508688A
:1006B000C06D40F010000968C86570470A6840F0D6
:1006C0000100D0650868C06D40F00800F3E72DE92F
:1006D000F043DFF8B09080462025D9F800000926C5
:1006E0000221C161002704217F20FFF79DFE002425
:1006F000032C02D0062C02D006E0052100E00621E2
:100700007F20FFF791FE0027002308EB441C07E041
:100710001CF803103846FFF787FE7F1CFFB25B1CF6
:10072000AB42F5D3641CB442E2D3D9F800000121F6
:10073000C161002704217F20FFF776FE00241CE022
:10074000032C02D0062C02D006E0052100E0062191
:100750007F20FFF769FE0027002308EB441C09E017
:100760000CEB030090F820113846FFF75DFE7F1C6C
:10077000FFB25B1CAB42F3D3641CB442E0D3BDE8D0
:10078000F083000010A91100FC06002000000020EA
:10079000DC60002070B5A049044603200968C861E8
:1007A0000425E9B27F20FFF73FFE0023E1B2D8B273
:1007B000FFF73AFE03F12000E1B2C0B2FFF734FECA
:1007C00003F14000E1B2C0B2FFF72EFE5B1C202B0C
:1007D000ECDB0BF08FFA00B900246D1C072DE0DB79
:1007E00070BD8D4803210268D16102681121C2F8F1
:1007F000301300684FF00111C0F8201300217F2052
:1008000012E62DE9F0410546002403F071FB0228B1
:1008100004D003F06DFB052803D006E00BF06AFA64
:1008200001E008F09EFB00B37C4CFFF797FE7A498D
:1008300003200968C8617A4E01234FF4A67736F881
:100840002300C0F307217F20FFF7EEFDE95C16F8D7
:100850002300FFF7E9FD1CB1E118E85C81F8C00650
:100860005B1CBB42EBDBBDE8F0816E4CDDE76A4B05
:1008700000B519680320C86100217F20FFF7D4FD6F
:1008800000210120FFF7D0FD00210320FFF7CCFD60
:1008900001217F20FFF7C8FD0A210E20FFF7C4FDCC
:1008A00002217F20FFF7C0FD35210220FFF7BCFDAC
:1008B00078210720FFF7B8FD8B210420FFF7B4FD56
:1008C0000F217F20FFF7B0FD01210320FFF7ACFDD2
:1008D00019680120C1F8140319681120C1F8300308
:1008E00019684FF00110C1F8200303217F20FFF7A2
:1008F0009BFD01210020FFF797FD00210120FFF75C
:1009000093FD21210520FFF78FFD04216D20FFF7C6
:100910008BFD08216E20FFF787FD10216F20FFF768
:1009200083FD01217F20FFF77FFD08210020FFF7D5
:100930007BFD04210120FFF777FD5DF804EB93E6D2
:10094000354900B509680320C86100217F20FFF701
:100950006BFD00210120FFF767FD01217F20FFF7DC
:1009600063FD21210E20FFF75FFD02217F20FFF7AD
:100970005BFD45210220FFF757FD35210320FFF7DE
:1009800053FD20211620FFF74FFD03217F20FFF7A5
:100990004BFD092103205DF804EB45E570475A2122
:1009A000B0FBF1F0C0EB00108000704700207047F2
:1009B00000207047002070470020704708467047AD
:1009C0000020704770470020704770477047002034
:1009D0007047704770470020704700207047002024
:1009E000704700207047704770470020704770477D
:1009F000704770470020704700207047704770476D
:100A000070470020704700207047704700207047F3
:100A1000704770477047704710A91100DC600020D4
:100A2000000000204C080020FF4910B50968032091
:100A3000C86100217F20FFF7F7FC02210020FFF7AB
:100A4000F3FC01210220FFF7EFFC0121BDE810407B
:100A50000020FFF7E9BCE7E7F44808B501684969F9
:100A6000C1F30721009101684969009AC1F3072188
:100A70009142F8D0EC480168D1F82C13006841F09D
:100A80000401C0F82C13FFF7BFFD002804D0BDE817
:100A900008400020FFF79EBD08BDDDE710B503F05C
:100AA00027FA052807D0E0480068D0F82C03400753
:100AB00005D5002010BDDE480068006810BD01208B
:100AC00010BD70B50546FFF7E9FF01281ED103F000
:100AD0000FFAD54C052815D0FFF7BEFF012D15D113
:100AE0002068406C216840F40060486400BF00BF8B
:100AF00000BF2068406C216820F400604864BDE8B5
:100B0000704091E70020FFF765FDE9E770BD10B583
:100B1000FFF724FD0120FFF7D4FF102003F0B5FC00
:100B20000121052001F01DFF0121062001F019FF20
:100B3000C0490120887010BD10B5602001F062FF2F
:100B4000602001F052FFB84903200968C86410BD55
:100B5000B84A0146507900B1012001B1012151711B
:100B60007047B44A0146106911617047B1480021CD
:100B70000171C1700189B04818F0B2BCF6E7AA490A
:100B800000280868406C20F4407013D00A68506454
:100B90000868426CA9480068037EC3F3001342EA68
:100BA00043220B685A640A68526C007EC0F3C0008E
:100BB00042EA00200968486470471CB500208DF89F
:100BC0000000ADF8040003F093F904460120FFF79C
:100BD000D6FF022C21D10BF08DF802281DD19249AD
:100BE00001200968C86103217F20FFF71DFC8921CE
:100BF0000520FFF719FC67210620FFF715FC4521AA
:100C00000720FFF711FC23210820FFF70DFCBDE8AA
:100C10001C40F1210920FFF707BC1CBD2DE9FF5F37
:100C20000026824634464FF010090196009603F0E4
:100C30005FF9022804D003F05BF9052803D004E033
:100C40000BF058F801E008F08CF903F051F97C49F9
:100C5000052804D10868022808D04FF03609086832
:100C600038B1012804D0022802D002E04FF0000978
:100C700001247448744900680969406BFF3100F52C
:100C8000E03021F0FF01503004FB010712200290F8
:100C9000202000240390032C01D214261AE0E01E29
:100CA000032801D2152615E0A01F032801D216261D
:100CB00010E0A4F10900032801D224260AE0A4F1DF
:100CC0000C00032801D2252604E0A4F10F0003281C
:100CD00000D226260198B0420AD053490196C6F3A5
:100CE00003100968C86106F00F017F20FFF79CFB25
:100CF0000BF000F818B1FF208046002562E0B42018
:100D0000FAE7202D5BD2C6F3031001284FF0030051
:100D1000B4FBF0F100FB114010D0C5F11F0101EB55
:100D200040101FFA80FB01226946384600F0A9FFF7
:100D30007F1C03F0DDF8022821D026E005EB401BE4
:100D400001226946384600F09CFF7F1C03F0D0F872
:100D5000022805D10098404502D380384F2806D29A
:100D600003F0C6F8052804D10098FF2801D1CDF87A
:100D700000900098C1B20AEB441041551AE0009867
:100D8000404502D380384F2806D203F0B1F8052839
:100D900004D10098FF2801D1CDF800900920B4FBC0
:100DA000F0F100FB11410AEB411000992844C9B24F
:100DB00080F820110BF0FF00FFF736FB00E07F1CEE
:100DC0006D1CEDB2039885429BD3641C0298E4B27B
:100DD0008442FFF460AFBDE8FF9F1649C8607047CA
:100DE00010B503F085F8052802D0BDE8104033E6C1
:100DF000FFF754FE012804D1BDE810400020FFF7A2
:100E0000E9BB10BD2DE9F04782460C460120FFF7F3
:100E100058FE03F06DF805468CB3FFF7E1FF6068FC
:100E200068B3206858B311E010A911002CA9110073
:100E300014A911003005002038110020FC06002004
:100E4000C8050020B8060020BC06002001276FF06E
:100E5000FE284FF09909FE4E052D02D0022D1BD021
:100E600031E008F07EF80546D4E90010FFF7C9FC30
:100E70003068C0F81473022D02D055B123E02CE085
:100E80003168C1F820833168C1F83093FFF758FD0D
:100E900019E0FFF7ECFC16E00AF02CFF0546D4E958
:100EA0000010FFF7AEFC3068C0F81473022D01D0BB
:100EB0003DB108E03168C1F820833168C1F8309352
:100EC00001E0FFF78EFC31680020C1F82803E149FA
:100ED000C1F80CA0A068FFF7A1FEBDE8F0476CE6E2
:100EE000704710B5FFF78EFFFFF740FE0020FFF7B9
:100EF00038FE0020FFF72CFEBDE810401CE6602005
:100F000001F077BD10B5602001F073FDBDE8104021
:100F10000120D6E5CF48C0687047CE480078002849
:100F200000D001207047F8B500240094FFF7B6FD0B
:100F3000002851D1FFF71AFEC54D2868406C29687A
:100F400040F40060486400BF2868406C296820F4C1
:100F500000604864C04EC149307800280868406984
:100F60001ED0C0B2009008684069009AC0B290429A
:100F7000F9D009680220C8612868D0F82C032968D4
:100F800020F00400C1F82C032868C0F81043FFF7D4
:100F90003BFB002820D1BDE8F8400120FFF71ABB39
:100FA000C0F30720009008684069009AC0F307204A
:100FB0009042F8D000200A685269D2B200920A68C2
:100FC0005269009BD2B29A42F9D0401CC0B20428A8
:100FD000F1D301203070CCE7F8BD70B502F088FF86
:100FE00000249C4D052803D02C70BDE870409AE782
:100FF000FFF754FD002810D1FFF7B8FD2C7094487E
:101000000168D1F82C13006821F00401C0F82C13FA
:10101000BDE870400120FFF7DDBA70BD8D490120A9
:101020000870704770B502F063FF0124894D0528F0
:1010300007D0FFF733FD00280FD12C70BDE87040BA
:1010400071E7FFF72BFD002807D1FFF78FFD2C700C
:10105000BDE870400120FFF7BDBA70BD012030E54A
:101060007C490020C870B8E77A4A0146506951614E
:10107000704778488069704776498861704775483D
:10108000806970477348407870477249487070476C
:10109000012808D8724900280868406E04D040F042
:1010A000020009684866704740F00100F9E701282E
:1010B00008D86B4900280868406E04D020F0020070
:1010C00009684866704720F00100F9E770B50546E9
:1010D000FFF7DEFF5F4CA069401CA061216909B1E8
:1010E00028468847207810B10120FFF7EAFC5848CD
:1010F00045B10121006801655A48016841F02001AD
:10110000016070BD0221F5E70020DFE70120DDE787
:1011100010B5504CE069401CE0614D480168096D14
:10112000006841F004010165FFF79EFAFFF779FAC4
:10113000207810B10120FFF7C4FC606900B180473E
:101140004848016841F40061016010BD10B50120FC
:10115000FFF7B7FCBDE8104000F05BBB42487047AA
:101160004148093070473B48006A70473948406A37
:1011700070473848806A70473648002101624162F2
:1011800081627047384900EBC0002C3101EBC01080
:10119000704748434FF6FF7101EA40002D4908812E
:1011A00070472C4A921D1070517070472949891D53
:1011B000085C7047F0B50746A1B020240121022049
:1011C000FFF760FA294D00206E46296831F81010AB
:1011D00026F81010401CA042F7D300210220FFF790
:1011E00051FA01210020FFF74DFA002007E029689D
:1011F00006EB400231F81010A2F84010401CA0424B
:10120000F5D300210846FFF73DFAA20069463846AB
:1012100018F0C5F821B0F0BDF0B50E460546202403
:10122000E1B002212046FFF7B4FF4FF0010175B194
:101230000420FFF727FA0D4900206A46096801EBF0
:10124000053303EB800101F580510F6810E027E0C2
:1012500010A9110030050020AA0500202CA91100BA
:101260000CA91100640500200C11002034A9110004
:1012700042F8207002EB8007D1F88010401CC7F8BC
:101280008010A042DDD34FF000015DB10420FFF7D4
:10129000F9F9E2006946304618F081F861B0F0BD16
:1012A0000520C6E70520F2E770B50400FB480E46AE
:1012B0004FF00101058914D00420FFF7E3F9F84845
:1012C0002A46006800EB0431304601F5805118F0E1
:1012D00066F84FF0000134B10420BDE87040FFF71C
:1012E000D1B90520E9E70520F7E730B591B005460B
:1012F00020244021684618F0F3F80021684605EBE9
:10130000410335F81120B3F840321A4420F8112077
:10131000491CC9B2A142F2D301466200284618F026
:101320003EF811B030BDF0B5DC4EDD4FADF2844D6E
:10133000002435894FF00101ECB10420FFF7A2F938
:1013400038682A4600EB0431684601F5805118F0F0
:101350006BF84FF0000184B10420FFF793F9641C8F
:10136000022CE6DB0020FFF7A2FE0120FFF79FFE24
:101370000DF2844DF0BD0520E0E70520EDE7C94BF7
:10138000C94900201A6802EB8002D2F8C02021F877
:101390001020401C0728F5D31868D0F8E4004882D4
:1013A0007047C14A10B5BF4B803AF0B100201968B0
:1013B00001EB8001D1F880110904090C01D022F859
:1013C0001010401C2028F2D30020196801EB800186
:1013D000D1F880120904090C03D002EB4004A4F8F0
:1013E0004010401C2028F0D310BD196801EB80018B
:1013F000D1F800110904090C01D022F81010401C8A
:101400002028F2D30020196801EB8001D1F80012E6
:101410000904090C03D002EB4004A4F84010401C5E
:101420002028F0D310BDF8B504460020009002F04B
:101430005FFD0127994E84F00105052802D00AF0CE
:1014400059FC98B12046FFF704F928B92C462846E4
:10145000FFF7FFF800281ED094492046FFF724FF2D
:10146000FFF78DFF2046FFF79CFF0DE02046FFF7BA
:10147000F0F828B92C462846FFF7EBF800280AD0E8
:101480008A492046FFF710FF2046FFF710FE37710C
:1014900084F00100F070F8BD70B5804D04466879A5
:1014A00010B9E878FFF7BFFF287900280DD07E48F3
:1014B000AB69A0F18001A0610020C4E902102061A5
:1014C0007A4A6061C4E90032012070BD734900208E
:1014D000087170472DE9F14F82B00025122000906D
:1014E0002020A8462C460190032C01D214251AE096
:1014F000E01E032801D2152515E0A01F032801D204
:10150000162510E0A4F10900032801D224250AE0E1
:10151000A4F10C00032801D2252504E0A4F10F005A
:10152000032800D22625A8450AD05E49C5F303103A
:10153000A8460968C86105F00F017F20FEF774FF17
:101540000298032100EB441AB4FBF1F001FB1047B1
:1015500000260921B4FBF1F001FB10400299C5F30C
:10156000031B01EB40190FE0BBF1010F16D0C6F1D0
:101570001F0000EB471080B2FEF76EFF09EB06017B
:1015800081F82001761CF6B201988642ECD3641CE7
:101590000098E4B28442A7D3BDE8FE8F06EB471063
:1015A000FEF75AFF0AF80600ECE701207047704783
:1015B000002070472DE9F0411E4615460F46804633
:1015C000FFF76CFA040002D00120FFF77AFA01233A
:1015D00007EB060C0DE00021404605E003FA00F29F
:1015E000324200D0491C401CA94201D22028F5D328
:1015F0007F1CBC45EFD8002C02D0BDE8F0412FE5A0
:10160000BDE8F0812DE9F047994690460D46064623
:10161000089CFFF743FA070002D00120FFF751FAB8
:1016200002F0A0FD224906EB080305EB090C086057
:101630000EE0304607E00A68127824F8022B0A68A8
:10164000521C401C0A60834201D92028F3D36D1C30
:10165000AC45EED8002F02D0BDE8F04700E5BDE86C
:10166000F087704710B5FFF7AEF90C49488110BDFF
:101670000A4A10B55289C1B200F47063914200D990
:10168000114664246143B1FBF2F11A0A02FB041112
:1016900089B2C0040ED508B210BD0000300500208C
:1016A00034A9110010A911003816002038110020AB
:1016B000DC050020484200B2EEE7002803DA404291
:1016C00080B2002102E080B24FF4805100F47062D9
:1016D0000A434749C0B24989484342EA102070474B
:1016E00008B50921732000F0FBF8BDF8001000F0E8
:1016F0001F0021F0FF010843ADF800000D21732009
:1017000000F0EEF800F01F01BDF8000061F31F20AB
:10171000ADF80000BDF8000008BD7047FFF769B9DB
:1017200034484FF41071006800F5405017F0D8BEEF
:101730002DE9F84F1220DFF8C4B000902E484FF08A
:10174000200A0024CBF80000032C01DA14251AE04B
:10175000E01E032801D2152515E0A01F032801D2A1
:10176000162510E0A4F10900032801D224250AE07F
:10177000A4F10C00032801D2252504E0A4F10F00F8
:10178000032800D22625A9450AD01D49C5F3031018
:10179000A9460968C86105F00F017F20FEF744FEE5
:1017A0000026032194FBF1F001FB1047C5F3031859
:1017B00010E0B8F1010F15D0C6F11F0000EB471083
:1017C000DBF80020C0B212F8011BCBF80020FEF7B6
:1017D0002BFE761C5645ECDB0098641C8442B3DB80
:1017E000BDE8F88F06EB4710EAE70020FFF7E0B806
:1017F0003005002034A911005C650020DC050020C4
:1018000010A91100054908B1002000E0012008706E
:101810007047704770477047704700005C050020B4
:1018200070472DE9F04101F093FB294E294D2A4BD9
:101830002A494FF47A7700224C682CB14A6001F0B3
:101840008CFB2046BDE8F081307860B90888B8424A
:101850000BD930BF287830B1186800681C6820F0B8
:10186000010020602A700A80E6E7401C0880E3E758
:1018700010B501F06DFB194844682CB1002141609E
:1018800001F06BFB204610BD30BFF5E770B501F0ED
:101890005FFB124D6C682CB10020686001F05DFBAD
:1018A000204670BD30BF01F0D1F80028F2D001F021
:1018B000D1F8A860EEE70020704730BF704772B6DD
:1018C00062B670477047704772B662B670470000E4
:1018D000300600204207002014A9110060050020F6
:1018E000C24BC2081B681A6401F0FC0141EA0020E7
:1018F000BF4908430068704710B50C46FFF7F0FF7A
:10190000A107C90EC840C0B210BDBA4800B5002139
:1019100001707220FFF7F0FF000601D5012000BD25
:10192000002000BD30B5B14BC4081D682C6401F027
:10193000FC0141EA0020AE490843026000E000BF1C
:101940001868006C8005FAD430BD70B516460C4698
:101950000546FFF7C5FFA107CB0EFF21994088433D
:101960009E4046EA000221462846BDE87040D9E77D
:10197000A1484FF4F4610268116101684968026886
:1019800041F00201516000680321816170479A496A
:1019900010B5096810200860FFF7EAFF0722082148
:1019A0007120FFF7D2FF0E2001F007F8BDE81040CC
:1019B0000E2001F00EB88D4910B509688F480862F5
:1019C000072201217020FFF7C0FF3F220021742071
:1019D000FFF7BBFFBDE81040D9E787480021026848
:1019E000116002684FF4E0611161006801218161BA
:1019F0007047814800210268116002681161006827
:101A0000816170477C4806210268116002680221EA
:101A10005160006881617047774800210268116059
:101A20000068816170477449002009680860704748
:101A30007148082102681160026802219161016801
:101A4000C9680907FBD500680F218160704710B590
:101A5000044602460021F020FFF764FF22460121E0
:101A6000F020FFF75FFF22460021F120FFF75AFF29
:101A700022460121F120FFF755FF22460021FC20DC
:101A8000FFF750FF22460121BDE81040FC2049E746
:101A90004FF4807141EAD00254490B681A64544AE9
:101AA00042EA0022106000E000BF0868006C800578
:101AB000FAD470474D4A4FF4807141EAD001126860
:101AC00011644B4941EA00200068704708227020E9
:101AD00000213AE700227020114636E743480168AA
:101AE000496E026821F4007151660168496E02680E
:101AF00041F4807151660168496E026841F4806169
:101B000051660168496E006821F480614166E1E731
:101B100036480168496E026841F480615166016887
:101B2000496E026821F4806151660168496E02685D
:101B300021F4807151660168496E006841F40071BA
:101B40004166704729480168496E026841F4806126
:101B500051660168496E006821F4806141667047F2
:101B600000B50021DE20FFF7C7FE0121DE205DF871
:101B700004EBC1E610B5204C2068C068204908601D
:101B800020494FF6FF70096808602068C068C006E9
:101B900007D5FFF7E5FF20688068216840F0100056
:101BA00088602068C068000705D5206880682168C3
:101BB00040F0080088602068C06840070AD52068A7
:101BC0008068216840F004008860FF2200217020B6
:101BD000FFF7BBFE2068C068C00705D0206880689A
:101BE000216840F00100886010BD00000CA91100C0
:101BF00000F000406C0500202CA911002222A260F8
:101C000000070020F8A81100704770B5FC4D04468D
:101C1000C0F30741286801F0BEF8C4F30721286823
:101C200001F0B9F8E1B22868BDE8704001F0B3B83E
:101C30002DE9F041F34F0446154638680E46806A98
:101C4000396840F003008862DFF8B4830321D8F8D4
:101C5000000001F0A0F82046FFF7D7FF002405E0C0
:101C6000D8F8000001F0B5F83055641CAC42F7D349
:101C70003868806A396820F0030088620120BDE876
:101C8000F08170B514460D46064601F06BF9224608
:101C900029463046BDE87040CAE710B50422DA494B
:101CA0000020FFF7EEFFD8490422091D1046FFF778
:101CB000E8FFD549042208310820FFF7E2FFD249A6
:101CC00004220C312020FFF7DCFFCF490422103121
:101CD0002420FFF7D6FFCC49042214312820FFF737
:101CE000D0FFC94904221831C848FFF7CAFFC649C6
:101CF000C64804221C31001DFFF7C3FFC249C34878
:101D0000042220310830FFF7BCFFBF494FF4FC30FC
:101D100004222431FFF7B5FFBB4904222831BC4817
:101D2000FFF7AFFFB849BA4804222C310C30FFF757
:101D3000A8FFB549B648042230311030FFF7A1FFA3
:101D4000B149B348042234311430FFF79AFFAE4949
:101D5000AF48042238311830FFF793FFAA49AC4846
:101D600004223C311C30FFF78CFFBDE81040A9482D
:101D70000122A94985E77047F8B50E4605460024BB
:101D800015E0042269462846FFF752FF9DF800003F
:101D90009DF801109DF8032008409DF802101140A5
:101DA0000840FF2801D00020F8BD641C2D1DB4425E
:101DB000E7D30120F8BD2DE9F84390460C460746CD
:101DC000002501F0CFF80026E94612E0042269461A
:101DD0003846FFF72DFF00204946235C0A5C9A42F3
:101DE00001D06D1CADB2401C0428F6D3241D761C16
:101DF0003F1D4645EAD315B10020BDE8F883012018
:101E0000FBE70120704770B57E4C05462068806A6C
:101E1000216840F003008862794E0521306800F0A7
:101E2000BAFF306800F0D5FF2168896A226821F086
:101E3000030191622870012070BD08B56846FFF764
:101E4000E2FF9DF80000C00700D0012008BD10B5DA
:101E50006C4C2068806A216840F003008862684802
:101E60000621006800F097FF2068806A216820F052
:101E700003008862012010BD70B50546FFF7DDFF45
:101E800008B1022070BDFFF7E2FF5E4C2068806A57
:101E9000216840F00300886259482021006800F062
:101EA0007AFF2846FFF7B1FE2068806A216820F09B
:101EB0000300886201E000BF00BFFFF7BEFF0028FB
:101EC000F9D1012070BD70B50646032401F04AF82F
:101ED0004FF480653046FFF7CFFF29463046FFF7C5
:101EE0004BFF08B1012070BD201EA4F10104F1DCFC
:101EF000022070BD2DE9F04115460E460446FFF75D
:101F00009CFF08B10220BAE6FFF7A1FF3D4F3868F9
:101F1000806A396840F003008862DFF8E4800221BB
:101F2000D8F8000000F037FF2046FFF76EFE0024CF
:101F300005E0315DD8F8000000F02DFF641CAC42D4
:101F4000F7D33868806A396820F00300886201E0BE
:101F500000BF00BFFFF771FF0028F9D101208EE616
:101F60002DE9F043C1B00E46814603254FF480773A
:101F7000E84600F0F7FF3A4631464846FFF7BAFF19
:101F800000243A4669464846FFF752FE4046315D16
:101F9000025D8A4205D06D1EEBD2022041B0BDE841
:101FA000F083641CFF2CF2D90120F7E72DE9F04102
:101FB000194C8046134E124F6068C0B00D4640B1B8
:101FC000386800F0E8FE6068FF2827DA401C60608F
:101FD0003EE000F0C7FFFFF73AFF3068806A3168E3
:101FE00040F0030088620221386800F0D4FE4046C9
:101FF000FFF70BFE2946386800F0CDFE6068E5E784
:1020000028A911000CA911005816002068C0010071
:1020100004F8010004300300700500200020606017
:102020003068806A316820F00300886200244FF431
:10203000807269464046FFF7FBFD68462A5D015DF8
:10204000914202D0022040B019E6641CFF2CF5D961
:102050000120F8E770B50C46054600F083FFB4F5A3
:10206000807F0FD8F9490868806A096840F003004A
:102070008862F7480321006800F08DFE2846BDE81D
:102080007040C2E570BDF248006800F0A2BEEF48A3
:102090000168896A006821F003018162704770B5A8
:1020A0000C46054600F05EFF21462846BDE870401C
:1020B0004FF48072BCE570B5E44D04462868806A30
:1020C000296840F003008862E14E9F21306800F0EB
:1020D00062FE306800F07DFE2070306800F079FE0E
:1020E0006070306800F075FEA0702868806A29680A
:1020F00020F003008862012070BD10B5044600F096
:1021000031FF2046FFF7D7FF012010BD2DE9F04732
:10211000DFF8389304461746D9F800008846806AED
:10212000D9F8001040F003008862C94D03212868E7
:1021300000F031FE2046FFF768FD002415E0286816
:1021400000F047FE0646286800F043FE46EA0026F7
:10215000286800F03EFE46EA0046286800F039FE96
:1021600046EA006048F82400641CB4EB970FE6D3FD
:10217000D9F80010896AD9F8000021F003018162C2
:102180000120BDE8F08770B514460D46064600F004
:10219000E9FE224629463046BDE87040B6E710B554
:1021A000FFF74BFE08B1022010BDFFF750FEA74C11
:1021B0002068806A216840F003008862A44860219A
:1021C000006800F0E8FD2068806A216820F00300C4
:1021D000886201E000BF00BFFFF72FFE0028F9D1A1
:1021E000012010BD10B500F0BDFEBDE81040D6E7DF
:1021F00070B50D46064600F0B5FE0024294630466F
:10220000FFF74DFF641C05F5807506F58076102CF0
:10221000F4D3012070BD70B50D46064600F0A2FE55
:10222000002429463046FFF79BFE022807D0641C95
:1022300005F5807506F58076102CF2D3012070BD6F
:102240002DE9F047ADF5804D054614460E460005D4
:102250004FF48058E9461FD0280B000382464946B8
:10226000FFF7C6FFC5F30B00C0F58057A74200D9A2
:10227000274648443A46314617F091F85046FFF752
:1022800022FE02283BD049465046FFF7C4FF0228F1
:1022900037D03D443E44E41B4F464246944215D35A
:1022A0003146384617F07BF82846FFF70CFE022827
:1022B00025D039462846FFF7AEFF022821D0A4F5E5
:1022C000805405F5805506F58056E6E79CB1394601
:1022D0002846FFF78DFF22463146384617F05FF853
:1022E0002846FFF7F0FD022809D039462846FFF7B7
:1022F00092FF022805D001200DF5804D41E70A200C
:10230000FAE70B20F8E710B5ADF5806D04466AB129
:10231000684617F044F82046FFF7D5FD022809D09B
:1023200069462046FFF71CFE022805D001200DF566
:10233000806D10BD0A20FAE70B20F8E770B506465D
:10234000FFF77BFD08B1022070BDFFF780FD3F4C19
:102350002068806A216840F0030088623C4D0121BA
:10236000286800F018FD3146286800F014FD206848
:10237000806A216820F00300886201E000BF00BF8E
:10238000FFF75BFD0028F9D1012070BD08B500F012
:10239000E9FD6846FFF737FD9DF8000040F040007A
:1023A0008DF80000FFF7CAFF08BD70B50546002490
:1023B00004E0AC4201D9002070BD641CFFF73DFD74
:1023C0000028F6D1012070BD70B5204C054620686C
:1023D000806A216840F0030088621D4E0921306840
:1023E00000F0D9FC306800F0F4FC2168896A2268AA
:1023F00021F0030191622870012070BD38B5FFF70C
:102400001CFD38BBFFF723FD104C2068806A216853
:1024100040F0030088620E482F21006800F0BBFCEA
:102420002068806A216820F00300886201E000BF14
:1024300000BFFFF702FD0028F9D16846FFF7C4FF8F
:102440009DF80000800706D5012038BD0CA91100B9
:1024500028A91100FFE70220F7E74A4810B5042138
:10246000006800F098FC012010BD70B5FFF7E5FC96
:1024700008B1022070BD444C2068806A216840F099
:10248000030088623F4D0521286800F084FC28681D
:1024900000F09FFC06462068806A216820F0030057
:1024A00088622068806A216840F003008862FFF734
:1024B000CEFC0121286800F06EFC26F0400128685F
:1024C00000F069FC2068806A216820F003008862BF
:1024D000012070BD70B50546FFF7AFFC08B10220C2
:1024E00070BDFFF7B4FC284C2068806A216840F07A
:1024F0000300886223485221006800F04CFC284603
:10250000FFF783FB2068806A216820F0030088625F
:1025100001E000BF00BFFFF790FC0028F9D10120C7
:1025200070BD10B50446FFF788FC08B1022010BD4D
:10253000FFF78DFC1348D821006800F02CFC2046E2
:10254000FFF763FB10480168896A006821F0030106
:10255000816201E000BF00BFFFF76FFC0028F9D1E6
:10256000012010BD074810B5B921006800F013FC28
:10257000012010BD034810B5AB21006800F00BFC32
:10258000012010BD28A911000CA9110001218140D2
:1025900030480268114301602F48006801607047AD
:1025A0002C49012282400868904308602A49096842
:1025B0000860704727490968C14001F00100704771
:1025C00000B50246FFF7F6FF0028104602D05DF87E
:1025D00004EBE5E75DF804EBD8E71F4909680968F3
:1025E000C14001F0010070471B490A68526801238D
:1025F000834008681A434260704717490A68526866
:102600000123834008689A434260704712490A6870
:10261000126A0123834008681A43026270470E4918
:102620000A68126A0123834008689A43026270476D
:1026300000B50020FFF7D8FF0120FFF7D5FF0020ED
:10264000FFF7A4FF0120FFF7A1FF0449012009685B
:10265000C86000BD7805002004A911000CA9110074
:1026600070477047964810B502683F21D1600268F4
:10267000002191640068C0F8B41003210A2000F022
:1026800070F9BDE810400A2000F08DB98C4A13683B
:102690001860136859604843116888607047884A19
:1026A00013681860136859604843C10700D0401C84
:1026B00011688860704782490968C1F8B4007047A2
:1026C0007F4900B101200968886470477C4801682F
:1026D000C968006841F00201C160704730B5784CAC
:1026E0002568286220684162206882622068C3628F
:1026F00021680120086303E000BF00BF00BF00BFE6
:102700002068406BC107F7D140F3400030BD6C48F2
:102710000168C968006821F00201C160704768481B
:102720000168C968006841F00101C1607047644BED
:1027300010B51C68206218684162186882621968C6
:102740000120086403E000BF00BF00BF00BF18689D
:10275000406CC107F7D110F0060000D0481E10BD34
:1027600057480168C968006821F00101C1607047DD
:1027700053480168C968006841F00401C1607047AE
:10278000027C017B02F03F0241EA02414C4A13689D
:102790009965136801685962136841689962136802
:1027A0008168D96213680121196503E000BF00BF89
:1027B00000BF00BF1168496DCB07F7D11368DB6D0F
:1027C00083821368DB6D1B0CC38213681B6E03834B
:1027D00013681B6E1B0C438313685B6E8383126844
:1027E000526EC2F30E42C28341F340007047344838
:1027F0000168C968006821F00401C1607047016880
:102800004FEA31422E490B68C3F89C200A684068A1
:10281000C2F8A0000868C068096840F02000C860DD
:102820007047274A136818621068416211680120D6
:10283000C1F8900003E000BF00BF00BF00BF1068F8
:10284000D0F89800C107F6D110F0060000D0481E5D
:1028500070471B480168C968006821F02001C16009
:10286000704717480168C968006841F01001C160ED
:10287000704730B5124C5B1F2568C5F88830236857
:102880001862206842622068816221680120C1F8D4
:10289000800003E000BF00BF00BF00BF2068D0F889
:1028A0008400C107F6D110F0060000D0481E30BDEC
:1028B00003480168C968006821F01001C1607047D1
:1028C00018A91100234810B5026801211166026899
:1028D00010215167026841F2060151660268002129
:1028E000916602680A21C2F8881002689021C2F835
:1028F00084100168D1F88410026841F00101C2F827
:10290000841002684FF4817111660068016603202B
:1029100000F049F80021032000F023F80E490220BE
:1029200009688862002010BD10B5032000F045F84A
:1029300008484FF480710268116602680021116630
:10294000006810218167002010BD04490020087034
:102950007047000008A9110014A911007C0500208F
:10296000704710B500F00303DC00FF22A2400524ED
:1029700004EBC303994000F00C03002808DA2E484A
:10298000006818444369114093430B43436110BDF1
:102990002A4800681844D0F80033114093430B4391
:1029A000C0F8003310BD00F01F0201219140234AFE
:1029B0004009126842F82010704700F01F02012100
:1029C00091401E4A4009126802EB8000C0F8801056
:1029D000704700F01F0201219140184A4009126817
:1029E00002EB8000C0F88011704714490968086044
:1029F000704712490968C1F8800070470F480068A5
:102A0000006870470D490968C1F8800170470A489D
:102A1000006880687047084A01461068806812683C
:102A200091607047044B1B689B6800F1100253F8DB
:102A3000220043F822107047FCA81100F8A81100EA
:102A40007047704770477047704770470020704765
:102A5000002070470020704770477047294A0146A0
:102A60001068116070477047274B996801B99860EA
:102A7000596819609A68C3E90120224B914209D92B
:102A8000814205D9824201D95A6070475860704727
:102A9000596070478142FBD88242F7D8F4E7194861
:102AA0004068704710B500F084F8184804210268A7
:102AB000C2F8881002684FF6FF71C2F88C1072B627
:102AC00000684FF40071016662B610BD72B60F481F
:102AD0004FF400310268116662B60068D0F8040253
:102AE00068B14FF6FF71081A0649094A8860A0F5D7
:102AF0000840B938904202D24FF00110C86000F08F
:102B00005DB80000800500209C1600201CA9110063
:102B1000372B1A001A4801684969026841F40071AC
:102B2000516101680969026821F0060111610168BB
:102B30000969006841F0100101617047104801689F
:102B40000969026821F006011161016809690268DA
:102B500041F00401116101680969006841F0100148
:102B6000016170470649096888607047BFF34F8F5D
:102B7000034904480968C860BFF34F8FFEE70000AF
:102B8000FCA811000400FA05022801D300207047B8
:102B90006E4B53F8202043F820101046704710B5B4
:102BA0000920FFF700FF0221BDE810400920FFF7D0
:102BB000D8BE674902200968086570476449022049
:102BC0000968486570470020704761480168096FCF
:102BD000890502D54FF4407101E04FF4807100681F
:102BE0000166704710B55A4C2168C96F8A074FF0CB
:102BF000010100D50321226851670521B0FBF1F0E6
:102C000022684FF405710009C2F8801017F0B8F877
:102C1000504A514B17F004F917F06EF82168C1F8CB
:102C20008400BDE81040D0E749480168096FC90534
:102C300002D54FF4407101E04FF400710068016665
:102C4000704770B4424B1A68D26FD20701D003228A
:102C500000E002221C68626700EB4006C6EBC01071
:102C60004FF49675C1EBC0004D4300EB800005EBBF
:102C700040100A21B0FBF1F00521B0FBF1F0022475
:102C80000022E10302E04008521CD2B28842FAD28C
:102C900042EA04211A6841F01001C2F8881019684C
:102CA000C1F88C0070BCBFE729480168096F89032F
:102CB00002D54FF4403101E04FF4803100680166E5
:102CC000704723480168096FC90302D54FF44031AA
:102CD00001E04FF400310068016670471C4800684D
:102CE000006FC0F30020704719480068006FC0F300
:102CF00040207047164902220B681A650B680122B2
:102D00005A670B684FF40172C3F880200A68C2F852
:102D1000840009684FF480700866704705F0F1BFC1
:102D200010B506F03AF80A49044601200968C86659
:102D300001F0DEF8022805D1204605F0E2FF02206E
:102D400005F0BEFEBDE8104038E700009405002005
:102D50001CA911007B14AE47E17A843F70B50026B0
:102D6000DDE90445066001F00F0141EA85110160CB
:102D70000168D2B241EA0221016023F47F4101617E
:102D800010214160416804F0040211434FF6807243
:102D90009143416070BDC268D20700D08160C168B4
:102DA000C906FCD400E08168C1684907FBD47047BC
:102DB00010B5002305E0CC5C8460C468E406FCD454
:102DC0005B1C9342F7DB00E08168C1684907FBD4D4
:102DD00010BDFF22C168C906FCD48260C168C90663
:102DE000FCD4C1684907FCD58068C0B2704770B593
:102DF00014460D460646002304E03046FFF7E9FF7F
:102E0000E8545B1CA342F8DB70BD41684FF680724A
:102E100041F0020191434160704741684FF6827270
:102E20009143416070470000704702480068406865
:102E3000704770470CA91100244900200A6890606F
:102E40000968086022494860704710B51F4C216826
:102E500048602168002088600221401EFFF781FD44
:102E6000216807200860BDE8104005F025BE17491D
:102E700000200968086005F026BE154908707047F3
:102E800013480078704710B505F01DFE0F4900206B
:102E90000968086010BD0E488068704770B50C4C1A
:102EA000054600206080A0684FF47A71B0FBF1F015
:102EB000401EFFF7CAFF6188A942FCD3BDE87040FD
:102EC000D5E704494843024988607047F4A81100D7
:102ED0009C05002040420F00704770B52B4C054602
:102EE0004FF40D502168886621680320C866216868
:102EF0002748486621684CF2710008662168254819
:102F0000C1F88000216842F2463088660221002024
:102F1000FFF727FD0020FFF746FD002D06D02068B3
:102F2000806E42F2413108432168886670BD1748BF
:102F300010B502680121916700684FF40D51816658
:102F40000020FFF73AFDBDE810400020FFF741BD2B
:102F50000E4901200968486770470C49012009683B
:102F60008867704709494CF2710009680866704724
:102F7000064808B502684CF2710111660168096FD4
:102F80000268D1660068006F009008BD00A91100BA
:102F900007383937009C1C9110B500210A20FEF734
:102FA00089FD7C49887110BD024670200121FEF721
:102FB000CCBC024670200021FEF7C7BC2DE9F041D1
:102FC0000024264672201421FEF78AFC0546C0071D
:102FD00000D00124A80701D544F00204680701D5F8
:102FE00044F0040428070DD56B4844F00804016838
:102FF000D1F82C13006841F00401C0F82C13002014
:10300000FDF7E8FAE80601D544F01004614FA80680
:1030100006D544F0200400210A20FEF74BFDB871CC
:1030200014B12046FFF7C0FF280AC10700D01026C0
:10303000040AE0074FF0010507D046F020063D7076
:1030400000210A20FEF736FDB871200AC00702D021
:1030500046F040067D7016B13046FFF7AAFFB879FA
:103060009C2801D00020B870BDE8F081A6E710B51B
:1030700000210A20FEF71EFDC0B2002245499C280F
:1030800008D0C878401CC0B2C870032804D9CA70E0
:10309000012010BDCA700A70002010BD10B53D4C53
:1030A0006079401CC0B26071142817D900210A2031
:1030B000FEF700FDA279C0B2002182420CD06079F7
:1030C000401E60712079401CC0B22071032805D9D0
:1030D00021716171012010BD21716171002010BD4D
:1030E00010B5C9200021FEF7FBFB002010BD70B514
:1030F0007424002133222046FEF727FC01210D46CF
:103100002A462046FEF721FC02212A462046FEF7E9
:103110001CFC03212A462046FEF717FC70200121E3
:103120007722FEF712FC0C20FFF73DFC00210C205B
:10313000FFF717FCC82000211422FEF706FC154CEF
:1031400000200146A0700A20FEF7B4FCA07170BDFB
:1031500070B5FFF7A3FF20B10020FFF721FAFEF7BB
:10316000D7FC0C4C0025207840B1FFF780FF28B138
:1031700025700020FFF714FAFEF7CAFC60780028DB
:1031800007D065700020FFF70BFABDE87040FEF72E
:10319000BFBC70BDA805002010A9110070B5F84C87
:1031A00000254FF490662570A5703146F54816F05D
:1031B00097F93146F44816F093F93146F34816F082
:1031C0008FF96560E5708021F14816F089F9BDE856
:1031D0007040EF488021803016F082B9E848C0780E
:1031E000002800D001207047E5488078002800D0F2
:1031F0000120704770B50546E648E7490078097830
:1032000000FB01F4FFF742FADE492B46DF4A08468D
:10321000FFF764FA62002946DC4816F0C0F8D84986
:103220000120887070BD2DE9F0410746D9480E464F
:103230000478D948057800F05BFE022802D108F036
:1032400059FD38B16C43620031463846BDE8F04163
:1032500016F0A5B86400F6E770B505464FF4906423
:103260002146C84816F03CF92146C84816F038F9FE
:10327000C34C2946C3482278FFF7D5FF2278294658
:10328000BDE87040C148CEE72DE9F0411D46164625
:103290000F468046069C00F02BFE022803D108F062
:1032A00029FD00B90224FFF7DBF921462846FFF784
:1032B000F6F93A4631464046FFF739FABDE8F041A3
:1032C000FFF7CFB9AE4840687047B44A10B51278DE
:1032D00001469200AE4816F062F8A9490120C87074
:1032E00010BD2DE9F14FDFF898A2002488B09AF8BC
:1032F00002709AF803602546A146FEF714F8A84824
:103300000168496C026841F40061516400BF0168C2
:10331000496C006821F400614164A24902200968F7
:1033200008660020FDF714FCFDF757FEDFF87882F1
:1033300005F0C8F801280BD001A8FEF7ADF8002869
:10334000F6D001A805F011FB039830B11EB104E0DE
:103350004FF0010932E0FFF7B8FF029830B32FBBFE
:103360009AF800108346D1B9DAF80440BCB18A4813
:103370005A46214600780090864803785846FFF761
:1033800083FF98F80000022802D1204605F046FA93
:1033900098F80000092802D1584605F03FFA08982D
:1033A0000128584619D0FFF725FF0424FEF78EF8B0
:1033B0006D1CA542BCD3B9F1000F03D08AF802708E
:1033C0008AF803600120FDF77CFB7649022009683A
:1033D000086609B04846BDE8F08FFFF73DFF0124BD
:1033E000E4E710B5002000F05EFBBDE810400020CF
:1033F00077E708B50F2100F035FE012804D1FFF76B
:10340000F0FF009000F09FFEFFF7EEFE20B1FFF707
:10341000E5FE08B1012008BD002008BDE9E75848D5
:1034200000218170C17070475648704756487047F8
:10343000F0B5584A0021534B1678544F0C460022E1
:1034400012E033F9115030F911C0654553F81150AD
:1034500001DAAD1C00E0AD1E43F8115033F91150F4
:1034600047F81150491C521CB242EAD3641C022C8A
:10347000E5D3F0BD00B101204149887070472DE9C6
:10348000FC47DFF8FCA007001FD000254FF410799F
:103490002C4600F02DFD05281BD008F02BFCD0B1E8
:1034A000424C4348DFF80C810068D8F81410806B58
:1034B000FF3100F5E03021F0FF01503005FB01063F
:1034C00000F016FD022808D010E0CAF80470BDE82C
:1034D000FC870125E5E7384CE3E708F00BFC28B949
:1034E000D8F81400FF3020F0FF00064400F000FD83
:1034F000022802D108F0FEFB28B3002506F10108DE
:10350000012269463046FEF7BCFB08F10106404641
:10351000012201A9FEF7B5FB0198C1B2009861F341
:103520001F2000B2394627F815000CB124F8150009
:103530006D1C4D45E2D301222048FFF774FE1F4960
:10354000CAF80410C3E7402300200546294627F89F
:1035500010500CB124F81010401C9842F6D30122F0
:1035600039461748FFF75FFE1549E9E710B5012214
:103570000E491248FFF757FE01491048486010BD38
:10358000B0050020A8160020281B0020A81F00203E
:10359000282D0020BA050020BB050020C105002011
:1035A00010A911000CA911002D060020DC600020DC
:1035B000B8060020BC0600204C080020282400206B
:1035C000A828002010B5FA4C28B101460122F9487C
:1035D000FFF729FEF7486060D1E7F748704700B170
:1035E0000120F349C870704710B50246FFF717FF76
:1035F000104600F058FABDE81040002071E610B502
:103600000246FFF70CFF104600F04DFABDE81040EF
:10361000012066E610B54FF44C301422E749FEF75E
:1036200030FBE648ABE710B5FFF7F4FF0068A6E70C
:10363000F0E70268521C0BD0052936D023DC0129A3
:103640002BD002292BD003292BD0042923D12AE007
:10365000052916D008DC01291DD0022911D0032923
:103660000FD0042917D10CE0142906D0152904D055
:10367000162904D017290ED103E02D2070472820E9
:10368000704700207047142911D0152911D0162930
:1036900011D0172911D0FF20704700797047007AA8
:1036A0007047407A7047807A7047C07A7047007BD5
:1036B0007047407B7047807B7047C07B704730B558
:1036C000C5B0142140A815F00BFF4FF480752946B2
:1036D000684615F005FF4FF44C34142140A815F04E
:1036E000FFFEFF222946684615F0D0FE4BF6BB30A0
:1036F00040902D22FF208DF80C218DF804018DF8CB
:103700000D21282000218DF80E0142918DF80F1116
:10371000142240A9684615F087FE2046FEF771FB8B
:1037200069462046FEF71CFC45B030BD2DE9F0434C
:10373000C5B00C46DDE94C8905461E4617461421E6
:1037400040A815F0CDFE9E4804602868401C01D1B9
:10375000FFF7B5FF1422294640A815F065FE8DF845
:1037600008718DF809618DF80A81FF228DF80441F6
:103770008DF80B91511C684615F088FE142240A963
:10378000684615F051FE4FF44C342046FEF79BFB83
:1037900069462046FEF7E4FB012800D0002045B032
:1037A000BDE8F0832DE9F041C6B015460E46074648
:1037B0004FF00008FFF72EFF0446142140A815F033
:1037C0008FFE2068401C23D01422214640A815F00B
:1037D0002BFEFF22511C684615F058FE8DF80C7127
:1037E0008DF80D618DF80E5101208DF80F01142216
:1037F00040A9684615F018FE4FF44C342046FEF7F9
:1038000062FB69462046FEF7ABFB46B0BDE8F0819F
:103810004046FAE7F0B5664D0646ADF2045D00207D
:10382000C8246870FEF774F9FDF7DAFA06F0FAFAC0
:1038300064494FF4906201F5906015F0B0FD0020EE
:10384000FFF71DFE0120FFF7CFFE4FF4A061C6B1C8
:10385000684615F045FE0021684606F077FE5A4B93
:1038600000206A464FF4207632F8101033F81070BA
:10387000C91B09B222F81010A14211DD01206870A5
:1038800012E0514815F00AFE00214F4806F05EFE96
:103890004E4800780C2807D14B4804F0BFFF03E0E6
:1038A000401C00B2B042DFDB4948FFF7D5FCFEF711
:1038B00015F9FDF792FB0DF2045DF0BD2DE9FF5FF8
:1038C0004FF0000ADFF80C9142F20F755646FFF7F1
:1038D000A1FE044617210368FFF7ABFE84461421BE
:1038E0002046FFF7A6FE4BF6BB3140B28B4204D117
:1038F000BCF1000F0FD12D280DD02160FF202071C9
:10390000002020726072A072E0722D212173617319
:103910002821A173E07314212046FFF78AFE40B2EC
:10392000039015212046FFF784FE40B20290162135
:103930002046FFF77EFE40B2019016212046FFF799
:1039400078FE404240B20090FDF7E4FA80077DD552
:1039500021481C4A002390F800B02048ABF1010830
:10396000007819E0002114E001F1010C01FB00379F
:103970000CFB003C32F8177032F81CC0A7EB0C07A8
:103980003FB2002F00DA7F423FB2B74200DD3E4631
:10399000491C4145E8DB5B1C8342E3DB02998E4214
:1039A00001DD4AF0020A0027BC46A0F1010E2FE01B
:1039B000B005002028240020282D0020282E0020DB
:1039C00070050020A8160020683100202D06002078
:1039D000281B0020F1D8FFFFBB050020BA050020FE
:1039E000002111E00CFB001332F8138002EB4303BB
:1039F0005B88A8EB03031BB2002B00DA5B421BB20F
:103A0000BB4200DD1F46491C7145EBDB0CF1010C8C
:103A1000DC45E5DB03998F4201DD4AF0040A4FF0F3
:103A2000000C10E000230AE00CFB003132F9111009
:103A3000494500DD8946A94200DA0D465B1C8342F8
:103A4000F2DB0CF1010CDC45ECDB00E007E0019956
:103A5000894502DC0098854201DA4AF0080A68428A
:103A6000C0B209F0FF01CDE90010F3B2FAB251463D
:103A70002046FFF75BFE1D208DF8000041208DF8E9
:103A8000010000208DF802A08DF804008DF80300DD
:103A90008DF8050006226946072007F0A8FDBDE85D
:103AA000FF9F05487047054A0146107800B1012084
:103AB00001B1012111707047282F0020B0050020AE
:103AC0002DE9FF4F8BB00020089032200790404234
:103AD0000990002005900090FD4814460678FD48A6
:103AE0000078069000200290834681460190049061
:103AF000039000F0FDF9052805D01E25FFF794FC82
:103B0000824600275CE04625F8E7002254E007FBE8
:103B100006200B9980B231F910E0AE4503DD05991E
:103B2000491C09B2059134F91010A9420ADD009B25
:103B30005B1C1BB20093594504DDBBB2019393B2E9
:103B40008B46029301F5FA63B3F57A6F03D9049BB0
:103B50005B1C1BB2049319B9039B5B1C1BB2039340
:103B60003AF910C0BEF1000FACEB01031BB210DA42
:103B7000002B02DAC3F1000800E09846BCF1000F08
:103B800001DACCF1000CE04503DD0C9921F810E0DE
:103B900003E0002901DA2AF8103034F91010099BEB
:103BA000994203DA494505DA894603E00C99002376
:103BB00021F81030521C12B2B242A8DB7F1C3FB277
:103BC00006988742A1DB0798834506DDB9F100001E
:103BD00001DAC9F10000584516DC0598A0B100983B
:103BE00090B1701E059080B24FF00009009000F077
:103BF0007FF901464FF0FF30052909D0079A934518
:103C000001DD089971B1B6E000200FB0BDE8F08F7A
:103C100006994E430399B1EB660FF6DA0499002931
:103C2000F3DCA8E0DDE9012102FB061B864634F93E
:103C30001B2002EBD27072454FEA600000DA40426E
:103C400003B2019870431FFA80F8029801B20F4640
:103C50002EE008EB070080B2002A15DD34F910C011
:103C600004EB400030F9020CBCEB000C18D5002826
:103C70001ADAC0F1000C9C4502DB11E0A84215DA0B
:103C80007F1E1FFA87F941E010DA34F910C004EB07
:103C9000400030F9020CACEB000CBCF1000FE6DC8C
:103CA0000028EBDA4042E9E78446E4E77F1E3FB2B2
:103CB000012FCEDA2AE008EB010080B2002A16DDDF
:103CC00034F9107004EB4000B0F902003F1A18D428
:103CD00004E0474200E007469F4204DB002800DA88
:103CE0004042A84210DA491C88B2009011E00BDA79
:103CF00034F9107004EB4000B0F902003F1A002FB5
:103D0000ECDD0028E7DAE4E7491C09B205988142B6
:103D1000D1DB01981FFA8BF100FB069083B2DDE93D
:103D2000000202FB060086B23AF913203AF91100AC
:103D300034F8133034F81110D31A1DB23AF9163092
:103D400034F81640411A1C1B09B224B24E1B00D590
:103D50006E1A0D1B00D5651A71190CB2811A00D5A7
:103D6000111AC21A00D51A1A881800B2B0EB440F03
:103D700001DD704649E7012047E72DE9F05F564C29
:103D80008246002520682E4690F8241100296DD027
:103D9000B0F83001002869D0FDF771F92168A34619
:103DA00091F82411B0FBF1F201FB1200F0BB01F01D
:103DB00003FB5FEA000959D048480078102802D177
:103DC000484604F02BFD42480027394690F800C0D1
:103DD000404890F80080504615E030F9023B01243D
:103DE0000EE030F9022BD31A1BB2002B00DA5B4233
:103DF0001BB2BB4202DD1F460D4626461346641C1D
:103E00006445EEDB491C4145E7DBDBF80020B2F8F6
:103E10003001B8422ADC05FB0C600AEB40013AF89D
:103E2000103031F8021C591A09B200E01EE039F8CE
:103E3000104009EB400030F8020C201A081A00B2BA
:103E4000002801DA434200E00346002900DA494233
:103E50008B420BDA002800DA4042B2F83211884275
:103E600004DA01F0B3FA0020BDE8F09F0120FBE77F
:103E700070B515460E46044607F03CFF002C0ED1E7
:103E8000042807D0052805D01348006890F82400BE
:103E9000A84204D83046BDE87040FFF716BA70BD9E
:103EA00070B51546044607F025FF601C08D0002CAD
:103EB0000DD1002D0BD02846BDE87040FFF79AB910
:103EC000002D04D02846BDE87040FFF7C5B970BD8D
:103ED000BA050020BB050020FC0600202D060020AE
:103EE00010B506F007FA06F09FFA002010BD00009A
:103EF00099480078704798480078022803D0052830
:103F000003D00020704707F0F5BE05F02AB89249AB
:103F10000870704710B50446072C17D2DFE804F08C
:103F200014040811140D0900084600F01DF90BE0F7
:103F300051B1084607F0D3FE06E0084605F006F842
:103F400002E0084607F0B2FB8348047010BD8349C5
:103F500000200968B1F86410C90501D5FDF761BCFE
:103F600070477E4900200968B1F86410C90501D581
:103F7000FDF77EBC7047794900200968B1F86410EC
:103F8000490501D5FDF797BC70477349487800286B
:103F900001D0401E4870704710B572B6FEF7C7FFDB
:103FA000BDE81040FEF7E2BD10B56D48FDF729FFF2
:103FB000BDE81040F0E76848006970476648C0688F
:103FC000704765494861704763484069704710B55C
:103FD000FCF706FFFCF77BFAFCF7EFFDFCF7ACFD06
:103FE000FFF7C4FABDE81040FDF7A2BB10B5FCF71F
:103FF000F7FEFCF76CFAFCF7A3FCFCF79DFDBDE8AF
:104000001040FDF795BB30B5ADF2844D05464FF439
:104010009061684615F064FA4F4C2846256106F019
:104020008FF8E060D0B10278A2704178E1708378B7
:104030002371531C03F0FE0363710023E3712372A9
:104040001225A57104F10A052B706B70007860725F
:104050001046FDF79EF80DF2844D30BDFFF781FF4D
:104060000020F8E7F0B5ADF2CC4D0E4604464FF413
:104070009061684615F034FA374F20463C6106F0EF
:104080005FF8F860002857D00278BA70417804468B
:10409000F97080783871501C00F0FE0078710020B3
:1040A000F87138721223BB7107F10A031870587047
:1040B000207878721046FDF76CF80DF59061204677
:1040C00006F05FF8608A7D6908B145432D0B00203A
:1040D000710700D50620310701D540F00200626A61
:1040E0000DF598610240DDF88004CDF8C004DDF8DC
:1040F0009C04CDF8C404DDF89004CDF8C804104643
:10410000FCF7EFFEDDF88C0420B12B46FA78B97885
:1041100005F039FB6421284605F0D8FBFFF7EBFEDC
:1041200002280DD06846FFF7AAF9002001F043F9F4
:1041300001200DF2CC4DF0BDFFF713FF0020F8E792
:10414000DDF89404EFE710B5FCF7DCFE024900202F
:10415000C860012010BD0000B8050020FC0600204A
:1041600000FE1100FE487047FE4948707047FD4848
:104170004078704710B5FC4CFC4A204621689142BB
:1041800006D14168B1F5887F02D801F037F900B156
:104190000024204610BD4FF4FC30FDF794BE70B5EE
:1041A0000D460446FFF7E6FF010004D0302220460A
:1041B00015F03AF917E0FF223021204615F066F994
:1041C000EA4820604FF4887060603020A0600020D2
:1041D000AA21C4E903016061A061E061401EE062C0
:1041E000A062606220623DB94FF4FC30FDF76BFEC7
:1041F0002021DF4815F074F9012070BDD949012054
:1042000048707047D74900200870704770B5ADF509
:10421000107D0446FFF7D2FE0546A0070AD5042606
:10422000FFF769FE48B1D34C95F92C102246304671
:1042300005F0BDFF0DF5107D70BD6C462046FDF705
:1042400049F9F1E770B50D4606461024FFF7B6FEB2
:10425000B10700D505242A46102C09D2002A07D020
:10426000204490F928102046BDE8704005F09FBF1B
:1042700070BD2DE9F05F002480464FF0120A4FF028
:10428000200B2746FFF734FE022802D107F032FD4B
:1042900030B1FFF72DFE052804D104F062FE08B905
:1042A0004FF0020A00254FF0030970E000266BE092
:1042B000FFF71EFE022802D107F01CFD50B1FFF7E8
:1042C00017FE052802D104F04CFE18B1032D21D2AF
:1042D00014243AE0ADB12424A74209D0A64821090C
:1042E00027460068C16104F00F017F20FCF79CF8AD
:1042F0002009012807D0681EB0FBF9F209FB120063
:1043000038E01424E8E7B5FBF9F109FB115006EB9E
:10431000401033E0E81E032801D2152415E0A81F41
:10432000032801D2162410E0A5F10900032801D2C8
:1043300024240AE0A5F10C00032801D2252404E07E
:10434000A5F10F00032800D22624A7420AD08A48EC
:10435000C4F3031127460068C16104F00F017F20F8
:10436000FCF762F8C4F303100128CCD0B5FBF9F1D7
:1043700009FB1150C6F11F0101EB401018F8011B99
:10438000C0B2FCF751F8761C5E4591D36D1C5545C3
:104390008CD3BDE8F09F2DE9F84F804671484FF06F
:1043A000000B0C46B0F904704FF0120A4FF02009D0
:1043B00058460091FCF7E6FE0646C8F10705FFF7F0
:1043C00097FD022802D107F095FC30B1FFF790FD70
:1043D000052804D104F0C5FD08B94FF0020AB8F170
:1043E000000F05D0002D4ADB00234FF0010C3EE00A
:1043F000002212E000210DE036F8023B2078DB1BA2
:104400001BB2502B01DD40F0800040F0400004F86A
:10441000010B491C4945EFD3521C5245EAD328E011
:10442000002221E036F8021B2078C91B09B25FEA9E
:10443000D01806D000290CDA45B911F1280F05DB98
:104440000FE0002905DD0DB928290ADD0CFA05F178
:104450008843002D05DDA5F101080CFA08F10143A0
:10446000C8B204F8010B521C4A45DBD35B1C534510
:10447000D6D30098FFF7FDFE0DB94FF0010B58465B
:10448000BDE8F88F37498880704770B5354E3A4996
:10449000F08009680320C8610425E9B27F20FBF79A
:1044A000C3FF0024B179E0B2FBF7BEFF04F12000A6
:1044B000B179C0B2FBF7B8FF04F14000B179C0B2E6
:1044C000FBF7B2FF641C202CECDB6D1C072DE4DB3A
:1044D00070BD2DE9F04387B00025FCF781FC26492B
:1044E0000720096808652548016841F0200101603E
:1044F0000020FFF7CAFFDFF86C804FF400604FF434
:104500001079A8F8040049461A4814F0E9FF002081
:10451000FCF71EFBFCF786FD00273C463E46FFF7F6
:10452000EAFC03F0CFFF01282FD06846FCF7B4FF68
:10453000A8B10120FCF70CFB684604F016FA7F1CBA
:10454000012F20D000270B492046FFF724FF072C1E
:104550002ED00020FCF7FCFAFCF7B8FF10E012E0C8
:1045600068360020D005002000F811005443524660
:104570007C160020A838002010A911006405002036
:10458000FCF750FD641C002DCBD0FFF7B4FCFE48B7
:10459000C8F80C00FD4B424600204C461F5CD16819
:1045A000401CA04201F8017BD160F7D36EB907E04F
:1045B00000F07BFF01284FF00105E6D00126E4E77B
:1045C0001DB1002007B0BDE8F0830120FAE770B507
:1045D000002420252046FCF7D5FD00214FF44D7323
:1045E00030F9022BA2F266629A4200D9641C491C7F
:1045F000B1EB450FF4D30CB1002070BD012070BDAC
:10460000F0B587B000260120FCF75BFAE0480168AE
:1046100041F0200101600020FFF737FFDD494FF432
:10462000006088804021DC4814F05AFF0020FCF72D
:104630008FFAFCF7F7FC00252C462F4603F042FFCB
:10464000012824D06846FCF727FFF0B10120FCF7D1
:104650007FFA6D1C012D13D00025CF492046FFF7AE
:104660009AFE072C06D00020FCF772FAFCF7DAFC61
:10467000641C0AE0FFF7ABFF01280DD1012606E01C
:104680000020FCF765FAFCF7CDFC002ED6D01FB950
:1046900016B1002007B0F0BD0120FBE72DE9F14F76
:1046A0004FF0000B82B0BD48CDF800B05C460078FA
:1046B000D9465D46022802D0052802D004E0012038
:1046C00001E0022404208146DFF8D4A2DFF8D4827E
:1046D00052E1204605F034FD002873D00689029887
:1046E000064040F233300642F7D0AF4F3868406999
:1046F000396840F40070486138680069396820F012
:104700000600086138680069396840F010000861E7
:1047100034B1012C33D0022C7ED0032C2ED152E0A8
:1047200002210846FFF7F6FB0120FCF7CAF905F065
:104730008AFB0F212046FFF795FC0028CDD0DAF840
:1047400000105046496CDAF8002041F400615164D1
:1047500000BF00BF00BF0168496CDAF8000021F417
:1047600000614164FCF777F905F05CFB012007F07C
:10477000DEFB0020FCF7ECF9FCF7A8FEA4E000212A
:104780000220FFF7C7FB0120FCF79BF90F21204611
:10479000FFF768FC0028A0D0DAF800105046496CFA
:1047A000DAF8002041F40061516400BF00BF00BF8F
:1047B0000168496CDAF8000021F400614164FCF7FB
:1047C0004AF981E0D7E000210520FFF7A3FBFCF7C1
:1047D00007FB38680069396820F00600086138680E
:1047E0000069396840F00400086138680069396878
:1047F00040F01000086113F0B7FD0F210220FFF711
:1048000031FC00289AD0D8F800100720474688606D
:104810000420D8F8001000E010E0486002212020B9
:10482000FCF7B7FC0020FCF793F9FCF7D6FB3868DF
:104830000068396840F00100086045E00221052069
:10484000FFF768FBFCF7CCFA38680069396820F09C
:104850000600086138680069396840F004000861A2
:1048600038680069396840F01000086113F07CFD79
:1048700005F0D8FA0F210320FFF7F4FB00287AD0C7
:10488000D8F800007F218160D8F800000221416043
:10489000DAF800005746406CDAF8001040F4006087
:1048A0004864012007F00EF93868406C396820F43C
:1048B00000604864FCF791FBD8F80000006840F005
:1048C0000101D8F8000001600098E8BBF00725D08E
:1048D0000120FCF7F6F80020FCF751F9FFF70BFB7D
:1048E00088B1FCF720FDFF210F20FFF7F2FD012129
:1048F00081430D430020FCF72BF90120FCF73FF921
:10490000009858B12BE0FCF70EFDFF210F20FFF7B8
:1049100077FE0121814345EA4105EBE716F0060FDA
:104920001DD0FFF7E8FA022819D1FEF737FC002066
:10493000FEF75AFE0120FCF7C4F8FEF775FD0146AC
:104940000220FFF77FFC00E011E0FEF76DFDFEF7AF
:1049500039FEFEF769FD4FF4906114F09FFD0220CF
:10496000FFF754FC114981F800B0FCF736FBFFF764
:10497000BFFAFFF7E8FB641C4C4503D200980028FF
:104980003FF4A7AE034913E068360020A8380020A2
:1049900064050020D0050020E83A0020250600200C
:1049A00010A9110014A91100FCA811003A07002059
:1049B00081F800B02846BDE8FE8F70B5FE48FF4D77
:1049C0008CB04678102000242870FFF791FA012857
:1049D00005D001222121072006F0E5FD70E0F8480E
:1049E0000068B0F93610B0F9340004F0DAFFB0070F
:1049F00045D52878002140F0200028706846FFF750
:104A0000CEFB0598401C059040F27770FFF746FEFC
:104A1000C0B2032805D078B1012817D0022820D0D1
:104A200029E04AF2A11004900698401C06902878CC
:104A3000012440F001001DE045F250000490079869
:104A4000401C0790287840F0020013E04AF2501012
:104A500004900698401C06902878012440F003003A
:104A600008E045F2A10004900798401C07902878C0
:104A700040F004002870684600F0CEFC0BE0F00720
:104A800009D0287840F04000287040F22220FFF73B
:104A900005FE00B10124FEF7C2FC44B132464021BC
:104AA000072006F080FD287840F0800007E0002213
:104AB0002121072006F077FD287840F08800287033
:104AC0000CB0BDE8704003F09BBB70B50C46BD490F
:104AD000054603200968C86101217F20FBF7A4FC7B
:104AE00000217520FBF7A0FC01217620FBF79CFC40
:104AF0007C210820FBF798FC00210920FBF794FC9F
:104B00003E210A20FBF790FC00210B20FBF78CFCD8
:104B100006210E20FBF788FCE1B22620FBF784FC7F
:104B2000E1B22720FBF780FCE1B22820FBF77CFCF8
:104B3000E1B22920FBF778FCE1B22A20FBF774FCF4
:104B4000E1B23020FBF770FCE1B23120FBF76CFCE6
:104B5000E1B23220FBF768FCE1B23320FBF764FCE2
:104B6000E1B23420FBF760FCE1B23620FBF75CFCDD
:104B7000E1B23720FBF758FCE1B23820FBF754FCD8
:104B8000E1B23920FBF750FCE1B23A20FBF74CFCD4
:104B9000E1B24020FBF748FCE1B24120FBF744FCC6
:104BA000E1B24220FBF740FCE1B24320FBF73CFCC2
:104BB000E1B24420FBF738FCE1B24620FBF734FCBD
:104BC000E1B24720FBF730FCE1B24820FBF72CFCB8
:104BD000E1B24920FBF728FCE1B24A20FBF724FCB4
:104BE000E1B25020FBF720FCE1B25120FBF71CFCA6
:104BF000E1B25220FBF718FCE1B25320FBF714FCA2
:104C0000E1B25420FBF710FCE1B25620FBF70CFC9C
:104C1000E1B25720FBF708FCE1B25820FBF704FC97
:104C2000E1B25920FBF700FCE1B25A20FBF7FCFB94
:104C3000E1B26020FBF7F8FBE1B26120FBF7F4FB87
:104C4000E1B26220FBF7F0FBE1B26320FBF7ECFB83
:104C5000E1B26420FBF7E8FBE1B26620FBF7E4FB7E
:104C6000E1B26720FBF7E0FBE1B26820FBF7DCFB79
:104C7000E1B26920FBF7D8FBE1B26A20FBF7D4FB75
:104C800002217F20FBF7D0FB6A210220FBF7CCFB3F
:104C90008E210420FBF7C8FB05210820FBF7C4FB8D
:104CA000F1210720FBF7C0FB15B1012D06D101E072
:104CB000042100E008210620FBF7B6FB03217F203A
:104CC000FBF7B2FB21211020FBF7AEFB00211120E6
:104CD000FBF7AAFB00211220FBF7A6FB0021132003
:104CE000FBF7A2FB00211420FBF79EFB00211520FF
:104CF000FBF79AFB01211620FBF796FB02211720F8
:104D0000FBF792FB00211820FBF78EFB00211920F6
:104D1000FBF78AFB00211A20FBF786FB00211B20F2
:104D2000FBF782FB01212020FBF77EFB20212120C5
:104D3000FBF77AFB00212220FBF776FB00212320E2
:104D4000FBF772FB00212420FBF76EFB00212520DE
:104D5000FBF76AFB01212620FBF766FB00212720D9
:104D6000FBF762FB02212820FBF75EFB00212920D4
:104D7000FBF75AFB00212A20FBF756FB00212B20D2
:104D8000FBF752FB01213020FBF74EFB00213120C5
:104D9000FBF74AFB20213220FBF746FB00213320A2
:104DA000FBF742FB00213420FBF73EFB00213520BE
:104DB000FBF73AFB012107E0D0050020B1050020F8
:104DC000FC06002010A911003620FBF72DFB002166
:104DD0003720FBF729FB00213820FBF725FB0221B8
:104DE0003920FBF721FB00213A20FBF71DFB0021B6
:104DF0003B20FBF719FB01214020FBF715FB0021AD
:104E00004120FBF711FB00214220FBF70DFB202185
:104E10004320FBF709FB00214420FBF705FB0021A1
:104E20004520FBF701FB01214620FBF7FDFA00219D
:104E30004720FBF7F9FA00214820FBF7F5FA00219B
:104E40004920FBF7F1FA02214A20FBF7EDFA002195
:104E50004B20FBF7E9FA01215020FBF7E5FA00218E
:104E60005120FBF7E1FA00215220FBF7DDFA002187
:104E70005320FBF7D9FA20215420FBF7D5FABDE8DF
:104E8000704000215520FBF7CFBA10B50322FB4933
:104E900006287DD2DFE800F00324FDFCFBFA086859
:104EA000C26101217F20FBF7BFFAAF210820FBF789
:104EB000BBFA73210A20FBF7B7FA0A210E20FBF791
:104EC000B3FA02217F20FBF7AFFA00210720FBF79E
:104ED000ABFA1F210120FBF7A7FA1021062002E1FF
:104EE0000868C26101217F20FBF79EFA0F210E2086
:104EF000FBF79AFAAE210820FBF796FA8F210A20D9
:104F0000FBF792FA02217F20FBF78EFA712107202E
:104F1000FBF78AFA6A210220FBF786FA8E21042029
:104F2000FBF782FA03217F20FBF77EFA6121102034
:104F3000FBF77AFA00211120FBF776FA0021122004
:104F4000FBF772FA00211320FBF76EFA0021142000
:104F5000FBF76AFA00211520FBF766FA01211620FB
:104F6000FBF762FA06211720FBF75EFA00211820F2
:104F7000FBF75AFA00211920FBF756FA00211A20F4
:104F8000FBF752FA00211B20FBF74EFA012100E04B
:104F9000B9E02020FBF748FA60212120FBF744FA12
:104FA00000212220FBF740FA00212320FBF73CFAE6
:104FB00000212420FBF738FA00212520FBF734FAE2
:104FC00001212620FBF730FA00212720FBF72CFADD
:104FD00006212820FBF728FA00212920FBF724FAD4
:104FE00000212A20FBF720FA00212B20FBF71CFAD6
:104FF00001213020FBF718FA00213120FBF714FAC9
:1050000060213220FBF710FA00213320FBF70CFA65
:1050100000213420FBF708FA00213520FBF704FAC1
:1050200001213620FBF700FA00213720FBF7FCF9BD
:1050300000213820FBF7F8F906213920FBF7F4F9B5
:1050400000213A20FBF7F0F900213B20FBF7ECF9B7
:1050500001214020FBF7E8F900214120FBF7E4F9AA
:1050600000214220FBF7E0F960214320FBF7DCF947
:1050700000214420FBF7D8F900214520FBF7D4F9A3
:1050800001214620FBF7D0F9002103E036E033E0B0
:105090002FE02CE04720FBF7C7F900214820FBF761
:1050A000C3F900214920FBF7BFF906214A20FBF78D
:1050B000BBF900214B20FBF7B7F901215020FBF78A
:1050C000B3F900215120FBF7AFF900215220FBF783
:1050D000ABF900215320FBF7A7F960215420FBF71F
:1050E000A3F900215520BDE81040FBF79DB9AA2186
:1050F00000E05521002003E0AA2100E05521012015
:10510000BDE81040E1E410BD10B5FEF78DF904468E
:10511000FEF78CF92146BDE810404FF4906214F080
:105120003EB92DE9F0415648047856480578FEF717
:105130007DF90646FEF778F90746002013E000FBEC
:1051400004F206EB420C002107EB420207E0CB071A
:1051500003D03CF8113022F81130491CC9B2A142E9
:10516000F5D3401CC0B2A842E9D3BDE8F08100B538
:10517000ADF2844DFEF75AF901464FF4906268464D
:1051800014F00DF96846FEF767F80DF2844D00BD86
:105190002DE9F84F122000903C483B494FF0200A7F
:1051A00000244FF0030BC160032C01DA14251AE030
:1051B000E01E032801D2152515E0A01F032801D207
:1051C000162510E0A4F10900032801D224250AE0E5
:1051D000A4F10C00032801D2252504E0A4F10F005E
:1051E000032800D22625A9450AD02449C5F3031077
:1051F000A9460968C86105F00F017F20FBF714F983
:1052000000261FE094FBFBF1C5F3031001280BFB04
:1052100011401FD0C6F11F0101EB40101B4987B29E
:10522000C86810F8018BC860F8B24146FBF7FCF87B
:1052300000BF00BF00BF00BF00BFF8B24146FBF790
:10524000F3F8761C5645DDDB0098641C8442ABDB2A
:10525000BDE8F88F06EB4010E0E72DE9F84FDFF8E6
:105260002CB009491220CBF80C104FF0200A002472
:105270000090032C0CDA142525E0000010A9110081
:10528000BA050020BB05002068360020D0050020AC
:10529000E01E032801D2152515E0A01F032801D226
:1052A000162510E0A4F10900032801D224250AE004
:1052B000A4F10C00032801D2252504E0A4F10F007D
:1052C000032800D22625A9450AD09449C5F3031026
:1052D000A9460968C86105F00F017F20FBF7A4F813
:1052E0000026032194FBF1F001FB1047C5F30318DE
:1052F00010E0B8F1010F16D0C6F11F0000EB471007
:1053000080B2FBF7A9F8DBF80C10761C01F8010B52
:10531000CBF80C105645ECDB0098641C8442A8DBEB
:10532000DBF80C0094E706EB4710E9E77C48C088FF
:105330007047F0B5002587B02F46FBF751FD78493F
:105340004FF400608880FBF711FC0020FBF700FCA5
:1053500000245A262046FFF798F8FBF73EFE03F09C
:10536000B1F86846FCF798F8C0B1684603F0FDFA5A
:10537000FFF72DF901280DD0B44213D2FBF730FD11
:10538000A0B2641CFFF781F8FBF727FE06F0B2FC21
:1053900010B103E0012503E0FCF71FFB002DDED078
:1053A0003FB902E0FBF71CFD03E015B1002007B098
:1053B000F0BD0120FBE770475948816811B10178C1
:1053C000890701D400207047C06870475548544988
:1053D000006890F825218878401CC0B2887082420D
:1053E00005D20020887001210846FEF793BD704762
:1053F0004FF410724C494D4813F0D1BF024610B51E
:1054000000200146936803E052F82140491C2044E3
:10541000B1EB930FF8D310BD10B5C0B0044604F043
:105420007FFE40B181692162C16961624169A16207
:10543000C068E06205E04FF0FF30E062A0626062A9
:1054400020623B4820604FF4887060603020A0608C
:105450000020E0602046FFF7D1FF4042FF22E060DD
:10546000511C684614F012F830222146684613F0A9
:10547000DBFF4FF4FC306946FCF772FD01462D4816
:105480002268026062684260226982606269C2606A
:10549000A2690261E2694261226A8261012902D045
:1054A000002040B010BD0120FBE72DE9FC5F122079
:1054B0000090202001901A480027B0F90480384657
:1054C000FBF760FE0546B946002418E035F9026B8B
:1054D000404614F03EFC184A184B14F0A1FC8246DA
:1054E0008B46B6EB080001D5A8EB060014F031FCA2
:1054F00052465B4614F092FD00D27F1C641C01985A
:105500008442E3D3009909F101098945DCD317B13D
:105510000020BDE8FC9F0120FBE7000010A911005E
:10552000D0050020FC060020683600205C650020C5
:10553000544352467C1600209A9999999999C93FEB
:105540001FB55807069C04D003F00700022808D0B6
:1055500004E0012202A9112002F038FE002004B06C
:1055600010BDF94A507905280DD1D089A04201D249
:10557000401CD08180B2A04205D10020D081012002
:105580000870032050710120E9E71FB5580704D0C7
:1055900003F00700022807D004E0012202A911202D
:1055A00002F014FE0020DAE701200870D7E71FB5EB
:1055B000580704D003F00700022807D004E00122B6
:1055C00002A9112002F002FE0020C8E701200870A5
:1055D000C5E71FB5580704D003F00700022807D01D
:1055E00004E0012202A9112002F0F0FD0020B6E73C
:1055F00001200870B3E71FB5580704D003F0070077
:10560000022807D004E0012202A9112002F0DEFDE9
:105610000020A4E701200870A1E72DE9F0478A46A1
:1056200003F007040026C84D08998146012C0DD0CF
:1056300028465F07C089DFF814C300F10103DFF8D3
:1056400010839BB206D0022C17D000E0EE81002020
:10565000BDE8F087884202D2D8F800402254EB819E
:105660008B4226D1D8F80000D8F80010407809788D
:1056700000EB0120ACF80E001BE0BCF80E20D8F8BF
:105680000040120A88422270D8F800409CF80E2090
:10569000627005D2D8F80020125C89F80020EB81F6
:1056A000E889884205D10121EE818AF800100320A3
:1056B00068710120CCE71FB5580704D003F007003C
:1056C000022807D004E0012202A9112002F07EFD89
:1056D000002044E70120087041E71FB5580704D0B7
:1056E00003F00700022807D004E0012202A91120DC
:1056F00002F06CFD002032E7012008702FE71FB593
:10570000580704D003F00700022807D004E0012264
:1057100002A9112002F05AFD002020E701200870A4
:105720001DE71FB55807069C04D003F007000228A8
:1057300007D004E0012202A9112002F047FD002059
:105740000DE7814A507905280DD1D089A04201D2B8
:10575000401CD08180B2A04205D10020D081012020
:105760000870032050710120F9E60020704708B549
:1057700003F00700012806D18DF8000002466946B3
:105780000B2002F023FD002008BD08B503F0070040
:10579000012807D100208DF80000012269460B2066
:1057A00002F014FD002008BD10B503F00700012829
:1057B00001D1FEF7F1FB002010BD08B503F0070092
:1057C000012807D103208DF800000122694600203E
:1057D00002F0FCFC002008BD08B503F0070001281A
:1057E00007D103208DF8000001226946002002F055
:1057F000EDFC002008BDF0B503F007020024524B79
:10580000059D012A02D0022A07D004E00520587124
:10581000DC811C639C820020F0BD5A79052A11D1DD
:10582000DA89AA4206D24B4EB668D700FE4006700F
:10583000521CDA8190B2A84204D1DC8101200870A8
:10584000032058710120F0BD1FB5580708D19DF8FD
:105850000800F02806D0012202A9072002F0B6FCB9
:1058600000207CE6FEF797FCFAE71FB5580704D145
:10587000012202A9104602F0A9FC00206FE6F0B553
:1058800003F00706304F012E0CD05FEA437C324B09
:105890001C683B46DB8903F10105ADB205D0022E41
:1058A0000FD00CE00020F88109E013B1012B03D0E8
:1058B00004E084F8EB2001E084F8EA20FD81002078
:1058C000F0BD13B1012B04D008E094F8EB10017087
:1058D00004E094F8EA20027001200870FD810120A4
:1058E000F0BD70B503F00704174D012C06D05E071C
:1058F0002B46DB8905D0022C15D012E00020E88170
:105900000FE073B9AA71082A0BD2DFE802F004078E
:105910000704040404044FF4906001E04FF4107095
:10592000E862002070BD084AD26A13B1012B03D08F
:1059300005E0110A017002E00270012008705B1C92
:10594000EB81012070BD0000E80500206010002000
:1059500040A911007C160020FC060020F8B50F4677
:1059600003F007010026FF4C0546012906D020461A
:105970005B07C08906D0022926D01BE00520607194
:10598000E68117E0B0B9A2714FF49060A082401098
:10599000082A0FD2DFE802F00406080C10121416D1
:1059A000F14806E0F14900E0F1492163A08201E0FD
:1059B000F04820630020F8BDEF48FAE7EF48F8E729
:1059C000EF48F6E7EF48F4E76179052947D1236B03
:1059D000F3B3ED49096891F8EB20E249012A898A7D
:1059E00007D0032A05D0EC4688422CD2800717D076
:1059F00020E0884227D2C1070BD1DA49A279C989B0
:105A0000042A21F0010101D0E04A00E0E04A515EA1
:105A1000E16294F82C102970E16A090AE16210E051
:105A2000042261461846FCF72CF90098E062206BCE
:105A3000001D206394F82C002870E06A000AE062E0
:105A4000E089401CE081E089A18A884207D100E01A
:105A500005E0E68101202663387003206071012093
:105A6000F8BD2DE9F843074603F007000026BD4CBA
:105A7000089D8846012802D0022806D002E00520B1
:105A80006071E6810020BDE8F883607905281CD1AB
:105A9000E089A84210D2FDF7C8F9AC208DF80000CB
:105AA0007A208DF8010070208DF80200E0891DF841
:105AB00000103970401CE08180B2A84205D101215C
:105AC000E68188F80010032060710120DBE72DE9F2
:105AD000FC41074603F007000025A24C089E8846BB
:105AE000012802D0022806D002E005206071E5817D
:105AF0000020BDE8FC816079052821D1E089B04211
:105B000015D2FDF792F953208DF8000045208DF84D
:105B100001007A208DF8020070208DF803008DF8C6
:105B20000450E0891DF800103970401CE08180B2FB
:105B3000B04205D10121E58188F800100320607191
:105B40000120D6E72DE9F04388B0894603F007012C
:105B50000027DFF810C20F9C012908D06246D289C5
:105B6000551CAEB2022906D0580729D032E00520D4
:105B70008CF805002CE09CF8051005291CD1A242E8
:105B80000ED2DFF8108200216B4618F801505D54E8
:105B9000491CC9B22029F8D3995C0170ACF80E6099
:105BA000BCF80E00A04207D10121ACF80E7089F8B4
:105BB000001003208CF80500012008B0BDE8F08338
:105BC000A24201D2ACF80E60BCF80E00A04201D196
:105BD000ACF80E700020F0E72DE9FE4781466A48D8
:105BE0008A460B99006803F007080026C28A848A57
:105BF0005C4FB8F1010F0BD038464FF0010CC08953
:105C0000451CADB2B8F1020F05D05A0733D03CE0C5
:105C10000520787138E07B79052B29D188421FD285
:105C2000130A8DF800308DF804308DF801208DF8BE
:105C300005204FEA142812228DF8082020228DF822
:105C400002808DF806808DF809208DF803408DF8CC
:105C500007408DF80A601DF8002089F80020FD81BA
:105C6000F889884204D1FE818AF800C00320787147
:105C70000120BDE8FE87484A884282F800C000D271
:105C8000FD81F889884200D1FE810020F1E72DE9ED
:105C9000FC47804603F007000026324C0A9D8946E7
:105CA000012802D0022806D002E005206071E681BA
:105CB0000020BDE8FC87607905282CD1E089012708
:105CC000A84220D20021B220FBF70AFE8DF8000086
:105CD000010A8DF80110010C8DF80210000E8DF8EC
:105CE00003007A208DF804001F208DF805000420A1
:105CF0008DF807008DF80670E0891DF8002088F8FF
:105D00000020401CE08180B2A84204D1E68189F8DD
:105D10000070032060710120CBE72DE9F8430746AE
:105D200003F0070000260F4C089D8846012802D08A
:105D3000022805D002E005206071E6810020A2E67D
:105D40006079052831D1E089A84208D26846FCF77D
:105D5000D4F9E0891DF800103970401CE08180B250
:105D6000A8421BE0E805002054B0020054D802000D
:105D700054DC020054C8020054D0020054C0020097
:105D800054B8020054EC0200FC0600200070002011
:105D900000780020283B00206C07002005D101215D
:105DA000E68188F800100320607101206BE630B5B1
:105DB00003F00701FE4C012905D05D07FD4B06D01D
:105DC00002290BD008E00020E081208204E0E08975
:105DD00019680A54401CE081002030BD218A1A68ED
:105DE000525C0270491C2182012030BDFEB503F0D7
:105DF000070201270025EF4CED4EDDF820C0012AF7
:105E000002D0022A7ED09AE0FDF70FF8012202A903
:105E100012200295FBF735FF0520707121687A206A
:105E2000087020684770216821208870E248226845
:105E30000168897CD17000682268017C1171017E43
:105E400049070CD5C18A2268090A51712268817DEF
:105E50009171818A2268090AD171007D0BE0818AE3
:105E60002268090A51712268017D9171C18A2268F4
:105E7000090AD171807D21680422087269461046A2
:105E80000095FBF7FEFE2168009848722268010A1F
:105E900091722268010C000ED172216804220873ED
:105EA000694614200095FBF7ECFE216800984873C2
:105EB0002268010A91732268010C000ED1732168D7
:105EC000087402980095E0B3042201A948200195C6
:105ED000FBF7D7FE019804225030019069461C3030
:105EE000FBF7CFFE2168009848742268010A91747C
:105EF0002268010C000ED1742168042208750095F7
:105F000001A900E035E048200195FBF7BAFE0198B1
:105F100004225030019069462C30FBF7B2FE216814
:105F2000009848752268010A91752268010C000EDC
:105F3000D175216808762168FF204876F581002018
:105F4000FEBDFFE7042269469C48FBF79AFE2168E4
:105F5000009848742268010A91742268010C000EAE
:105F6000D174216804220875944869461030009560
:105F7000D3E77279052A0ED1F289624504D22368EB
:105F80009B5C0370521CF28190B2604503D1F58195
:105F90000F70032070710120D2E770B503F0070580
:105FA0000024844B824E049A012D02D0022D30D061
:105FB0002DE0022070718248F4810168880A454210
:105FC00011EB852500D0401C404201EB8000C01C35
:105FD00020F003007B49B0F5003F014410D8CD7894
:105FE000086865F31F60784DA84209D1002004E0DD
:105FF0000C181D6824792C54401C9042F8D306E0FC
:10600000002002E019680C54401C9042FAD3002092
:1060100098E47579022D0FD1F589954204D21B6859
:106020005B5D03706D1CF581A8B2904204D1F481D0
:106030000120087003207071012083E4F8B503F09B
:1060400007025C4C00265A4B069D012A02D0022A08
:106050006DD06AE0022058715C48DE8100685C49BE
:1060600088422BD15B480168226811700168226860
:10607000090A517001682268090C91700168226850
:10608000090ED17041682268117141682268090ABD
:10609000517141682268090C917141682268090EAA
:1060A000D17181682268117281682268090A51726F
:1060B00081682268090C9172806833E00422694685
:1060C00020200096FBF7DDFD21680098042208706F
:1060D00000982168000A487000982168000C8870B8
:1060E00000982168000EC87069462420FBF7C9FD9E
:1060F0002168009808712268010A51712268010C18
:10610000000E917121680422C87169462820FBF7AE
:10611000B8FD2168009808722268010A517222684D
:10612000010C91722168000EC8720020F8BD5A79E6
:10613000022A0FD1DA89AA4204D22468A45C04702E
:10614000521CDA8190B2A84204D1DE81012008708D
:10615000032058710120F8BD70B503F00702002636
:10616000144C134B049D012A02D0022A0DD008E0E2
:1061700002205871DE8103F097FF20B18020216852
:106180000870002044E74020F9E75A79022A24D118
:10619000DA89AA4204D22468A45C0470521CDA8111
:1061A00090B2A84219D1DE8101200870032013E0CB
:1061B000E805002040A91100FC0600205CC0010099
:1061C00000FE1100E8FF0F0034CD12AB581600207E
:1061D00054464953641600205871012018E770B5E1
:1061E00003F007020026FE4CFE4B049D012A02D05C
:1061F000022A10D00DE002205871DE810020FCF749
:10620000ECF905460120FCF7E8F9216845EA0010A1
:1062100008700020FCE65A79022A0FD1DA89AA42D6
:1062200004D22468A45C0470521CDA8190B2A842A3
:1062300004D1DE8101200870032058710120E7E6B7
:1062400070B503F007020025E54EE64B049C012AD9
:1062500002D0022A08D005E002205871DD813168A1
:10626000552008700020D3E65A79022A0FD1DA8926
:10627000A24204D23668B65C0670521CDA8190B233
:10628000A04204D1DD810120087003205871012053
:10629000BEE62DE9F84303F007020027D04EDFF8F1
:1062A0004483089C4FF00109012A02D0022A2AD017
:1062B00027E003F035FF8569022088F80500A8F87B
:1062C0000E70042269460020FBF7DBFCC6480099EB
:1062D00081420FD13168042081F800903168487004
:1062E000306885703168280AC87030684771306836
:1062F000877106E0002002E031680F54401CA04284
:10630000FAD300201BE598F80520022A13D1B8F82B
:106310000E20A24205D233689B5C0370521CA8F881
:106320000E2090B2A04206D1A8F80E7081F800901D
:10633000032088F80500012001E5F8B503F0070205
:10634000A74C0025A74E069F012A02D0022A72D030
:106350006EE003F0E5FE70B3A44801682268117096
:1063600001682268090A517001682268090C91705D
:1063700001682268090ED170416822681171416874
:106380002268090A517141682268090C91714168BB
:106390002268090ED17181682268117281682268B1
:1063A000090A517281682268090C9172806821681B
:1063B000000EC87239E0FFE7042269468C48009558
:1063C000FBF75FFC216800980422087000982168A0
:1063D000000A487000982168000C887000982168B5
:1063E000000EC87082486946001DFBF74AFC216810
:1063F000009808712268010A51712268010C000E90
:10640000917121680422C871794869460830FBF708
:1064100038FC2168009808722268010A51722268CB
:10642000010C9172010E2068C17202207071F58119
:106430000020F8BDFFE77279022A0FD1F289BA4233
:1064400004D223689B5C0370521CF28190B2B84264
:1064500004D1F58101200870032070710120E8E764
:10646000F8B503F007025E4C00265E4B069D012A3C
:1064700002D0022A4CD049E0022058715D48DE81EA
:106480000168594A91421BD14168226811704168E4
:106490002268090A517041680A0C21688A704168B3
:1064A0002268090ED17081682268117181682268A2
:1064B000090A517181682268090C9171806822E093
:1064C0000422694610460096FBF7DBFB2168009822
:1064D0000422087000982168000A4870009821681A
:1064E000000C887000982168000EC870694608206A
:1064F000FBF7C7FB2168009808712268010A5171F7
:106500002268010C91712168000EC871002090E78B
:106510005A79022A0FD1DA89AA4204D22468A45CEB
:106520000470521CDA8190B2A84204D1DE810120AD
:1065300008700320587101207BE72DE9FF4F85B0DB
:1065400003F00702DFF89CA0129C4FF0000B012A19
:1065500004D05B0708D0022A6CD067E002218AF8D9
:106560000510AAF80EB061E0079800244FF001086A
:106570004FF04009C00725D04027042202A9384621
:10658000FBF77FFB042203A94820FBF77AFB1A489C
:106590000299814248D100250BE007EB85000422D7
:1065A0006946FBF76EFB0098032D044400D10646B4
:1065B0006D1C0398B5EB900FEFD304B93446B8F1D6
:1065C000000F31D00798800728D50020042201A9A8
:1065D000FBF7D9FD04490198884225D1002518E030
:1065E00040A91100E80500205446495370160020C8
:1065F00068C001005816002054464353A8000422E6
:106600006946FBF7C0FD0098062D044400D10646FC
:106610006D1CB5EB990FF1D304B93446B8F1000FF6
:1066200002D0CAF82C4001E0CAF82CB0002009B012
:10663000BDE8F08F9AF805205346022A14D1DA8972
:10664000A24207D2C2F10305EE00DD6AF5400570F3
:10665000521CDA8190B2A04206D1A3F80EB00120FC
:10666000087003208AF805000120E0E710B503F068
:106670000700012804D1002211461E2001F0A6FDCA
:10668000002010BD70B5044603F00700FD4D0E4616
:10669000012804D0590705D0022819D016E000209F
:1066A000E88113E0E889F84B032801D219680A54FD
:1066B000401C80B2E881032808D1186890F90220B4
:1066C00090F9011090F90000FDF76CF800209FE4AC
:1066D000FCF7AEFFE98931B1012906D0022906D0C5
:1066E000032909D00EE0142102E0152100E0162153
:1066F000FCF79FFF207005E01721FCF79AFF207040
:1067000001203070E889401CE881012080E45A07AC
:1067100004D003F00702022A05D002E0D949002084
:10672000C88100207047D94A1268027001200870A1
:10673000704770B503F007020025D24B049C012A74
:1067400002D0022A07D004E005205871DD81202004
:10675000987100205CE45A79052A0ED1DA89A242A8
:1067600003D29E790670521CDA8190B2A04204D105
:10677000DD810120087003205871012048E42DE9D3
:10678000FC4703F0070C0026BF4CBE4D0A9F89460C
:10679000BCF1010F0BD029465FEA4378C98901F1AA
:1067A00001039BB211D0BCF1020F1FD01BE001A965
:1067B000684601F0C9FE05206871216801980870DB
:1067C000216800984870EE810DE0B94202D220683D
:1067D0004254EB81E889B84205D1EE812068017806
:1067E000407801F0A8FE0020BDE8FC876A79052A00
:1067F0000ED1B94203D22268515C0170EB81E88965
:10680000B84205D10121EE8189F80010032068719A
:106810000120E9E72DE9F04103F007000026994C3B
:10682000994D069F012802D0580706D040E0E68126
:1068300028680670286846703AE0E089B84203D2BA
:106840002B681A54401CE08180B2B84230D190A02D
:1068500001220068E6810A702968C2B20978914273
:1068600026D12968C0F307204978814220D11C2510
:1068700000244FF4801606EB0430FBF724FB0228BB
:1068800017D0641CE4B2AC42F5D3032500244FF4C6
:106890008E1606EB0430FBF716FB022809D0641CA9
:1068A000E4B2AC42F5D37B48FBF70DFB022800D0E5
:1068B0000020BDE8F08110B503F00700012801D1E8
:1068C00002F01AF9002010BD2DE9F04103F007068F
:1068D0006C4D012E07D05F072B46DC6ADB8908D0A0
:1068E000022E17D014E00020E88104F056FEE86282
:1068F0000EE013B1012B03D007E01002E86204E0C0
:1069000044EA0200E86204F041FEE889401CE881A4
:106910000020CEE713B1012B03D005E0210A01705E
:1069200002E00470012008705B1CEB810120C0E7CD
:1069300070B5064603F00700524C0D46012804D0FE
:10694000590704D002280CD009E0002006E0E089B5
:1069500010B9104611F011FDE089401CE0810020C3
:1069600010E411F007FD3070012028700AE470B5C2
:10697000054603F00700434C0E46012804D0590792
:1069800006D0022817D014E00020E081208210E019
:10699000E08910B1012803D008E01002E06205E0B0
:1069A000E06A1043E06280B2FDF76FFDE089401CB1
:1069B000E081002012E4208A02280CD2FEF7B6FC07
:1069C000218A11B1012903D005E0000A287002E0F4
:1069D000287001203070208A401C2082012019E498
:1069E00010B55C0704D003F00702022A08D005E0C6
:1069F0000AB1012000E0002008F022F9002010BDBB
:106A0000254A92F85420D20802700120087010BD67
:106A1000002070472DE9F04103F0070200261A4DCF
:106A2000184C069F012A02D0022A15D012E005F068
:106A3000D5F929680870FDF75BFA2968487003F0FA
:106A40000AFA29688870FDF756FA2968C870052087
:106A50006071E68100202CE76279052A0FD1E28976
:106A6000BA4204D22B689B5C0370521CE28190B244
:106A7000B84204D1E6810120087003206071012032
:106A800017E70000E805002040A91100700500206C
:106A900055AC000000FE11006010002070B50646E5
:106AA00003F007000D46022801D000200FE601F098
:106AB000A1FB08B1012400E0002401F09EFB08B115
:106AC000022200E000222243327001202870FEE5FD
:106AD00070B503F00703F94A0024F94D049E012B19
:106AE00002D0022B4AD037E0F6480168F64B9942B3
:106AF00034D14168B1F5887F30D8C168FF2902D20E
:106B0000C168C9B200E0FF21136819700169FF294B
:106B100002D20169C9B200E0FF21136859704169CE
:106B2000FF2902D24169C9B200E0FF2113689970C0
:106B300081681368090AD9708169136819718169BC
:106B40001368090A597181691368090C9971806980
:106B5000000E1168C871EC810020B8E5106804705F
:106B600010684470106884701168FF20C870116844
:106B700008711168487111688871EAE7EB89B342BE
:106B800004D21268D25C02705B1CEB8198B2B042F6
:106B900002D1EC8101200870012098E52DE9F04137
:106BA000074603F007000025C54C012802D0022843
:106BB00004D001E0E561E58100207AE6207FBF4E48
:106BC00000F00700E0812178014304D1306802F031
:106BD00019F801202070E089052800D3257031685C
:106BE000085C3870E069401CE061012061E670B526
:106BF00003F007020025B14BB14C049E012A02D0DC
:106C0000022A08D005E0186801F0FCFF0520607139
:106C1000E58100205BE56279052A0FD1E289B24265
:106C200004D21B689B5C0370521CE28190B2B0429C
:106C300004D1E5810120087003206071012046E540
:106C40002DE9F04103F0070200269D4D012A02D0F4
:106C5000022A11D00EE0052068710021EE8108465D
:106C600001F072FC4FF6FF7101EA4000688201F00A
:106C70008FFCA86100201CE66A79052A13D1EA89F5
:106C80006C8AA24205D2D3070FD0AB790370521C95
:106C9000EA8190B2A04206D1EE8101200870032063
:106CA000687101F083FC012003E6AF6922F0010363
:106CB000FB5A1F0A0770AB71E9E77FB506461C4611
:106CC0000D46580708D103F0EFF928B1012202A9B7
:106CD0001F2001F07BFA03E004F00700022802D035
:106CE000002004B0F3E401F0F3FC307001202870C0
:106CF000F7E72DE9F041064603F007000027704D45
:106D00008846012802D002280AD007E005206871D1
:106D1000EF810A20688201F03BFCA8610020C8E5F1
:106D20006879052816D1E889698A884206D2C007A1
:106D300012D0A8793070E889401CE881698A80B255
:106D4000884207D1EF81012188F800100320687183
:106D500001F02CFC0120ACE5002401F0B9FC012875
:106D600004D1E889A96920F001000C5A200A30708A
:106D7000AC71E0E77FB505460C46580704D003F038
:106D80000700022807D004E0012202A90A2001F02E
:106D90001DFA0020A5E705F021F8287001202070D9
:106DA0009FE7F8B5074603F007000025444C0E4660
:106DB000012802D002280ED00BE00520607103F0FC
:106DC00072FB206318B144F26440A08200E0A58207
:106DD000E5810020F8BD6079052821D1E089A28AEB
:106DE0006946904213D2800708D10422206BFAF73B
:106DF00048FF0098E062206B001D206394F82C008F
:106E00003870E06A000AE062E089401CE081A18AF3
:106E100080B2884204D1E581012030700320607186
:106E20000120F8BD10B55C0704D003F00702022A68
:106E30000DD00AE0012A01D022B106E00120FBF7C3
:106E4000A5FB02E00120FBF7ABFB002010BD1F4AB1
:106E50001268126802F0020202700120087010BD70
:106E600070B505460C46580704D003F00700022809
:106E700008D005E00AB1012000E0002001F00EFE7C
:106E8000002024E401F011FE08B1012200E00022FC
:106E90002A70012020701AE470B503F00700084D35
:106EA0001446012802D0580702D021E000201EE03D
:106EB000E88968B101280DD017E0000040A9110051
:106EC000E80500207C1600205443524604A9110016
:106ED000AA710AE0A879FBF787FBA8792040FBF7A5
:106EE00055FBA879A043FBF75BFBE889401CE881D0
:106EF00000200BE4F0B503F0070CF74D059FBCF143
:106F0000010F0CD05FEA437E2B46F44EDB8903F180
:106F10000104A4B206D0BCF1020F2DD02AE000205B
:106F2000E88127E0EE497F1EBB420868C25420D1A9
:106F30000868007830B101280AD002280ED0032852
:106F400017D111E008683168407881F8800110E0BD
:106F500008683168407881F881010AE00868316882
:106F6000407881F8820104E008683168407881F84F
:106F70008301EC810020F0BDD84A126813B1012BC7
:106F80000AD014E092F8801101F00F0392F88111F9
:106F900063F31F1101700AE092F8823192F88321A5
:106FA00003F00F0363F31F12027001200870EC81DD
:106FB0000120F0BD30B5CB4C5D0704D003F00702D3
:106FC000022A11D00EE0012A01D02AB10AE020687D
:106FD000806A20F0030003E02068806A40F003002C
:106FE00021688862002030BD2268926A0270012008
:106FF000087030BD70B503F007000025B64C0E4692
:10700000012802D0580705D01CE002206071E581FC
:10701000E56217E06079022814D1E089A18A8842EC
:1070200007D2B14811460068FBF7B5FEE089401C65
:10703000E081A18A80B2884204D1E58101203070CC
:107040000320607100208BE42DE9F041074603F036
:1070500007000025A04C0E46012802D0022805D0CA
:1070600002E002206071E581002022E460790228BC
:1070700014D1E189A08A814207D29B480068FBF7BE
:10708000A8FE3870E089401CE081E089A18A88422E
:1070900004D1E5810120307003206071012008E4F3
:1070A00070B503F007028C4C012A02D0022A21D0CD
:1070B0001EE003F0FBF90023B8B100F15401216395
:1070C0004168B1F5887F10F8201F08D342788D18E9
:1070D00001FB02518278C0781044084403E08078B4
:1070E0000A1801FB0020A08201E02363A382E38150
:1070F000002035E4E289A38A9A4204D2256BAD5C74
:107100000570521CE28190B2984201D101200870B2
:10711000012025E410B55C0704D003F00702022A21
:1071200005D002E0104601F04EFA002010BD6F4A73
:10713000127802700120087010BD1FB5580704D1E5
:10714000012202A9092001F041F8002004B010BD7D
:1071500070B503F007006049012802D0580703D03A
:1071600020E00020C8811DE0C8895D4C032801D2C1
:1071700023681A54401C80B2C881032812D1F9F741
:10718000AFFE2068B0F8010045BAF9F787FC0400AB
:1071900001D0F9F763FF29460020F9F70FFC0CB185
:1071A000F9F75EFF002005E470B503F007004A49D7
:1071B000012802D0580703D023E00020C88120E036
:1071C000C889474D022801D22B681A54401C80B24E
:1071D000C881022815D1F9F783FEF9F75FFC040096
:1071E00001D0F9F73BFF2868007818B1286840788B
:1071F000F9F7E8FB28684078F9F7E4FB0CB1F9F7F8
:107200002FFF002052E4580701D13348C2700020FC
:1072100070477FB505460C46580704D003F00700B9
:10722000022807D004E0012202A9102000F0CEFFBE
:10723000002056E504F04EFD08B1012200E00022D6
:107240002A70012020704CE57FB505460C46580792
:1072500004D003F00700022807D004E0012202A9AD
:10726000112000F0B3FF00203BE504F027FD28705B
:107270000120207035E570B503F007001649049C25
:10728000012802D0580703D017E00020C88114E07D
:10729000C889134B032801D21D682A54401C80B2B0
:1072A000C881A04209D118681968B0F801000978AE
:1072B00040BA00B209B9FDF7E5F8002007E470B55F
:1072C00003F007000449049C012802D058070FD09E
:1072D00021E00020C8811EE0E8050020FC06002017
:1072E00040A911000CA9110028A911002D060020A9
:1072F000C889F74B032801D21D682A54401C80B26C
:10730000C881A04207D11868B0F8010041BA1868D6
:107310000078FAF7A6F900201FE470B503F0070221
:10732000EC4C049D012A02D0022A07D004E0002080
:10733000E081FBF7B4FBE06200200EE4E289AA42A0
:1073400005D2C2F10303DE00E36AF3400370521C6E
:1073500090B2E081A84201D10120087001201CE414
:107360002DE9F04103F007040026DA4D0746012C11
:1073700004D0580706D0022C13D00EE0EE812E82E6
:10738000AE710AE0E88950B1D2490122891D12206C
:1073900000F01CFFE889401CE88100200DE4AA7180
:1073A000F8E7288A38B13E7001200870288A401C0E
:1073B000288201201AE404F071FD3870F6E770B5F8
:1073C00005460C46580704D003F00700022805D0F4
:1073D00002E010460BF097FB00201BE40BF096FB3D
:1073E00028700120207015E410B51446580710D1FC
:1073F000032C0ED8B84903200968C86102217F20F8
:10740000F9F712F8062000EB041140F21620F9F704
:107410000BF8002010BD70B5044658074FF0010569
:1074200004D003F0070002284DD04AE0AB49002009
:10743000122A096845D2DFE802F0090B0D2525253F
:10744000252A2D303336393B443F4243087738E014
:107450000D7736E0A04903200968C86101217F202B
:10746000F8F7E2FF15214FF48770F8F7DDFF75217B
:107470004FF48470F8F7D8FF4D214FF48570F8F77A
:10748000D3FF1EE00021D01E04F0CBFD19E0FAF777
:1074900025FB16E0FAF73CFB13E0F9F79EFD10E040
:1074A000F9F79EFC0DE001F0F9FC0AE0012000E094
:1074B000022004F02AFC04E0FDF7CFFE01E00220E8
:1074C00008860020DDE4834A854BD08910B101286D
:1074D00004D006E01968090A217002E01B682370D5
:1074E0000D70401CD0810120CBE403F00702794BE2
:1074F000012A02D0022A03D005E00220587102E0DE
:107500005A79022A01D000207047764A1278027018
:1075100001200870032058710120704770B514468F
:1075200058074CD103216C4A072C11D81068C1614F
:1075300002217F20F8F778FF0A2040EA041140F288
:107540000220F8F771FF04F188014FF4017034E074
:10755000A4F10805042D18D81068C16101217F200D
:10756000F8F762FF4FF48470052D28D2DFE805F0AC
:10757000030507090B0036211FE040211DE04A21C9
:107580001BE0542119E05E2117E0A4F10D00022850
:1075900015D81068C16101217F20F8F745FF4FF42D
:1075A00087700D2C04D00E2C04D00F2C07D103E0D3
:1075B000132102E0182100E01D21F8F735FF00201B
:1075C0005FE47FB505460C46580704D003F007007A
:1075D000022807D004E0012202A9062000F0F6FDEF
:1075E000002026E6FCF784FC02280AD003280CD0F1
:1075F00004280CD0052806D0FF2028700120207018
:1076000017E60020F9E70120F7E70220F5E703205D
:10761000F3E710B51046590701D104F0AFFB002085
:1076200010BD10B51046590701D104F0B0FB002081
:1076300010BD70B5054603F007000C46022801D0C6
:1076400000201EE404F0ACFB28700120207018E438
:10765000F0B503F0070200251E4B059C012A02D05D
:10766000022A0AD01DE0022058711F48DD816FF008
:107670007F410068081AD86213E05A79022A10D1B3
:10768000DA89A24205D2DE6AD700FE400670521C9B
:10769000DA8190B2A04204D1DD810120087003207C
:1076A00058710120F0BD580701D110480270002028
:1076B000704770B5114603F00700064C049A012884
:1076C00002D0580714D022E00020E0811FE0000023
:1076D00040A91100E805002010A91100FC060020B7
:1076E000700700202C060020A00500203205002095
:1076F000E089F94B904201D21D682954401C80B2A8
:10770000E081904203D10E20196800F05FFD002057
:1077100099E42DE9F04103F00706F04C012E07D063
:1077200025465F076B8A2D6B06D0022E20D016E00F
:107730000020E081208212E0E08990B1012812D07F
:10774000022813D0C11E994206D2217D0844C01ED2
:10775000C1B2E8B2FAF7F9F8E089401CE0810020F4
:1077600083E42263F8E7521C6282F5E7A282F3E722
:10777000FF22027063B1228A1544521CFF2D06D8E5
:10778000D74EAD5D05709A4201D10120087022826A
:1077900001206AE42DE9F04103F0070C0027CF4CEB
:1077A0001546BCF1010F0AD05FEA437E2346CC4E5A
:1077B0005A8A1B6B06D0BCF1020F23D016E0E7817A
:1077C000278213E0E08998B1012813D0C249801EB6
:1077D000904201D20F683D54401C904203D1096889
:1077E0009819FAF72DFDE089401CE08100203CE467
:1077F0002563F8E76D1CE8186582B0F5807FF2D943
:107800006782F0E7FF2505705AB1258A2B446D1C6D
:10781000FF2B05D89B5D0370954201D101200870B4
:107820002582012021E470B5114603F00700AB4C1E
:10783000049A012802D0580703D011E00020E0810B
:107840000EE0E089A44B904201D21D682954401CEF
:1078500080B2E081904203D10220196800F0B6FCAA
:10786000002046E470B5114603F007009B4C049AD3
:10787000012802D0580703D011E00020E0810EE07B
:10788000E089954B904201D21D682954401C80B27A
:10789000E081904203D10320196800F097FC00209A
:1078A00027E4580703D003F00700022801D0002086
:1078B0007047012070471FB5580704D1012202A963
:1078C000132000F083FC002040E410B503F0070013
:1078D0008249029C012802D0580706D018E00120F6
:1078E00048710020C881886211E0487901280FD1D1
:1078F000C889A04205D28B6A401C42EA03238B62EE
:10790000C88180B2A04203D103204871886A08630D
:10791000002010BD10B503F0070001246F490128B5
:1079200002D0580706D01CE04C710020C8810871B5
:10793000486216E04879012813D1C88928B1012886
:1079400006D0032302280BD107E00A71CC8108E09E
:10795000100248620220C88103E0486A104348626E
:107960004B71002010BD70B51546580718D15B4CFF
:10797000214620794B6A03280DD85A490968C86105
:10798000C3F307217F20F8F74FFD94F82400294620
:10799000F8F74AFD04E0001FD9B2C0B2F9F7D5FFED
:1079A00000202FE470B5044603F007000D460228BE
:1079B00001D0002026E44948484900794A6A032852
:1079C00003D891B2F8F7E8FC04E0001FD1B2C0B2CE
:1079D000F9F792FF20700120287013E403F00701EB
:1079E0003E48012902D0590703D003E00021C1819C
:1079F00000E0827200207047F8B503F00702002310
:107A0000354F364E012A02D0022A22D01FE0002430
:107A10000220009370714FF44835F38114E0042282
:107A200069462846FAF72DF93968009808550098F4
:107A3000010A38682044241D41700099090C8170A6
:107A40000099090EC1702D1DB07A8442E7DB002039
:107A5000F8BD7279022A11D1F289B47AA24204D215
:107A60003C68A45C0470521CF28190B2B27A9042DD
:107A700004D1F38101200870032070710120F8BD4A
:107A800010B503F007001549012802D0580703D0AC
:107A900015E00020C88112E0C8898C7A0E4BA04204
:107AA00003D21C682254401CC8818A7A80B290425A
:107AB00005D18A7A4FF448301968FAF7C1FB0020E3
:107AC00010BD1FB5580704D1012202A90D2000F0F6
:107AD0007DFB0020F8E6000040A91100E805002029
:107AE00000F0110010A91100580701D1F8484272A6
:107AF00000207047F8B503F007020027F54EDFF8C5
:107B0000D0C3012A02D0022A2CD029E09CF8090017
:107B1000002400EB40004FF4443101EB002502202B
:107B200000978CF80500ACF80E704FF41077ACF8A5
:107B30001470042269462846FAF7A3F831680098C1
:107B40002D1D08550098010A30682044241D4170FD
:107B50000099090C81700099090EC170BC42E8DBE4
:107B60000020F8BD9CF80520022A15D1BCF80E2093
:107B7000BCF814309A4205D23468A45C0470521CDC
:107B8000ACF80E2090B2984206D1ACF80E700120ED
:107B9000087003208CF805000120F8BD70B54FF483
:107BA00044314FF4407202FB00140120F8F789FFC2
:107BB000FDF753FBFCF7D6FA0546F9F70EFAC44970
:107BC0004FF4107220460C638A822946BDE870404B
:107BD000FAF736BB10B503F00700BD49029C012837
:107BE00002D0580706D018E0022048710020C88152
:107BF000C86212E0487902280FD1C889A04205D294
:107C0000CB6A401C42EA0323CB62C88180B2A04207
:107C100003D1888D888203204871002010BD70B583
:107C200003F007000025AA4C0E46012802D0580791
:107C300005D026E002206071E581E56221E06079EF
:107C400002281ED1E089A18A884211D2E16A401C33
:107C5000090A41EA0261E162E081800708D19C499A
:107C600004222C31206BFAF7EBFA206B001D206305
:107C7000E089A18A884204D1E58101203070032087
:107C8000607100201EE4F8B5074603F007000025E8
:107C90008F4C0E46012802D0022805D002E00220B7
:107CA0006071E5810020F8BD6079022821D1E0896A
:107CB000A18A884214D2800709D104226946206B28
:107CC000F9F7DFFF0098E062206B001D206394F855
:107CD0002C003870E06A000AE062E089401CE08114
:107CE000A18A80B2884204D1E5810120307003204E
:107CF00060710120F8BDF0B503F007020026744D55
:107D0000012A02D0022A05D002E002206871EE8129
:107D10000020F0BD6A79022A19D1EA89AC8AA24210
:107D20000DD2930703D12B6B80CBC5E90B7395F86C
:107D30002C300370E86A000A521CE862EA8190B2B3
:107D4000A04204D1EE810120087003206871012057
:107D5000F0BD70B503F0070000255D4C012802D08E
:107D6000580705D023E002206071E581E5621EE03E
:107D7000607902281BD1E089A38A98420FD2E66A73
:107D8000401C360A46EA0262E262E081800706D1C0
:107D9000206BB0F5002F00D30260001D2063E08946
:107DA000984204D1E5810120087003206071002011
:107DB00006E470B503F007050026454C012D04D0FC
:107DC0005B0704D0022D2ED01DE0E6811BE0042AC3
:107DD00020D007DC92B1012A13D0022A15D0032A41
:107DE0000AD115E0052A18D03B48102A006809D0AE
:107DF000112A14D0202A14D0A66204E04FF4801077
:107E000000E03648A06200201BE44FF48E10F9E732
:107E10003348F7E74FF42C30F4E73248F2E73248C2
:107E2000F0E7B430EEE7E289042A05D2C2F1030399
:107E3000DD00A36AEB400370521C90B2E08104287D
:107E400001D301200870012062E410B503F007009F
:107E5000012804D1002211460C2000F0B7F90020BF
:107E600010BD2DE9F0410E46054603F00700184C01
:107E70000699012806D05F072346DB8905D0022832
:107E800014D011E00020E0810EE0124D022B01D24F
:107E90002868C2545B1C98B2E081884204D1022257
:107EA0000520296800F092F9002059E413B1012B54
:107EB00004D008E0FCF71CF8287004E0FCF71BF87D
:107EC000287001203070E089401CE081012047E4E7
:107ED000E805002040A91100FC06002000FE11006A
:107EE00000F8110000F011006010002070B503F0E0
:107EF0000700AB4C012802D0580705D022E0002033
:107F0000A062E062A0711CE0A549E6898D79886ACB
:107F1000A918CBB2022E03D242EA0020A06206E0EA
:107F20009F49042EC96A04D242EA0120E062A3718B
:107F300005E0052E03D2AA4201D100F06BFFE089D3
:107F4000401CE08100208CE470B5954C2346E1890B
:107F50009A6A9B79022904D240EA02211844A1625C
:107F60000AE04FF48175A94208D28E4A1268114482
:107F700001F8020CA1790844A07107E0A94205D8D4
:107F8000984203D18849104600F066FFE089401C02
:107F9000E08166E410B503F007011046012902D024
:107FA000590706D007E07E49002088628871C881A1
:107FB00001E0FFF7C9FF002010BD10B510465907BA
:107FC00001D1FFF7C1FF002010BD70B503250024CB
:107FD0004FF48E1606EB0430F9F775FF022804D033
:107FE000641CE4B2AC42F5D301203AE470B503F06E
:107FF000070200256A4B049C012A02D0022A07D0FE
:1080000004E005205871DD81187A9871002028E479
:108010005A79052A0ED1DA89A24203D29E790670D6
:10802000521CDA8190B2A04204D1DD810120087097
:1080300003205871012014E42DE9F0415BA0069F54
:10804000046803F007000026554DDFF858C10128E9
:1080500002D0580708D027E0EE81DCF80000067057
:10806000DCF8000046701FE0E889B84204D2DCF872
:1080700000301A54401CE88180B2B84214D1EE811D
:1080800001270F70DCF80000E1B2007888420BD1C4
:10809000DCF80000C4F307214078884204D1FFF7E0
:1080A00094FF012802D02E720020FEE62F72EE719E
:1080B000FAE72DE9F041002103F007003A4E384C71
:1080C0000D46012802D058070CD067E06570A581E5
:1080D0002562A570002046F82050401CC0B2402800
:1080E000F9D35BE06078052801D2401C6070C0B213
:1080F00001281FD02A4B0228B3F816C01CD04DD936
:10810000A38963454AD2264F03F0030034374FF466
:108110008E1E3A5422485A1C6245006A0EEB00201B
:108120000ED10021491CC9B20429FBD31E49F9F71D
:1081300017FF2AE0100201E00CEB0200E0822DE0C4
:10814000DA43920721D1BB5C4FEAC20C03FA0CF36D
:10815000521C1943D2B2042AF5D3A27802F03F038D
:10816000521C46F82310D1B2A17040290DD10E49FE
:10817000F9F7F6FEA570206A401C2062002046F840
:108180002050401CC0B24028F9D3A089401C80B2C6
:10819000A081E18A884201D10120E071002084E6BB
:1081A000E805002040A91100483B002055AC000024
:1081B000D248002101704170C1700171CF4A084658
:1081C000921D1154401C0428FBD3704730B5CB4C92
:1081D00063780BB1002030BDE0702271C74B0020E6
:1081E0009B1D02E00D5C1D54401C9042FAD30120FF
:1081F000607030BDC14840787047C0488078704793
:10820000BE490020887070472DE9F05FDFF8EC92DE
:108210000024012589F8025099F8030009F10606A7
:10822000A246202829D2DFE800F0131E2930103A98
:10823000FE3D289BA0A4D323FD28B0BBBFC32828A4
:108240002828282828282828FCFBFBF7ADFEBDE0BD
:10825000FBF74EFE89F8050031784C460120FBF70C
:1082600059FEA570B2E0307802F01AF9012110E051
:1082700089F801A03078FFF791FC1EE17078317821
:1082800040EA012003F092FB17E1307803F014FC80
:1082900004210320FBF73EFE89F8025096E0717836
:1082A0003078E5E04FF00008AB460127594689F8E1
:1082B00002B089F801A099F80000E0BB357889F890
:1082C0000010E80617D50120F8F7FBFB0020F8F7AF
:1082D00056FCFBF710FE78B3F9F725F8FF210F20C5
:1082E000FCF7F7F8074645F001050020F8F730FCE9
:1082F0000120F8F744FCE8071CD0FAF74FFF0020F4
:10830000FBF772F90120F8F7DCFBFBF78DF801466B
:108310000220FBF797FF0220FBF778FFF8F75DFEDE
:10832000FBF782F8FBF74EF9FBF77EF84FF490610C
:1083300011F0B4F801E002E00BE089F800A089F840
:1083400002A0002F99D008F10108B8F1030FACDBAF
:10835000B3E0F8F7E8FFFF210F20FCF751F9C1E780
:108360003078401E01F07FFD30E0307803F03BFDB7
:108370002CE0307820B103F0C2FC0146022001E07D
:1083800000210320FBF7C6FD97E0307800B1012003
:1083900003F096FC307800B1012000F0C8FD8CE0BD
:1083A000307803F082FC11E0307803F035FD84E092
:1083B000307820B1012805D002287ED103E0504852
:1083C000F9F71FFD79E001F0A7FE57E0012474E002
:1083D00089F801A000273E4672B6FAF7F4FB48B1CF
:1083E000FAF77CFC0746FAF75FFCFAF77DFC0646D5
:1083F000FAF767FCF8F774FDF8F750FB8046F8F7DA
:10840000A5FEFAF723FB050001D0FAF71EFB4FF497
:108410001870FAF7F7FA62B63A49C1F800A003E01B
:1084200048E03DE02DE017E0F9F745FA72B6B8F103
:10843000000F03D0F8F754FDF8F7CFFDFAF7C3FBB0
:1084400028B10FB1FAF7C1FB0EB1FAF7EDFB0DB190
:10845000FAF7F9FA62B630E03078012806D002283F
:1084600009D003280AD00221084601E00221052094
:10847000FBF750FDAAE700210320F9E700210420C3
:10848000F6E73078717840EA0122B078F17800049C
:1084900040EA016002436221072003F084F80CE007
:1084A000F9F750FB0120F8F70CFBFBF707FAF8F798
:1084B00094FD8BE7307800F0FDF889F802A02046A3
:1084C000BDE8F09F70B50024FAF74CFD0B4D6878BD
:1084D000012806D1FFF798FE04462020E87000200E
:1084E0006870FBF705FD022802D101F04FFD00B9CD
:1084F0000CB1012070BD002070BD000020060020DE
:1085000000FE11006405002002460020022909D265
:108510004AB1012A06D101EB810000EBC100FE49FE
:1085200001EB0010704701EB410000EBC100FB497B
:1085300001EBC010704700FB01F2B2F5307F02D8AA
:10854000F74AC2E9020170470200F548806800D08E
:108550001060F34AD26801B10A605043704770B5A9
:10856000FAF74CFA00F008060820FAF742FAEC4C49
:108570002079002530B10120A0703046FAF735FA95
:10858000E57070BD207880F001002070A570F4E7E0
:10859000E34801210171007880F0010000EB400107
:1085A00001EBC000DD4901EBC0107047DC48827868
:1085B000002132B1C27822B9027882F00102027041
:1085C000817001717047D64910B54C7848701E28EB
:1085D00004D01F2804D00E2809D003E0002000E0BA
:1085E00001200870012003F017FC204610BD8120F7
:1085F000F9E7F0B5CA4F3C7804EB440505EBC40439
:10860000C64D05EBC414BD6803FB05F604EB460438
:108610008D4201D22E4600E00E46D7F80CC0ACEBDE
:108620000307974200D317461A44624511D8002326
:108630000DE0002204E030F812C024F812C0521CF1
:10864000B242F8D304EB450400EB41005B1CBB4293
:10865000EFD3F0BD70B51546B14A1C460E465378AF
:108660000499834216D10120D070012902D0022939
:1086700007D00CE0002322462946304600F097F947
:1086800005E00023224629463046FFF7B2FFBDE849
:10869000704064E770BD10B500280AD0A0490122DF
:1086A000CA70497800230821FFF7A3FFBDE81040F6
:1086B00055E710BD9A490128C87106D0002806D197
:1086C0004878242803D130207DE72420FCE7704738
:1086D0009348C0797047F0B5924C2468A669740736
:1086E00002D50127B74301E006F0010705680C68D1
:1086F0000FB11C1B641EB30701D5551B6D1E7207FD
:1087000002D504600D60F0BD05600C60F0BD2DE980
:10871000F043814683488BB00C460068007E4007DA
:1087200002D517460E4601E00F461646B108A7EBE4
:1087300097000591401E0691BA0800907908CDE98E
:1087400001210390A6EB960004927108401ECDE92A
:108750000710099033463A4605A96846FFF7BBFF64
:1087600005AD33463A46E84601A8291DFFF7B3FF99
:1087700033463A4607A902A8FFF7ADFF33463A460B
:1087800008A903A8FFF7A7FF33463A4609A904A89A
:10879000FFF7A1FF624800784F4600EB400101EB74
:1087A000C0005E4901EBC0160020814626F81090FB
:1087B00058F82010491E14E055F82020521E0AE0F7
:1087C00002FB041336F910C037F91330634501DD9D
:1087D00026F81030521C55F820305B1C9342EFD223
:1087E000491C58F82020521C8A42E5D2401C05281A
:1087F000DCD30BB0BDE8F08310B500280DD048499C
:108800000122CA704A78484B484902221B780978ED
:10881000FFF7EFFEBDE81040A1E610BD2DE9F041E5
:108820003F4E0121F17042490D783F490C78717833
:1088300026294FD2DFE801F0131A1A1A131A1A1A4E
:108840001A1A1A1A1A1A1A4E1A1E1E1E1A4E4E4EAC
:108850004E4E4E4E4E1A4E4E4E3F3F4E461A48B367
:1088600000232246294600F0CDF830E010B3002363
:10887000224623E02F480078012801D92E480478A9
:10888000F8F748FB800700D5641CFBF76BFC002160
:10889000224B65430CE010F8014B327802EB4207A3
:1088A00007EBC20203EBC21222F81140491C89B245
:1088B0008D42F0DC0BE050B10023A21C2946FFF7EB
:1088C00098FE04E018B122462946FFF720FFBDE8D4
:1088D000F04144E6BDE8F08111491E288A7988718B
:1088E00002D01F2802D003E0002000E001204871E0
:1088F0001046704770B50D4609490122CA700C4AEE
:1089000049781678084A2129147803D0222901D001
:10891000232929D128B311E0484A0020483F0020EC
:108920002C060020FC060020BB050020C10500200D
:10893000BA050020BC050020BE0500208DB1002333
:1089400022463146FFF755FE631C01222146284688
:10895000FFF74FFE05EB4400A31C01223146FFF751
:1089600048FEBDE87040FAE570BD10B5454C617831
:1089700011B94068FFF752FF6078112802D100203A
:10898000FFF74CFF6078122802D10020FFF746FF66
:108990006078132803D1FCF70FFDFFF73FFF6078E5
:1089A0001D2803D1BDE81040374837E710BDF0B5AA
:1089B000344D2C7804EB440606EBC404334E06EB2E
:1089C000C414AE6803FB06F704EB47048E4201D2E1
:1089D000374600E00F46ED68EB1A934200D21A4684
:1089E00000250CE0002304E010F803C024F813C0B5
:1089F0005B1CBB42F8D304EB460408446D1C954253
:108A0000F0D3F0BD2DE9F047984691460D46044657
:108A1000F8F7ACFB060011D01A4908788F6800EB14
:108A2000400202EBC000194AAF4202EBC01208FB41
:108A300007F002EB400008D2BC4607E043464A4636
:108A400029462046BDE8F047D3E5AC46CA6849460A
:108A5000A2EB0808C84500D3884600210EE000229A
:108A600005E0B35634F8133020F81230521C62453A
:108A7000F7D300EB470004EB4504491C4145EED316
:108A8000BDE8F0872C060020806B0020483F0020C6
:108A9000DD4908707047DC4800787047DA4908B152
:108AA000002000E0012088707047D748807808B126
:108AB0000020704701207047D3490120087170479A
:108AC000D1494870704710B5CF4C00202071A07874
:108AD000002810D0A06800280DD00120F9F760FD13
:108AE000E078002807D001206070BDE810404FF406
:108AF0002F60FAF7FFB810BD10B5C34CA07810B1C5
:108B00000120F9F743FD0020A060E0602061606172
:108B1000A06110BDF0E72DE9F0410446F9F76EFFC2
:108B200000F008070820F9F764FFB74DB7480026A2
:108B3000696900EBC100491C6961FF2900D96E61B8
:108B40002178017061784170A1788170E178C170FD
:108B50002179017161794171A1798171E179C171E5
:108B6000A969FF2902D8491CA96115E01D210170DE
:108B700001214170217881706178C170A178017103
:108B8000E1784171217981716179C1712869401C55
:108B90002861FF2800D92E61A86840F00100A86074
:108BA000A87808B1287910B1E878012803D101200C
:108BB000F9F7F6FCEE703846BDE8F041F9F715BF5D
:108BC00002460220117811F0030106D0012901D0DC
:108BD000022905D1104600F010B9104600F012B974
:108BE00070471CB5EC208DF8000001208DF80100C5
:108BF00000208DF802008DF8030001906846FFF711
:108C0000DFFF1CBD2DE9F0417F4E00250446B26810
:108C1000002A52D000200127F16807FA01F313421D
:108C200007D1491CF1600D2900D3F560401C0D28C7
:108C3000F2D3F16801B3754860388F40BA4300EB56
:108C4000C1000838B260317E0278227042786270CA
:108C50008278A270C278E2700279227142796271E0
:108C60008279A271C07901F03F0100F0C000014398
:108C7000E171B06898B117E0B3693746EBB163486A
:108C8000396900EBC100491C3961FF2900D93D61F8
:108C90005B1EBB61D7D122F00101B160D3E7B07890
:108CA00010B10120F9F772FCF068401CF0600D284B
:108CB00000D3F5600120BDE8F081B07810B101204B
:108CC000F9F764FC25706570A570E5702571657114
:108CD000A571E5710220EEE730B54B4900208A68A6
:108CE0008C69002A0CD001210D4605FA01F31342CC
:108CF00000D0401C491C0D29F7D3D10700D02044D7
:108D000030BD1CB501784278890102F00F0241EABA
:108D100082018DF80010418809098DF801108188C1
:108D200009098DF80210817801F00F02017962F3D0
:108D30001F118DF80310017A8DF80410417A8DF817
:108D40000510C179C02202EA0111827902F03F02C6
:108D500011438DF80610C07980018DF80700684630
:108D600000F04BF81CBD28484078704728494278ED
:108D70004A70027A0A72427A4A7202780A70C2799A
:108D8000CA7142884A8082888A80807988710020EE
:108D900088721D490120C87070471D4870471A49E4
:108DA00020B1012804D0087DC0B27047087EFBE7DF
:108DB000087CF9E710B50020FFF7F1FF00281BD071
:108DC0000120F9F7E3FB00BF00BF00BF00BF00BFF9
:108DD00000BF00BF00BF00BF00BF00BF00BF00BF9B
:108DE00000BF00BF00BF00BF00BF00BF00BF012029
:108DF000BDE81040F9F7D4BB10BD10B5FFF78BFEEE
:108E0000012010BDF9E700003C060020484C00207E
:108E1000485400202DE9F0410F460446022600F098
:108E200035F8A0B1E019401E00F030F878B1250304
:108E3000002408E02846F9F746F80646012806D13E
:108E4000641C05F58055BC42F4D3012E02D00020ED
:108E5000BDE8F0810120FBE710B5B0F5006F04D24A
:108E60000002F9F77DF8012800D0002010BD10B5F0
:108E7000094CFFF727FB012807D0206801F011FA01
:108E80000028F6D0FBF76DF8F3E710BD802801D37A
:108E90000020704701207047FC06002010B5FA4CF6
:108EA00020680068216820F0010008600020F7F7C2
:108EB00091FBF6480168496C026841F40061516415
:108EC00000BF00BF00BF0168496C026821F4006167
:108ED000516400BF00BF00BF0168D1F82C130268C5
:108EE00041F00201C2F82C1300BF00BF00BF0168AF
:108EF000D1F82C13006821F00201C0F82C1300BF38
:108F000000BF00BF0F210020FBF7ACF800280DD0F8
:108F100021685F208860216802204860F8F75DF8CA
:108F200020680068216840F00100086010BDD84A40
:108F3000D16810B141F0010001E021F00100D060E2
:108F40007047C00701D00120F1E77047D04BD968C6
:108F50000A0E120721F07F4142EA00600843D86000
:108F60007047CB48C068C0F30360704770B5C84B0A
:108F7000021E586900F1010058614FF000050CD045
:108F800000DD9D61187BC0072AD0FFF7EAFF0400CF
:108F900007D0022809D000241CE09869401C986181
:108FA000F0E7002A16DD022416E009B10A2408E0E1
:108FB0006AB9B8499A690968B1F81211914203D2A5
:108FC00000240FF0D5F907E0D969012909D05978B3
:108FD000012906D0844207D02046FFF7B7FF0120C1
:108FE00070BD0024DD61F7E7002070BD2DE9F04180
:108FF000A74D04460027A86A3E46012806D16068AE
:10900000FAF72AF9E86A032800D1AE626068A8B1CD
:1090100003F035FA002801DD01270EE02889401C05
:1090200028819C480068017FC90707D0807F298973
:10903000884203D26068FAF70FF92E813846BDE8FE
:10904000F041002192E792490120887170472DE993
:10905000F04FADF2B44D81460020CDF8B004FFF7DB
:1090600080FF4FF0FF360546CDF89064DFF820A270
:10907000D9F80400CDF8940400249AF80200274699
:109080000DF59368042803D2401C8AF802003AE1E7
:109090009AF80300012826D0092001907E484FF05D
:1090A0000009CB4605787D486A00DDF89414047801
:1090B00004A8624310F073F908200DF1100C4FF072
:1090C000000800FB04F1401C00B22CF811800928B4
:1090D000F7DD681E04FB00F7ADF8108000902CF857
:1090E000178000217AE0DDF89404D0B14FF0000B36
:1090F000CDE902B6CDF800B05B4642460DF592616F
:10910000CDF804B0DDF8940400F0A9FC074600F0A7
:10911000A0FC0446DDF89004002802DD59465046C4
:1091200003E0BAF808105046491C0181594800680C
:10913000017FC90715D0B0F81411BAF808205046BD
:10914000914202D3C16901290BD100230381CDE9EA
:10915000003402933A4631460393DDF89004FAF75F
:109160009FFEBCB1022D06D00DB1042D12D1DDF849
:10917000900401280ED1D9F80000CDE90004CDF803
:109180000C809AF801206846DDF890140FF029F958
:10919000CDF8B00442480078012874D12046ADE0F3
:1091A0000022484609E000FB04139BB23CF913304F
:1091B000934200DD1A46401C00B20828F3DD00206F
:1091C00000FB04139BB2401C3CF8136000B2B61ABB
:1091D0002CF813600828F3DD491C09B2A142DFD343
:1091E00000211EE00022019809E000FB04139BB25D
:1091F0003CF91330934200DD1A46401C00B2A842ED
:10920000F3D3092009E000FB04139BB23CF8136080
:10921000B61A401C2CF8136000B2A842F3D3491CC4
:1092200009B2A142DED3082000FB04F1401C00B2C9
:109230002CF811800928F7DD0020ADF810002CF87B
:109240001700012536E001224FF0FF39DFF854E026
:10925000A4F101082AE00023494648466F18161871
:1092600007FB0466B6B2401C3CF9166000B23344FA
:109270000128F4DD491C09B20129EEDD734513DA3A
:109280004FF0010B14E03BE014A9110010A91100EC
:1092900058060020FC060020BB050020BA0500206F
:1092A0002D06002024FAFFFF521C12B24245D2D3F1
:1092B0006D1C2DB200988542C5D3BBF1010F15D0AE
:1092C0009AF80500514628B10879401CC0B20871CF
:1092D000052806D901208AF80300DDF89404F9F77F
:1092E000BBFFFE480078012807D009E001218AF879
:1092F000051000218AF80410F3E704A8FFF78EFA9E
:10930000DDF8900498B1DAF810004FF400055446E7
:10931000A84206DB4FF07E5111F000FA2061A8420E
:1093200001DA607850B16078012809D00BE0EC498F
:10933000CAF8101000218AF8011004E001206070C2
:109340000020CDF89004DDF89004012800D0002022
:10935000DDF8B014FFF70AFE0DF2B44DBDE8F08F52
:10936000E04801680969006841F001010161DE48D7
:1093700001684969026841F4007151610168096935
:10938000026841F00401116101680969006841F057
:1093900010010161D54801680968006841F00101C8
:1093A0000160D3480078D349002208B14A81704750
:1093B0004889B0F57A7F02D94A8130BF7047401C96
:1093C000488170472DE9F04F89B0074605200025F8
:1093D0000790FAF790FDC74CDFF81CA30646C4F8C7
:1093E00010A02078012805D10F213846FAF73AFE5F
:1093F000002865D000F016FDDFF800835F21D8F863
:1094000000209160D8F8000002214160DFF8F0925E
:109410000321D9F80000C16101217F20F7F704F88A
:109420006A214FF48570F6F7FFFF21214FF4877012
:10943000F6F7FAFF207801281DD1D9F800004F4631
:10944000406CD9F8001040F400604864012002F03C
:1094500039FB3868406C396820F400604864F7F7DD
:10946000BCFDD8F800100968D8F8000041F00101EF
:1094700001600020207040F6FF7BC4F834B0C4F8CF
:1094800010A0FFF797FC9F4FDFF87CA2FFF71AF8B8
:10949000012804D0FFF765FDB04200D195B100F07E
:1094A000C1FCFAF725FD052805D0FAF721FD079044
:1094B0000520FAF72CFD0798052801D0FAF727FDBB
:1094C00009B04BE76846F7F7E7FFE0B3387848B3F1
:1094D000D9F800100320C86102217F20F6F7A4FF0D
:1094E0004FF400780C214046F6F79EFF00BF00BF06
:1094F00000BF0C214046F6F797FF00BF00BF00BF3A
:10950000002140F201284046F6F78EFF00BF00BF61
:1095100000BF00214046F6F787FF00203870012188
:109520008AF80010C4F834B0F8F70CFB6846FFF76F
:109530001CFA9AF8000018B96846FFF788FD05463E
:10954000F7F7C4FF00E002E0FAF71FFD9EE7606B4B
:10955000411E61630A2899D2FFF7A0FC96E72DE926
:10956000F04F87B000254FF0050AFAF7C4FC834698
:1095700000F058FC614852210268916000680421A3
:109580004160DFF87C914FF00308D9F80010C1F872
:109590001C8001217F20F6F747FF6C214FF4857076
:1095A000F6F742FF1F214FF48770F6F73DFF554C49
:1095B000554FFEF787FF012804D0FFF7D2FC58452E
:1095C00000D19DB100F02EFCFAF792FC052805D0E1
:1095D000FAF78EFC82460520FAF799FC5046BAF15C
:1095E000050F01D0FAF793FC07B0B7E66846F7F726
:1095F00053FF0028DDD0207840B3D9F80010C1F81F
:109600001C8002217F20F6F70FFF4FF400760C211B
:109610003046F6F709FF00BF00BF00BF0C213046FF
:10962000F6F702FF00BF00BF00BF002140F2012695
:109630003046F6F7F9FE00BF00BF00BF00213046FC
:10964000F6F7F2FE00202070012038706846FFF720
:109650008CF9387818B96846FFF7F9FC0546F7F732
:1096600035FFFAF792FCA4E770B5F7F7B9FBF9F705
:1096700065FA204C0126606A10B9F8F7D9F96662DC
:10968000224D2868B0F90E11B0F90C0100F089F9EB
:109690000EF06AFE1E4826622063002002F035FBB1
:1096A000002616E0FFF75DFC29688200D1F8F8106B
:1096B0006661D14001F00F01A66158B302282ED097
:1096C000042834D00220FFF741FCFEF7FBFE0128FE
:1096D00003D0FAF70DFC0528E4D01CE02D0600208D
:1096E0000000A0430CA91100FCA811002CA9110036
:1096F00030060020580600200000164314A911006F
:1097000010A911004107002043070020FC0600209B
:109710000000404007E0BDE870400EF027BE08465C
:10972000FFF750FED1E70846FFF719FFCDE70846DF
:1097300002F059FEC9E70000F0B5FF4FDDE906452C
:109740003F68059EBF695FEAC77C05D09C468B1BBE
:10975000A1EB0C06DBB2F6B25FEA877C05D5A44626
:10976000541BA2EB0C02E4B2D5B27A0706D5047002
:109770008A1B85704270C91AC170F0BD0370867073
:109780004470C570F0BD2DE9FF4716460D46714384
:1097900088460A4601461F46E8480FF000FEE74C9F
:1097A00002F0B0FB4FF0000A18B109F0AFF9012840
:1097B0000BD002F0A7FB18B109F0A8F908282ED0A9
:1097C000B7F5805F29D0002067E000210A46DFF866
:1097D000689320E00020D4461AE0D9F8003093F8CE
:1097E0003E81904510DC93F83F8190450CDB93F867
:1097F0003C81804508DC93F83D31834204DB6356AD
:109800007B431B13635401E004F801C0401C491C56
:10981000A842E2DB521CB242DCDBBDE8FF87AE426D
:1098200001D9701E00E0681EC2B2B54201D2681EA6
:1098300000E0701EC1B20420CDE90002002303A89D
:109840000292FFF779FF00210A46D4461DE000206E
:1098500018E09DF80D3093420EDC9DF80F309342D6
:109860000ADB9DF80C30834206DC9DF80E30834203
:1098700002DB04F801C003E063567B431B1363540F
:10988000401C491CA842E4DB521CB242DFDBC4E7A7
:109890002156794309132154401C4045F8DBBCE7AD
:1098A0002DE9F0411E4617460C460546F8F7D8FE4E
:1098B00031463846F8F7F3FE0623A04A21462846EB
:1098C000F8F7D7FFBDE8F041F8F7CBBE9C4A5060EF
:1098D000916070472DE9F00F0024DDE908959A4664
:1098E000B9F5805F01D1642D01D0002627E08842C0
:1098F00027D002FB0AF2BDE8F00F52000FF04FBD77
:109900000020A5F16407C5F1640C15E0B0FBF2F886
:1099100031F9143003FB09F31B13642D04D308FB46
:1099200007F803FB083303E008FB0CF803FB1833CC
:1099300021F81430401C641C9042E7D3761C564535
:10994000DED3BDE8F00F70472DE9FC4106467A48AA
:109950000D461F4600689046002490F84C10ADF864
:10996000001090F84D10ADF80210B0F84A10ADF8A4
:109970000410B0F84800ADF80600F8F771FE68462C
:10998000F8F73DFF39464046F8F780FE2946304655
:10999000F8F747FFF8F765FE6948C4602046BDE860
:1099A000FC816749088070472DE9F041654E8AB017
:1099B0000546A6F1480762488DE8E000B0F90000CE
:1099C0000C4603903F2801DD3F2004E001466FF084
:1099D0003F00814200DA039000200490F8F740FE37
:1099E0005948DFF86881017898F80000F8F74EFED2
:1099F0006846F8F7C5FE0890F8F733FEC4E900673B
:109A0000BDF814002081BDF816006081BDF8180073
:109A1000A081BDF81A00E081BDF81C002082BDF8CD
:109A20001E006082BDF81C10BDF81E2098F80000D2
:109A300002FB001035F910000AB0BDE8F081404883
:109A4000801C70473E4A921C032800D2107051704F
:109A500070473B48006970473948406970472DE9B5
:109A6000FF4FADF2A44D82460020DDF8E094CDF822
:109A7000A004ADF88C04CDF89004401ECDF89804F5
:109A800093464FF4906102A80FF02AFDB9F1000F40
:109A900003D099F80000CDF890042C4805782A48A6
:109AA000047825480068078E2648CDF894A48030B5
:109AB000CDF8880400F59060CDF89C04FAF718FA08
:109AC000234E02281BD1FAF716FA022817D1F9F70C
:109AD000F9FB5FEA000812D052462B464146104679
:109AE0000094F9F7D1FB3078022802D14046FEF706
:109AF00095FE3078092802D15046FEF78FFEFAF71E
:109B0000F7F9052828D0F80706D0514623462A46FB
:109B10000846FFF7C5FE0AE064214FF48050CDE906
:109B20000001514623462A460846FFF7D3FE307807
:109B3000082811D150460DE0FC06002054540020A6
:109B400090060020DC560020BB050020BA0500204E
:109B50002D060020FEF762FEB349DDF89484DDF89F
:109B600088040861F9F760FC824602462B464146AC
:109B700002A80094F9F788FB3078032802D15046F8
:109B8000FEF74CFE3078052802D102A8FEF746FE0B
:109B90003078B246062802D102A8FEF73FFE9AF8B6
:109BA000000002AE222803D100213046FEF7A2FEBB
:109BB000FAF79EF9052826D1F80724D03146234626
:109BC0002A460846FFF76CFE002003464FF00A0CB9
:109BD00010E000220BE036F9101001EBC10808EB91
:109BE000011191FBFCF126F81010401C521CAA42F6
:109BF000F1D35B1CA342ECD39AF80000082802D1F1
:109C00003046FEF70BFEFAF773F905280DD017F072
:109C1000060F02D001F0FFFF38B16A0062433146FF
:109C2000DDF888040FF0BBFB0EE023462A463146E0
:109C3000DDF88804FFF788FE9AF800000A2803D1AF
:109C4000DDF88804FEF7EAFDDDF8A804E0B1BBF119
:109C5000000F23D0DDF8A00400900DF28C433246B3
:109C6000DDF89C14DDF88804F9F72AFFCDF8980494
:109C7000FAF73EF905280AD06A0062433146DDF85A
:109C800088040FF08CFB02E0BBF1000F06D05946B0
:109C9000DDF88804FFF788FEABF814009AF800009E
:109CA000072803D1DDF88804FEF7B8FDDDF8A80425
:109CB00020B1DDF8A814DDF898040860DDF8D804B8
:109CC00010B1BDF88C140180B9F1000F03D0DDF89C
:109CD000900489F80000DDF894040DF2B44DBDE85D
:109CE000F08F524870472DE9F05F82465048904609
:109CF000894600784D4C4600F9F76FFCDFF834B127
:109D0000074600259BF80000042802D15046FEF7C4
:109D100073FD9BF80000052802D15046FEF76CFD4C
:109D20009BF80000032802D13846FEF765FD9BF83A
:109D30000000232802D15046FEF75EFD002007E018
:109D40003AF8101037F81020891A24F81010401C27
:109D5000B042F5D39BF800005F46062802D12046AA
:109D6000FEF74AFD3878222802D12046FEF744FD4E
:109D70000020721E10E004EB400134F810304988D6
:109D8000C91A09B224F81010002900DA494209B2B0
:109D9000A94200DD0D46401C9042ECD304EB460086
:109DA00020F8025C38780A2802D12046FEF724FD0C
:109DB0003878082802D12046FEF71EFD387807289B
:109DC00002D12046FEF718FD3878012802D120463E
:109DD000FEF712FD38780E2802D12046FEF70CFD62
:109DE0003878212802D12046FEF706FDB9F1000F90
:109DF00010D011494FF0FF300968B1F97220AA4222
:109E000001DA012004E0B1F97010A94200DD002060
:109E1000C9F80000B8F1000F01D0A8F80050504672
:109E2000BDE8F09F70477047900600205C600020FE
:109E3000C10500202D060020FC060020082801D2C4
:109E40008F49087070478E490020C8608D480068AF
:109E500090F88100F2E78A480078704710B500F06A
:109E6000C2F8012010BD012070478648844900686F
:109E7000B0F876004242C868824201DA401EC860EB
:109E800070472DE9F04FA1B09346894605464FF043
:109E9000000A01F0A3FF7B4F0446794E3868B0F901
:109EA0006E00A8420DDAB068401EB060401C08D1B8
:109EB0006420B060706803280AD0401C706000F015
:109EC00092F8DFF8C48198F80000072802D02BE050
:109ED0000020F3E76D4859460078820068460FF08D
:109EE0005EFAADF80050ADF80290ADF80440B089CC
:109EF000ADF80600B088ADF808003868B0F8721008
:109F0000ADF80A10B0F87410ADF80C1030F86E1FF0
:109F1000ADF80E100089ADF8100098F80000072881
:109F200002D16846FEF768FC21B05046BDE8F08FCC
:109F300053488078002800D001207047504B10B55E
:109F40009978002009B1012200E00022597801B17E
:109F500001218A4219D009B1012200E000229A7041
:109F6000484B1A68D2F8A420540708D521B1C2F38F
:109F70000310FFF763FF01E0FFF765FF0120196899
:109F800091F8A410890700D5012010BD2DE9F041FA
:109F90003C4F00263868D0F8A400C10520D5384DC4
:109FA000697809B1012400E00024C0F303310120E5
:109FB0008840F8F712FB3968B1F8A410890501D57B
:109FC00018B900E008B1002100E001218C4207D05F
:109FD00009B1012000E000206870FFF7AFFF0646DE
:109FE0003046BDE8F08170B50446F6F7F9FE284A20
:109FF00003211268D1614FF48475AE1C052C38D250
:10A00000DFE804F0030D17212B0001217F20F6F774
:10A010000BFA8C212846F6F707FA5C2126E001218D
:10A020007F20F6F701FA87212846F6F7FDF9592136
:10A030001CE001217F20F6F7F7F975212846F6F795
:10A04000F3F94D2112E001217F20F6F7EDF96721A8
:10A050002846F6F7E9F9432108E001217F20F6F7C9
:10A06000E3F958212846F6F7DFF93A213046F6F7AA
:10A07000DBF9F9F7B6F9BDE87040F6F7AEBF0000BE
:10A08000A8060020FC0600202D060020C1050020A7
:10A0900010A911006A48006800F5407070476848D0
:10A0A000006800F58070704770B5654C654A20689F
:10A0B0000168914223D14168B1F5087F1FD18568BD
:10A0C000B5F5405F1BD8604AC16891420AD00023B1
:10A0D00001461A4602E040C97340521CB2EB950F8C
:10A0E000F9D363B900F5807000F0DBF838B120686F
:10A0F00000F5407000F0E3F808B1012070BD0020C9
:10A1000070BD4F4910B54FF48E100860FFF7CCFFBB
:10A11000002800D0012010BD4FF48E10F7F771BE5B
:10A120004748484A00680168914203D14168B1F547
:10A13000087F00D0002070474148006800697047E0
:10A1400000B50146FFF7F8FF884201D8002000BDA6
:10A15000C1EBC1003A49096801EBC00000F580601D
:10A1600000BD374A126802EB80035B6A1A44344B25
:10A170001B1D53F82000FF3020F0FF0000FB0120E2
:10A180007047F0B500240D4606462746301990F971
:10A190002810002905DBE0B2FFF7E3FF45F82400B3
:10A1A00001E045F82470641C102CEFD3F0BD2DE9BC
:10A1B000F04100251746044600293FDB042C02D05D
:10A1C000052C10D014E0F9F793FE052810D1FEF706
:10A1D000C8FE022803D0FEF7C4FE10B108E0032534
:10A1E00006E0022504E0F9F783FE052800D10125E9
:10A1F0001348134E0068361D00EB840056F82410F7
:10A20000406AFF3100F5E03021F0FF01503005FBDE
:10A210000105F9F76DFE022808D101F06BFD28B9A0
:10A2200056F82400FF3020F0FF00054456F82420A3
:10A2300039462846BDE8F041F8F702B8BDE8F0819C
:10A24000B806002054465053EFBEADDE70B54FF453
:10A25000C475204CFFF755FFC0B1FFF71BFF014647
:10A26000AC221D480FF0E0F8FFF719FF01462A461F
:10A2700020680FF0D9F82068406D01F0C5FC206817
:10A28000D0F8F400BDE87040FEF75BBE29462068B8
:10A290000FF026F900210420F9F73CFEFEF7E7FD58
:10A2A000D8E750B10D4A0168914206D14068232198
:10A2B000B1EB101F01D1012070470020704730B171
:10A2C00000681221B1EB101F01D10120704700205E
:10A2D00070470000FC0600206010002041505352DF
:10A2E00005E0401E00BF00BF00BF00BF00BF002848
:10A2F000F7D170477CB5604D0024286804665F483C
:10A300000168D1F82C13006841F00801C0F82C1343
:10A31000F8F700FC28680069296840F0010008612E
:10A32000601EF8F766FB564880234FF48012002128
:10A3300052F8216040F82160491CB1EB930FF7D32C
:10A34000F8F769FBF8F7C8FDF8F7F1FD0020F8F71A
:10A35000C4FD2320F8F7B5FDF8F76AF9F8F76CFDAE
:10A36000F8F71DFCF8F77EF9F7F725FBF8F7EDFA9B
:10A37000F8F7A8FAF6F7CBFB424E009401940423B9
:10A38000002207213068F8F7E9FC3068F8F73DFD56
:10A390000420CDE900043C4C03460022072120683C
:10A3A000F8F7DCFC2068F8F730FDF7F7B1FBF7F7BA
:10A3B00074FC364800683649884201D0F7F76DFCD6
:10A3C000F8F795FEFDF7F4FEFEF7A4FB62B6FFF783
:10A3D0003DFF30480DF029FE2F4C2068B0F90C01EC
:10A3E0000DF0C0FFF8F7DAFEF9F708FF2068418AA0
:10A3F000008AFEF7A0F82068806EC0F34E0161F37A
:10A400005F0001F0C3F8FFF70EFD002211460220A5
:10A4100001F0C9F800226421072001F0C4F829687E
:10A420000120086600207CBD01F069FC0146022085
:10A43000F9F770FD0124194DF9F75AFD062818D2D5
:10A44000DFE800F0170A031114072C7002F0B9F9C5
:10A45000F2E7FFF709F9EFE7FAF7AFFA022108464A
:10A46000F9F758FDE8E701F061FAE5E7FEF7FFFCD0
:10A47000E2E7F9F791FDDFE70CA9110010A911003F
:10A48000006B002028A9110024A9110058160020F3
:10A490005446495360100020FC0600205806002056
:10A4A000FE49087070474FF42C30704710B54FF4D8
:10A4B0002C3044F264422146F7F7E3FBF84A216866
:10A4C0002046914206D14168B1F5007F02D300F0E9
:10A4D000ECFF00B10024204610BDF14940F2FF72AC
:10A4E00002C04FF40071016044F2644141600021F8
:10A4F0008160017741778177C177C0E903214161AC
:10A500008161C16400F58A6000F580404FF6FF71FB
:10A51000018041808180C180018141818181C1812F
:10A520000120704710B504460020E060204600F08E
:10A53000BCFF4042E0604FF42C3044F264422146BC
:10A54000F7F77EFE012800D0002010BD2DE9F04F66
:10A55000074691B00D460020F6F714FE0490F9F777
:10A5600001FE0C90CF48DFF8449303240678CE48D0
:10A5700000780990D9F80000C46102217F20F5F726
:10A5800053FF40F20220F5F767FFC0F30218012DD8
:10A5900066D000200090C6480190C6480790C74882
:10A5A0000390D9F80000DFF810A30025AB46C46182
:10A5B00001217F20F5F738FF4FF48770F5F74CFF46
:10A5C000C0B20E9002217F20F5F72EFF40F2072047
:10A5D000F5F742FFC4B24FF40270F5F73DFF0FF0FC
:10A5E000AFFFB7490D9051F828002031059051F880
:10A5F00028000290E00600D55546A00604D5514635
:10A6000028460FF057FE0546600604D528460399F4
:10A610000FF050FE0546E00904D0284603990FF0DC
:10A6200049FE0546E00700D0D346A00704D55146B1
:10A6300058460FF03FFE8346600704D558460399FD
:10A640000FF038FE8346200704D5584603990FF0D3
:10A6500031FE834615F1FF4F1BD385F0004019E012
:10A66000974D09980024403546430DE0B7F90000A6
:10A670000FF066FF55F828100FF07AFF0FF044FF37
:10A68000641C27F8020BA4B2A642EFD811B0BDE8B3
:10A69000F08F28468B49884200DC0D4629465846F3
:10A6A0000FF070FE06904FF0FF31019810F00BF99B
:10A6B000044607990FF05CFF8046414620460FF0A4
:10A6C000F9FD08904146204610F028F80790002038
:10A6D00017E100200EE10AFB0680099A81B272435D
:10A6E0004FF0000BB1EB520F03D2049931F9100077
:10A6F00008E00AFB06610498A1EB080100EB4100A9
:10A7000030F9020C03900C9810F8019B0C905FEA52
:10A71000096002D54FF07E500090002429FA04F021
:10A72000C00713D00120A0400FF013FB664A674B0F
:10A730000FF076FBCDE90A0158460FF08FFDDDE9F9
:10A740000A230FF0EDF90FF0B9F98346641CE4B267
:10A75000072CE3D3029905980FF0E0FF8146DDE96D
:10A7600007100FF0DBFF0A9003980FF0E9FE6FF07F
:10A770000A0110F0A8F84FF07E510FF0CFFF0B90B8
:10A78000059901980FF096FD00990FF0F1FE04462F
:10A790004FF07E5000990FF0C1FF0390DDE90101F9
:10A7A0000FF088FD03990FF0E3FE21460FF0B6FF8E
:10A7B00003900E98401E0FF0C3FE044610F1FF4FA9
:10A7C00001D384F000403F49884200DC0C464FF042
:10A7D00080410D980FF06EFD0F9021460A980FF002
:10A7E000D1FD0F990FF0C4FE0B990FF0C1FE019936
:10A7F0000FF08AFF364A04464846914501D389F056
:10A8000000403049884200DC8946954202D385F0F9
:10A81000004000E02846884200DC0D46DDE90510D6
:10A820000FF0A6FE0FF01AFDCDE90A0129465846A1
:10A830000FF0A8FD03990FF09BFE0FF00FFD83466C
:10A84000204603910FF00AFD4FF0FF3210F00DF893
:10A850005A46039B0FF064F9DDE90A230FF060F913
:10A8600004468B4649464FF07E500FF08BFD0FF0AB
:10A87000F5FC22465B460FF0D3FA0022154B0FF091
:10A8800003FC0446894628460FF0E8FC22464B4666
:10A890000FF0C6FA0FF012F90F491FE0040700206D
:10A8A00053454C46BA050020BB05002010A91100F5
:10A8B000CDCCBC40CDCC4C3FC3F5A04048E1DA4004
:10A8C00024AD11000AD7233C9A9999999999A93FE7
:10A8D000000080800000F03F00007A440FF048FE46
:10A8E000FE490FF0E7FC0FF00FFE27F8020B08F10E
:10A8F000010080B28046B042FFF4EDAE0AF10100E3
:10A9000080B2099982468842FFF4E3AEBEE670B594
:10A91000ADF5906D0C46054600264FF490616846F3
:10A920000EF0DEFDF6F72AF90020F6F71AF90020FE
:10A93000F6F70EF9F6F700F96846F8F743FEE8482F
:10A94000E8490078097869B160B12368002203F80A
:10A95000200F59709A70DA70AA0702D0224600F0D0
:10A96000B7FD0126F6F7CEFA0DF5906D304670BDB5
:10A970002DE9F74FADF5127D0D4604464FF41071E9
:10A9800068460EF0ADFDDFF8609343F254014FF0DE
:10A99000000A99F804004FF0FF3B8207949800EBFF
:10A9A000010604FB05F090903FD569463746D44632
:10A9B0002CE0002024E0621E904202D181F800A029
:10A9C0001CE037F91020002A02DC81F800B015E005
:10A9D00007EB4003B3F902309A4207DBD31A4FF07A
:10A9E000640803FB08F393FBF2F206E09A1A4FF0B7
:10A9F000640802FB08F292FBF3F20A70401C491C47
:10AA0000A042D8D307EB44070CF1010CAC45D0D3DE
:10AA1000949842F6540369461844909A0EF004FD47
:10AA20004FF4107168460EF05BFD99F80400400782
:10AA30003FD568464FF0000C31E000273A4605FB51
:10AA400004F925E0112F08D00CEB020336F913109E
:10AA5000002905DC80F800B017E080F800A014E0C1
:10AA6000234436F91330994207DBCB1A4FF06408C0
:10AA700003FB08F393FBF1F106E0591A4FF0640869
:10AA800001FB08F191FBF3F10170204422447F1C8B
:10AA90009145D7D804FB1500401C0CF1010CA445CE
:10AAA000CBD3949842F6544369461844909A0EF0DA
:10AAB000BBFC0DF5157DEAE52DE9F04105468B4817
:10AAC0000E468B490068144690F8E800088000F0B4
:10AAD00026FE00238748884A75430FE0016841F647
:10AAE000540631F8137004EB43017752166801F5F0
:10AAF000005136F81360A1F854605B1C9D42EDD8FC
:10AB000079490120C860BDE8F08130B5044691B0B4
:10AB100000250120F5F7D5FF2846FFF711FB694610
:10AB2000FFF72FFB00990798F5F76BFE734901209B
:10AB30000968C1F814032046FAF7A7F9FF20F9F7CE
:10AB4000A4FCF6F71BF80020F6F70BF80020F5F749
:10AB5000FFFFF5F7F1FF0020F8F791FC0020FAF76E
:10AB60002AFC0120F8F740FD11B030BDF0B5ADF280
:10AB7000C44D0E460446154600274FF490616846C2
:10AB80000EF0AEFC0120F5F79CFF3846FFF7D8FA2F
:10AB9000070001D1F9F7E5F90DF590613846FFF7A7
:10ABA000F0FADDF88014DDF89C04F5F72AFE53492D
:10ABB00001200968C1F81403FAF767F9F5F7DEFF19
:10ABC0000020F5F7CEFF0020F5F7C2FFF5F7B4FF40
:10ABD0002020F9F75AFC0120F8F706FD6846F8F73F
:10ABE000F1FC0020FAF7E7FB0020F6F7CBFA01466C
:10ABF000744341F25400620028440EF0D0FB0DF281
:10AC0000C44DF0BD70B5044615460E460020F5F75C
:10AC1000B6FFF8F709FC7443640021460EF03EFCD1
:10AC20000220FFF772FFFAF76FFA0320FFF76DFFBC
:10AC3000FAF777FAF8F7F8FB0146224605F65400D2
:10AC40000EF0ADFBF8F7F0FB21460EF027FCBDE857
:10AC500070400120F5F793BF2DE9F14FADF5065D8A
:10AC60000120074611904FF410610DF654100EF0BC
:10AC700037FC142013900A2014903C2000261290D8
:10AC80001090B34634460120F5F71BFF2046FFF72E
:10AC900057FA6946FFF775FA00990798F5F7B1FD7D
:10ACA000DFF858800121D8F80000C0F814134FF0E5
:10ACB000120A20254FF410740020F5F749FFF6F72B
:10ACC00005FCD8F800000321C16101217F20F5F7C0
:10ACD000ABFB11210E20F5F7A7FB11E000804144EA
:10ACE000BA050020BB05002004070020FC06002058
:10ACF0002A070020300700202C07002010A911008F
:10AD00005A210820F5F790FB36210A20F5F78CFB35
:10AD100002217620F5F788FB02217F20F5F784FBDE
:10AD20006A210220F5F780FB8E210420F5F77CFBD9
:10AD3000F1210720F5F778FB07210820F5F774FBD0
:10AD400000211620F5F770FB03217F20F5F76CFB3F
:10AD500089210520F5F768FB67210620F5F764FBDC
:10AD600045210720F5F760FB23210820F5F75CFB60
:10AD7000F1210920F5F758FB46E00120F5F7A1FE87
:10AD8000F6F7D1FA0020F9F780FBF6F726F9012053
:10AD9000F5F797FEF6F7C7FA1098F9F776FBF6F78E
:10ADA0001CF942F25C18E84429E04046F6F774FBCF
:10ADB00028B30020F5F7CCFEF6F788FB17B3761C16
:10ADC000B6B2012E4FF000000AD0F6F7DBF90146CB
:10ADD00041F65430620068440EF0E1FA002711E0B9
:10ADE000F6F7D0F9014641F2D460620068440EF0F3
:10ADF000D6FA13991098084480B2109002E0119886
:10AE00000028D2D101201190002FB6D1002633E0C6
:10AE100041F65430684415AF30F91610A0F5906033
:10AE200030F91600081A6421484300EBD070F94944
:10AE3000401047F82600096891F8EC10C9071AD0AD
:10AE4000202E08D0B6F5007F05D0E02E09D0B6F54B
:10AE5000A07F06D00FE00EF07CFF4FF06632EE4B85
:10AE600003E00EF076FFED4AED4B0EF0D9FF0EF049
:10AE700013FF47F82600761CA642C9D3002739469F
:10AE800038E0DFF890C300231E461A46384605FB1B
:10AE90000AF9DCF800E01CE09EF8ECC05FEACC7C2C
:10AEA0000AD049B9A0B1B0F5807F11D0B0F5907F3C
:10AEB0000ED0B0F5087F0BD00DF15408521C58F895
:10AEC00020C092B2664400EB590C58F82CC0634481
:10AED0002844B0EB590FDFD3B6FBF2F641F6D4703D
:10AEE000B3FBF2F2684440F82160803040F8212042
:10AEF000491C7F1CA942C4D341F6D47315AA002073
:10AF00006B4402F5005616E0B0FBF5F105FB1101AC
:10AF1000B0EB540F02D253F8211001E056F8211083
:10AF200052F82070C91B00D5494241F254276F44A2
:10AF300027F81010401CA042E6D3002739E041F268
:10AF40005420684400EB871100F6C86900264022AF
:10AF500048460EF024FA002028E0AE490022096895
:10AF600091F8EC10C90707D058B1082809D0092872
:10AF700007D0112805D0002642F2D4083146E84413
:10AF80000BE00126F8E758F820C039F81130521CC0
:10AF9000634448F8203092B2491CA942F3D358F8D0
:10AFA000201091FBF2F148F82010401C5045D4D3FA
:10AFB0007F1C5745C3D342F2D4066E440020A6F549
:10AFC00068680AE0410938F8102056F82130991ACB
:10AFD00000D5D11A28F81010401CA042F2D300204E
:10AFE0000DF6541907E059F8201038F810201144D4
:10AFF00049F82010401CA042F5D30BF1010000F0ED
:10B00000FF0B01271298CDE91007149900268B45F4
:10B01000FFF4B2AE00254FF06637DFF808A20EE06D
:10B0200059F82510B1FBFBF00EF0AAFE3A46534644
:10B030000EF0F6FE0EF060FE28F815006D1CA5421D
:10B04000EED30DF5005043F65443D0F88001620072
:10B05000414618440EF0E8F961B00DF5005DBDE819
:10B06000F08FF0B5704E00242246748006F1060C75
:10B0700035E06D4D7388103535F81350954220D169
:10B08000082B1ED200EB420341F2B355A3F85450F3
:10B09000851805F5005542F2540785F8544885F89F
:10B0A000544C03F58055A5F85448FC52A5F854407B
:10B0B000A3F8544803F54053A3F8544C73885B1C21
:10B0C0007380BCF80030934203D0BCF80230934246
:10B0D00004D1831803F5005383F8544C521C8A4260
:10B0E000C7D3F0BD2DE9F05FADF5924D44F2704449
:10B0F0006C444FF4906120460EF0F2F94A4D4FF047
:10B10000000885F8018003AEFF2244F26441304616
:10B110000EF0BCF902AFFF22042138460EF0B6F95A
:10B12000E8684FF4006B20B9FF2259463F480EF003
:10B13000ADF930460296FFF7D0F9DFF8D8904FF01E
:10B14000010AD9F8000010F8EA1FA9804078032806
:10B1500003D185F800A0FF20A8800120F5F7B1FCFD
:10B1600039462878FFF7D3FB2046F8F72BFA9DF8ED
:10B170002C409DF82D70002C7ED0002F7CD03246C4
:10B1800039462046CDF81C80FFF7F2FB28790007EE
:10B1900004D5324639462046FFF78EFC2878C00792
:10B1A0000FD02879800604D5324639462046FFF76D
:10B1B000DDFC2879400604D5324639462046FFF7A3
:10B1C00021FD2879A846000602D53046FFF744FD48
:10B1D000D9F800004D4690F8EC00C00704D004FBFD
:10B1E00007F13046FFF73DFFA9462D6895F8EB00C3
:10B1F000012836D1B8F80400C10702D05A4618A970
:10B2000006E0810716D55A4603A842F6540117E016
:10B21000074824E0FC0600206666EE3FCDCCCCCC8F
:10B22000CCCCEC3F6666E63F0407002000780020A7
:10B2300000700020410705D55A4603A842F6544144
:10B240000144E5E701077DD55A460DF5C351CC48C9
:10B250000EF0A5F842F260015A466944C9480EF062
:10B260009EF898F8000040066DD40898401C08909D
:10B270000798002868D000E013E10A98401C0A9063
:10B280007C43641E7ED4B8F80400C10713D006EBDB
:10B290004401B5F9D820B1F95410914203DBB5F956
:10B2A000DA20914207DD17990DF5804241F0010146
:10B2B0001791A2F86844810714D5311901F500519E
:10B2C000B5F9C82091F95418914203DBB5F9CA20A9
:10B2D000914207DD17990DF5804241F00201179167
:10B2E000A2F86044410714D5311901F50051B5F9B0
:10B2F000CC2091F9541C914203DBB5F9CE20914248
:10B3000007DD17990DF5804241F004011791A2F86D
:10B310006244010715D506EB440101F58051B5F9EA
:10B32000D020B1F95418914203DBB5F9D2209142F3
:10B3300007DD17990DF5804241F008011791A2F839
:10B34000644402E068E086E07EE0C10615D506EBC5
:10B35000440101F50051B5F9D420B1F954109142DE
:10B3600003DBB5F9D620914207DD17990DF5804230
:10B3700041F010011791A2F86644810617D506EB3B
:10B38000440100E044E001F58051B5F9DC20B1F959
:10B390005410914203DBB5F9DE20914207DD179985
:10B3A0000DF5804241F020011791A2F86A44410650
:10B3B00013D506EB4401B5F9E020B1F954189142D8
:10B3C00003DBB5F9E220914207DD17990DF58042C4
:10B3D00041F040011791A2F86C44010615D506EB27
:10B3E000440101F54051B5F9E420B1F9541C9142F2
:10B3F00003DBB5F9E620914207DD17990DF5804290
:10B4000041F080011791A2F86E44641E7FF53DAFB4
:10B4100095F8EB00E0B11EE043F6544103ABC206E1
:10B42000194401D55A46F3E6820604D541F2540187
:10B430005A461944ECE6420603D55A4603F654012F
:10B44000E6E60006EED40CE70998401C099017E7E1
:10B450003046FFF767F8D9F8000090F8EB000328B2
:10B4600002D14749179808801D208DF8000041201F
:10B470008DF801009DF85C008DF802009DF85D00DC
:10B480008DF803009DF85E008DF804009DF85F00C4
:10B490008DF8050006226946072000F0A8F888F814
:10B4A00001A00DF5924DBDE8F09F10B502460020B9
:10B4B000936844F264418B4200D90B46002103E0BB
:10B4C00052F82140491C2044B1EB930FF8D310BD32
:10B4D0002DE9F04115460E460446F5F77EFD0020A5
:10B4E000F8F782F80120F5F7ECFA2046F5F775FC3D
:10B4F000F9F7B3FE2D680020F5F744FE014604FB82
:10B5000006F743F254007A0028440DF048FFF8F79C
:10B5100029FE014643F654003A4628440DF03FFF09
:10B5200019480079C0070CD0F6F70CFB0020F5F79E
:10B5300026FB002105F15400FFF708F80120F5F77C
:10B540001EFB710818E001FB044C002010E001FB19
:10B55000040205EB4207ACEB000205EB4202B7F830
:10B560005430B2F852E0A7F854E0A2F85230401C30
:10B57000B0EB540FEBD3491CB142E4D3BDE8F081EA
:10B580000070002000780020040700203E49C2B26D
:10B59000C0F307200A80488070473B4841880088F4
:10B5A00061F31F2070477CB5374D012404FA00F386
:10B5B0002D882B421AD000F00F0004EB80008DF88C
:10B5C00000008DF801108DF80220100A8DF803009C
:10B5D000100C8DF80400100E8DF8050000208DF879
:10B5E00006008DF807006846FDF7EAFA7CBD1CB539
:10B5F0000123834024480088034213D0072A00D93E
:10B60000072200206B4602E00C5C1C54401C904258
:10B61000FAD30021082802D21954401CFAE7184630
:10B62000FDF7CEFA1CBD10B586B000210091019146
:10B6300016A10DF1080C1EC98CE81E0002218DF820
:10B64000001002A98DF80100095C8DF8021006288F
:10B6500003D11248807E8DF803006846FDF7B0FAEA
:10B6600006B010BD30B5084D40EA01230228AA8873
:10B67000144601D0052803D109B1022900D11A4688
:10B68000944200D0AA8030BD1C07002000030909A5
:10B690000909120C060606060F0F00003CCB00201D
:10B6A000FE4948707047FD4840787047FB49087074
:10B6B00070470EB5F94848F6B801007948430121B2
:10B6C0008DF8011000214A1E8DF807108DF800102A
:10B6D000ADF804208DF80810ADF802208DF80610A2
:10B6E0008DF80910F7F7B1FBFCF7ECFE01280DD03F
:10B6F0000120F6F74BFFF7F7C3FB0028F4D06846AC
:10B70000FDF7FFFA0020F7F7B8FBEDE7F7F7AFFB1F
:10B710000EBDE24988707047E048807870472DE997
:10B72000F04FADF6341D4FF49064214604A80DF09F
:10B73000D7FE21460DF592600DF0D2FED74F0221C3
:10B740000020B970FEF7FCFC08B9F8F70AFCF5F721
:10B7500047FBF5F713FA0020F5F703FA0020F5F799
:10B76000F7F9F5F7E9F904A8F7F72CFFF5F7D2FB9D
:10B77000F878C00601D5F5F7D0FFC9480078CDF8B4
:10B780002C09C8480578C8480478C848067815B117
:10B79000DDF82C0918B9002E70D0002CFCD0FEF773
:10B7A00041FB0020F7F76BFEF878C00604D50120B6
:10B7B000F7F71AFF012003E00020F7F715FF00203C
:10B7C000F7F712FF0120F5F7F3F8F5F706FC1E2056
:10B7D000FCF7F9FE00210846FCF796FEB860B94672
:10B7E00001210020FCF790FEF860DDF82C790020A4
:10B7F00047F6FF7A6FEA0A086F4308E0D9F8083085
:10B8000023F81080D9F80C1021F810A0401C8742B2
:10B81000F4D81E20FDF760F800210120FCF774FE2B
:10B82000834601210846FCF76FFE0021344404E002
:10B830002BF8118020F811A0491C8C42F8D8002662
:10B8400064E0FCF73FFE012865D00DF51160F5F7C7
:10B8500023FEC8B3DDF81409B8B3E078A146C006EA
:10B860000DD5DDF81449F7F7DFFD014622460095B6
:10B870001046DDF82C39F7F707FD20E050E00020F6
:10B88000002300900190029003901A461946DDF8BB
:10B890001409FEF7E4F8044699F80300800603D57E
:10B8A000FEF7D7F8044609E0F7F7BEFD0146224649
:10B8B00000951046DDF82C39F7F7E6FC2CB1002195
:10B8C0004FF4004B4B4619E01EE019E034F911002B
:10B8D000584501DB504602E0404500DA40469A6890
:10B8E00032F911C0844501DA22F81100DA6832F920
:10B8F00011C0844501DD22F81100491C8F42E5D8B2
:10B90000F5F7E4FD761C01E0F8F72BFBB9F806002B
:10B910004C46864295D30120F5F7D3F8FEF782FA1C
:10B92000F5F7F0FA0DF6341DBDE8F08F2DE9F04182
:10B930005A4D00242646AC70F6F704F905E044455C
:10B9400003D3F6F7FFF8002403E04FF47A78584F5A
:10B95000641CFCF7B7FD012803D1F8F7C9FA0328E6
:10B9600022D12878C00705D0FFF7BCFB3E702E70AF
:10B97000FCF746FC2878800707D5FFF7D0FE28782B
:10B9800020F002002870FCF73BFC2878400707D520
:10B99000FFF78FFE287820F002002870FCF730FCBB
:10B9A000F8F7A6FA0328CAD0BDE8F0814149096832
:10B9B000A1F8E80070472DE9F04FADF2A44D4FF427
:10B9C000906101A80DF08CFD354805783548CDF81B
:10B9D000A05407781E20FCF7F6FD00210846FCF76E
:10B9E00093FD2E4E0121B0600020FCF78DFDF0602C
:10B9F000DDF8A054002047F6FF786FEA080A7D437F
:10BA000006E0B26822F810A0F26822F81080401C0C
:10BA10008542F6D80024B14638E00DF28440F5F7AF
:10BA20003BFD98B30DF28440FCF79FFFDDF88804DE
:10BA300048B30646F7F7F8FC014632460097104631
:10BA4000DDF8A034F7F720FC00214FF4004B4B4603
:10BA500017E036F91100584501DB404602E0504539
:10BA600000DA50469A6832F911C0844501DA22F8AA
:10BA70001100DA6832F911C0844501DD22F81100A5
:10BA8000491C8D42E5D8F5F721FD641CB9F8060084
:10BA90008442C2D30DF2A44D46E7000024070020E3
:10BAA000BA050020BB050020BF050020C00500200E
:10BAB0003A070020FC060020014908717047000089
:10BAC00024070020002205E0002100BF491C0829AE
:10BAD000FBDB521C8242F7DB70472DE9FC5F002242
:10BAE000FF49009201920D794F8AB1F810C091F888
:10BAF0000580B7FBF5FEBCFBF8FB13461446B1F915
:10BB00000E90AA4615E000210FE001EB421530F936
:10BB100015504D4507DD03EB441630F91660B5426C
:10BB200001DD14460B46491C09B28845EDDC521C68
:10BB300012B29245E7DC53EA04004FF0010525D02C
:10BB4000E74A5B1C641C03FB0BF304FB0EF418B206
:10BB500021B2938AD48A5843614390FBFCF091FB55
:10BB6000F7F100B23A4609B2604503DBACF1010CD3
:10BB70000FFA8CF0B94201DB571E39B2D94A12686C
:10BB80009269560716D525EA020615E043208DF87E
:10BB9000000000208DF801508DF802008DF804009F
:10BBA0008DF803008DF805006846FDF709F80020C0
:10BBB000BDE8FC9F02F0010616B1611A491E09B2E8
:10BBC000940702D5181A401E00B2520701D50A4642
:10BBD00001E00246084641218DF800108DF8015021
:10BBE00011098DF8021001098DF8031002F00F0100
:10BBF00061F31F108DF804000A208DF805006846D7
:10BC0000FCF7DEFF0120D3E7B74982B26FF30F00E4
:10BC1000C1E905027047B44880787047B24A91691B
:10BC200010B141F0020001E021F002009061704784
:10BC300010B55A20F5F70BFF80220021B620F5F74A
:10BC400084FE00220121B620F5F77FFEBDE81040FA
:10BC5000A520F5F7FCBE10B55A20F5F7F8FE112225
:10BC60000021B620F5F771FE06220121B620F5F776
:10BC70006CFEBDE81040A520F5F7E9BE9B480068C2
:10BC8000C06899494207C87904D5022807D0022024
:10BC9000C871CDE7022802D10120C871DBE77047E7
:10BCA0009148007EC0F3400070478F4A00079169B9
:10BCB00021F0F00141EA10609061704700F0D2BDC0
:10BCC000894A916910B141F0010001E021F00100C1
:10BCD000906170478448007E00F001007047824BFD
:10BCE00059690A0E120721F07F4142EA00600843B9
:10BCF000586170477C484069C0F3036070477948D9
:10BD00000068406DC0F30360704770B5764C002545
:10BD10006573A573E5732070F8F7EAF8052829D153
:10BD20002078012800D160732078022822D1704940
:10BD300003200968C86102217F20F4F775FB1C21EC
:10BD40000020F4F771FB00BF00BF00BF1C210020E2
:10BD5000F4F76AFB00BF00BF00BF16210120F4F713
:10BD600063FB00BF00BF00BF16210120F4F75CFB9E
:10BD7000A573E57370BD5C48007870470121814070
:10BD80005948C9B2426942EA014141617047012103
:10BD900081405548C9B2426922EA01414161704778
:10BDA00051484069C0F30740704710B5044600F0A1
:10BDB00059FD0146FFF7F4FF022C02D0012C02D0FE
:10BDC00004E0490700E08907002905DA0121A140C4
:10BDD000014201D0012010BD002010BD4248808AE0
:10BDE000C0F30330704710B53F4B02464FF6FF7467
:10BDF000596904EA0232C1F3033021F470410A4365
:10BE00005A6110BD3848008BC0F340307047364847
:10BE1000008BC0F38020704770B5334E0446C0F3EA
:10BE20008000B569C5F30021884201D0F7F7F7FA21
:10BE3000600702D545F4807001E025F48070210789
:10BE400002D540F4007001E020F40070E10002D55A
:10BE500040F4005001E020F40050A10602D540F467
:10BE6000806001E020F48060610602D540F48050DB
:10BE700001E020F48050E10602D540F4006001E0CA
:10BE800020F40060210602D540F0800001E020F09F
:10BE90008000B061BDE87040FEF750B8124881697B
:10BEA00000204A0600D50120CA0501D540F0040053
:10BEB0008A0501D540F008008A0401D540F0805081
:10BEC0004A0501D540F02000CA0401D540F04000E9
:10BED0000A0501D540F0100009060DD50AE0000062
:10BEE00060100020FC060020340700200CA911007F
:10BEF00010A9110040F080007047F748007EC0F3A1
:10BF000040107047F448008BC0F300207047F2489F
:10BF1000008BC0F30030704700B5FFF7F8FF10B199
:10BF2000FFF7EBFF08B1002000BD012000BDEA498A
:10BF3000CA690243CA6170472DE9F041E64E021E0C
:10BF4000706A00F1010070621BD004DDB06A10B1AC
:10BF5000B06A401EB062002501B1B562307EC007F4
:10BF60005BD0FFF7C7FE0746DFF870833C4638001A
:10BF70000AD002281CD0042831D0052C2FD0002450
:10BF800045E0B06A401CE5E7002A05DD0220FFF726
:10BF90000CFF08B102243CE0D8F80000716A90F868
:10BFA0002900884233D8022401207562306330E0D2
:10BFB0000AB135632BE0D8F80000B16AB0F85C0034
:10BFC000884201D2B56204E0306B01281FD1B5620E
:10BFD00035630020FFF7E9FEC8B1002419E0002A0C
:10BFE00005DD0220FFF7E1FE08B102240FE0042F77
:10BFF00008D1FFF791FF28B10520FFF7D6FE08B161
:10C00000052406E00020FFF7D0FE0028B7D1BC428F
:10C0100005D02046FFF763FE0120BDE8F081002037
:10C02000FBE72DE9F0410F460446F4F7D9FEAC4A90
:10C0300003211068C161AB4D6A2614B1012C35D1C2
:10C0400018E001217F20F4F7EFF944210E20F4F7E6
:10C05000EBF986210820F4F7E7F96A210A20F4F7C2
:10C06000E3F9442085F8EE06862085F8E80685F891
:10C07000EA661BE001217F20F4F7D6F934210E2077
:10C08000F4F7D2F9AE210820F4F7CEF96A210A209C
:10C09000F4F7CAF9342085F8EE06AE2085F8E806F4
:10C0A0008D4885F8EA660121C1700171012F02D126
:10C0B0000020F7F799FABDE8F041F4F78EBF2DE9BB
:10C0C000F14F0024A2B0611EADF8584089462546C4
:10C0D0008DF87C402094FFF70DFE04912298059185
:10C0E000069107914768002082460A900C9022989A
:10C0F000A3468068CDF884B0089017A81D900898D2
:10C10000CDF82CB038B11EAA06A9FDF7ECFD0D90B4
:10C11000FDF7E7FD8346DFF8C081A7B108F10C0207
:10C120001FA916A8059B8DE80F0098F9013004A9F6
:10C1300038461D9AFDF793FC0C90FDF78AFC0A9097
:10C14000FDF78AFC8246FFF7ABFD0126002872D07E
:10C15000654801958068229800680F900A98CDE99B
:10C16000100A1D98CDE9125BCDE91450BDF870009E
:10C17000ADF8380000F07BFB0FB920F00100BDF8EE
:10C180005810072903D00499491C00D1012498F8BC
:10C190000A20414602B90124C97811B10421ADF841
:10C1A00058100094BDF8583001AA0EA90CF074F88C
:10C1B000099001984446806820F00801C8F82010D2
:10C1C000000798F802000CD5022804D102210122B0
:10C1D0000846FFF7E8F9A078032813D2401CA070A6
:10C1E00010E002280DD9022100220846FFF7DBF9F2
:10C1F000BDF970001E2804DD099810B94FF0FF301A
:10C200000490A5700198007AC0060DD5E07858B961
:10C2100060794FF0000178B10020FFF702FFE6706F
:10C2200001210220FDF70EFC0198007A8006607A59
:10C230000CD540B112E046E00120FFF7F2FEE670B7
:10C2400001210846EEE76672012203E0012805D1CC
:10C250006572002264210720FFF7A5F901980168A3
:10C26000002909DD6670BDF85810072924D104990A
:10C27000491C21D1049608E06570BDF858100729C3
:10C2800003D10499491C00D104950168A1B9416802
:10C2900091B9017A4A064FF0280107D4227A42B1B7
:10C2A000227A521C2272227A282A06D304952172FD
:10C2B00003E0049901290DD02572017A890700D580
:10C2C0000496D0F80090049800280FDD4046A8F8A6
:10C2D000105012E02672F0E734070020FC06002020
:10C2E00010A91100DC6000207C160020401CB8F86A
:10C2F0001010404605D0491C01820446807A10B1D6
:10C3000005E0891CF8E7A6724FF0FF300490F94869
:10C310000178012902D1891E04910570DFF8D883C4
:10C32000D8F80000017FC9072AD0407F218A8842BF
:10C3300005D3206B012802D00498401C20D125820F
:10C3400067B1DDE92003CDE90290CDE9003ADDE9EE
:10C350000401DDE90B32F7F7A3FD25720D9820B13A
:10C36000A26A01460698F7F783FDE078012807D115
:10C37000E570607948B1657102210320FDF762FB29
:10C38000DE4D2878242802D004E06671F4E70A988C
:10C39000FCF744FA2878012802D10A98FCF73EFA03
:10C3A00028780E2802D10A98FCF738FA089898B134
:10C3B000207B022810D0D8F8000090F86C00C0074D
:10C3C0000AD05A46BDF978000699FDF75AFD18B112
:10C3D000012023B0BDE8F08FDDE906230999049818
:10C3E000FFF7AAFDF5E7F0B587B00746F7F780FD40
:10C3F0000446F7F780FD0546052C09D0AFF241361B
:10C4000000F030FA0146052C04D0052D02D006E0DC
:10C41000BB4EF5E7FFF780FD08B141F00201384659
:10C42000F7F720FE002818D0F6F7DBFF07460020BC
:10C43000F4F7BEFAF4F7D1FDFCF744F8012808D070
:10C44000F7F756FDA04204D1F7F755FDA84200D1F9
:10C450002FB1F4F7C5FCF7F776FE07B0F0BD6846DC
:10C46000F5F71AF840B16846FCF77FFA6846B0471E
:10C470000746F5F72BF8DFE7F7F769FDDCE72DE96D
:10C48000F04F002685B09F49049633460D780096FC
:10C4900001960296324604A90396FDF7E0FAFDF7ED
:10C4A000D8FA0446B34600960196F7F721FD924963
:10C4B000052809680ED0888FC0F30B0A000BBAFB61
:10C4C000F0F9C88F002686463746324602FB05F350
:10C4D00000213AE0B1F80001C0F30B0A000BBAFBEF
:10C4E000F0F9B1F80201EDE734F913003DF912C09B
:10C4F000E846844505DA0DF1040C28F812002CF802
:10C50000121050451DDD584431B104EB430C3CF989
:10C5100002CC6044CC4500DD0127A5F1010C61454A
:10C5200006D204EB430CBCF902C06044CC4500DDEC
:10C530000126012F01D1012E01D0704501DB012020
:10C540000490491C4FF0000B5B1CA942CCD3521C39
:10C55000022ABBD369480078012802D12046FCF7A3
:10C560005DF9049805B035E72DE9F04387B08146C1
:10C5700000270224FDF7E4FD002866D000F072F9E0
:10C580008046F7F7B5FC0646F7F7B5FC0546414689
:10C590004846F7F767FD002857D002212020F4F71E
:10C5A000F8FD0020F4F7D4FA0120F7F71DF8564BF8
:10C5B0001868406C196840F4006048640120FFF777
:10C5C00081FA1868406C196820F400604864F5F737
:10C5D00085FAF4F702FD4D4901204863FBF772FF2D
:10C5E000012807D0F7F784FCB04203D1F7F783FCAA
:10C5F000A84204D0F5F78CFAF4F7F2FB10E0684695
:10C60000F4F74AFF50B16846FCF7AFF9684600F00E
:10C610005DF90746F4F75AFFF5F794FA002FDDD0DD
:10C62000F4F722F8F7F764FC022805D0F7F760FC6E
:10C6300004460220F7F76BFCF7F785FD022C02D0C9
:10C640002046F7F764FCF8F792FD07B0BDE8F083E9
:10C650002DE9F043ADF21C5D814600254FF0020844
:10C66000FFF748FB064600F0FDF80446022E07D10E
:10C67000FFF752FC10B144F0020401E024F0020480
:10C68000224FB879012849D021464846F7F7EAFCFD
:10C6900000286ED0F8F7E1FDF8F7AAFE0120B87186
:10C6A0001B48F4F75EFAFDF7BDFB0120FFF7B6FA71
:10C6B0000120FFF73CFC0020F4F74AFAF5F70EFAE8
:10C6C000144801688968006841F002018160F4F74C
:10C6D00084FC002078700BF091FC0F4C4FF4A069A3
:10C6E000064FFBF7EFFE012824D0F7F701FC0228E4
:10C6F00020D11AE005070020FC0600202D060020AE
:10C70000FF8F1000BA05002010A911003407002087
:10C71000E99511002CA91100EB050020F7F757FC53
:10C7200021464846F7F76FFCBAE7FFF7E3FAB04255
:10C7300000D10DB3F5F7ECF9F4F752FBFDF772FBFE
:10C74000F8F7E2FC0020F4F70CFAF6F790FBF7F7A5
:10C75000CFFB022805D0F7F7CBFB80460220F7F786
:10C76000D6FBF7F7F0FC4046B8F1020F01D0F7F71F
:10C77000CEFB0DF21C5D69E70DF5A060F4F78CFEB1
:10C780000028AED00DF5A060FCF7EFF82078012866
:10C790000DD1494668460CF0A3FE00216846FDF71E
:10C7A000D5FE38780B2802D16846FCF737F80DF52E
:10C7B000A060FFF784FC0546F4F788FEF5F7C2F9A0
:10C7C0008FE72DE9F041F6F7A5F9FDF73CFB554E53
:10C7D0003068B0F93610B0F93400FDF7E2F852498C
:10C7E00001204FF0000881F8C0065049504F81F8F1
:10C7F000C00627E0FFF77EFA04463068A100806D8E
:10C80000C7F82480C84000F00F05C7F82880C7F893
:10C810002C800020FFF779FA062C0FD2DFE804F015
:10C82000070303030B0B2846FFF712FF06E0284619
:10C83000FFF79AFE02E02846FFF7D5FDFBF742FE20
:10C84000012803D0F7F754FB0228D3D0BDE8F0410C
:10C85000FDF7F9BA70473649C8720BF07DBD344810
:10C86000C07A70473248007EC0F303107047304AE8
:10C870000021D069D161916940F400704B0603D565
:10C880004B0701D540F00100CB0501D540F0040075
:10C890008B0501D540F008004B0501D540F0200084
:10C8A0000B0501D540F01000CB0401D540F040004D
:10C8B000090601D540F08000918AC1F3033140EAB6
:10C8C0000140002901D040F4806070472DE9F0411B
:10C8D00005464FF0FF344068A046C0B1FFF7CFFDDA
:10C8E0000027134E002801DD01240FE0308A0024C8
:10C8F000401C30820B480068017FC90707D0807F49
:10C90000318A884203D26868F6F7A6FC3782FDF7C1
:10C91000ACFA41462046BDE8F04100231A46FFF735
:10C920000BBB0000FC060020DC6000204C0800204F
:10C93000340700204FF6FF7120F8A81F4180818046
:10C94000C180018141818181C18170472DE9F04120
:10C950000546FF480C460068868AC78A4FEA560893
:10C9600006F056F895F80C01022801D0032832D1C0
:10C9700095F8EB0000282ED195F8F30000282AD175
:10C9800095F8EF00002826D10BF0E9FC012812D021
:10C990000BF0E5FC28B30BF0E2FC02281BD1B5F844
:10C9A000B400A7F26917B8422CDBB5F8B610383ED0
:10C9B000B1420DDA26E0B5F8B600A6F26916B0422B
:10C9C0000BDBB5F8B400372802D9373FB84204DB97
:10C9D000A078401CA070BDE8F0812078401C207039
:10C9E000F9E7B5F8B400B0F5B47F11D8B5F8B600E2
:10C9F0003728EDD9383EB042EADA09E06078401CC9
:10CA00006070E8E7B84203DBB5F8B6003728DFD935
:10CA1000B5F8B6104145F1D2DFE72DE9F041044603
:10CA2000CB480068858A06F013F805F0F1FF0BF09B
:10CA3000AAFC07460BF0ADFC06460BF0B0FC002844
:10CA4000C9D094F80C01022801D00328C3D1B4F84E
:10CA5000B6000121B84202D9AA1B904202DB94F829
:10CA6000F10020B1002004F8EF0FA170B3E784F8C3
:10CA7000EF10B0E72DE9F04FADF51B7D05F0D3FFCA
:10CA8000939005F0C5FF909005F0D5FF044605F0A2
:10CA9000DFFF9290909804F11C0A1C30919005F0F1
:10CAA000E1FF4FF0000E0446F34670464FF6FF7C60
:10CAB00093E0C0EBC00101EB8102939901EBC2014D
:10CAC00091F85320C2EBC20202EB8203929A02EB6E
:10CAD000C30891F8F620012A7DD191F80B51022D5F
:10CAE00001D0032D77D10BF1010202F0FF0B91F879
:10CAF0005130984A02EB830636F8047C674505D02E
:10CB000036F8023C634501D03A4603E0B8F8062007
:10CB1000B8F80830032D5ED1B1F80680CDF8548204
:10CB20000A2508F10508B8FBF5F81FFA88F8CDF8D2
:10CB30006882B1F80880CDF8508208F10508B8FB8A
:10CB4000F5F81FFA88F8CDF8648202F10508B8FB01
:10CB5000F5F81FFA88F903F10508B8FBF5F81FFA94
:10CB600088F8CDF85C82DDF85482B8FBF5F8CDF892
:10CB70006082DDF85082B8FBF5F8CDF85882B2FB40
:10CB8000F5F8B3FBF5F5CDE99458DDF86882C845B2
:10CB900004D1DDF85C82999D454509D0DDF85482C9
:10CBA000989D454517D1DDF85082969D454512D197
:10CBB0000EF1010505F0FF0E664D67450BD136F805
:10CBC000027C674507D126F8042C91F8511005EB3B
:10CBD000810121F8023C401CC0B29099497D8142FC
:10CBE0003FF667AF5C49DE457ED19098807D022894
:10CBF0007AD30878401CC0B208700F2875D30F2074
:10CC000008704FF41072684691990CF0C8FB00262A
:10CC100071E0C6EBC60000EB8001939800EBC10009
:10CC200090F85310C1EBC10101EB8102929901EB25
:10CC3000C20190F8F620012A5BD190F80B21022A5C
:10CC400001D0032A55D10278437803FB0423919A3B
:10CC5000D25C02F03F0295920A7B037B9A4200D29B
:10CC600002734A7B437B9A4200D242738A7B837B66
:10CC70009A4200D98273CA7BC37B9A4200D9C2739D
:10CC800090F80C90427B94920A784978877B01FB5C
:10CC9000042290F80FB01AF80210949A01F03F0C99
:10CCA0001BE002FB04F11FFA81FE494611E00EEB86
:10CCB00001031AF8035005F03F08E04507D1DDF8FD
:10CCC000548225F03F0545EA08050DF80350491C3C
:10CCD00089B2B942EBD9521C92B25A45E1D980F8D7
:10CCE0000C909499417301E013E00EE0877380F893
:10CCF0000FB0761CF6B29098407DB04289D84FF4C0
:10CD00001072694691980CF04AFB0DF51B7DBDE849
:10CD1000F08F002008700F4901EB800221F820C03D
:10CD2000401CC0B2A2F802C00A28F5D3EDE72DE9F5
:10CD3000F05F05F078FE834605F06AFE82465024D7
:10CD400005F0E4FE012800D10824002206E00000DE
:10CD5000280800203280002074070020DFF85C9251
:10CD6000A9F10A0842E0C2EBC20000EB80010BEB24
:10CD7000C10090F80C31022B01D0032B34D190F874
:10CD80005110491EC9B2022B04D018F80130012BF2
:10CD90000AD029E030F8AC5F29F8215009EB810373
:10CDA0004088588001201DE009EB810539F8216099
:10CDB000B0F8AC306F88B0F8AEC0F31A1BB2A7EB76
:10CDC0000C073FB2002B00DA5B42A34209DC002FC4
:10CDD00000DA7F42A74204DC20F8AC6F698841800A
:10CDE00002E0002008F80100521CD2B29AF81500A7
:10CDF0009042B8D8BDE8F09F70B5044605F028FE13
:10CE0000014694F853000022C0EBC00000EB800004
:10CE100001EBC00194F80C010A25022804D0032874
:10CE20000ED084F8132170BD84F8132110E005F0B2
:10CE30001DFE6178C01E8842F5DD84F8135170BD77
:10CE400091F81301401CC0B284F813010A28F4D2EF
:10CE500060780228EBD870BD2DE9F05F8A468346E2
:10CE60004FF0000905F0DFFD064605F0F1FD8046B4
:10CE700005F0CEFD0546BAF1000F01D000206FE0AD
:10CE8000687D05F11C0700286DD0FFF7F3FD002435
:10CE900012E0C4EBC40000EB800006EBC00292F885
:10CEA000F600012806D11046FFF744FD39465846E2
:10CEB00002F0AAFB641CE4B2687DA042E9D8002716
:10CEC0003DE0C7EBC70000EB800006EBC004204646
:10CED000FFF792FF94F80C01022808D0032806D02F
:10CEE00094F80D01022823D0032821D025E0204604
:10CEF00001F08DFB94F8900001281ED194F85300A6
:10CF0000C0EBC00000EB800108EBC10191F80C01FF
:10CF1000022801D0032810D104F1A8004022A83132
:10CF20000CF082FA022084F8780084F85C9004E027
:10CF300034F8A80FA0806088E0807F1CFFB2687D75
:10CF4000B842BED80FE0C0EBC00101EB810106EB97
:10CF5000C101401C31F8A82FC0B28A824A88CA8217
:10CF6000697D8142EFD8002414E0C4EBC40000EBDB
:10CF7000800006EBC00090F8F610012908D190F867
:10CF80000B11022901D0032902D1514601F0B9FC4D
:10CF9000641CE4B2687DA042E7D8002409E0C4EB39
:10CFA000C40000EB800006EBC000FFF736FD641CF8
:10CFB000E4B2687DA042F2D81CE700000A8000209D
:10CFC000FD480078002800D001207047FB48006829
:10CFD00090F8580000F001007047F84909688A6D20
:10CFE00060F300028A65704730B5F44B1C68638AB1
:10CFF00003FB00F5608B5943B5FBF0F4B1FBF0F196
:10D000005343B3FBF0F0EE4D6443494340432C627D
:10D01000C5E9091030BD4FF6FF7202EA0023E84867
:10D0200002EA0121C38501864FF4A05141864910CF
:10D03000818670472022E24906280ED2DFE800F000
:10D040000D030D050709102005E0402003E08020B6
:10D0500001E04FF48070888570478A85704700B57D
:10D06000052210211920FFF7BFFF0A2314220321F4
:10D070000220FFF7D0FFD1480068B0F85C005DF8EF
:10D0800004EBC0F30330D5E770B516460D460446F1
:10D0900005F0BEFCECB1C94D012C35D0022C46D0B8
:10D0A000032C51D108221D211E20FFF79DFF286867
:10D0B0000A231422B0F85C00C0F303200146FFF7F6
:10D0C000AAFF2868B0F85C00C0F30330BDE87040E8
:10D0D000B0E7052210211920FFF786FFB848383045
:10D0E000284410F8010C38B9B5484230284410F8EB
:10D0F000010C08B996F80B010A231422032102201F
:10D10000FFF789FF0320E1E702220E210F20FFF73E
:10D110006BFF28680A231422B0F85C00C0F30321D7
:10D1200000F00F00491CFFF776FF0420CEE7052230
:10D1300010211920FFF758FF0A231422052102208D
:10D14000FFF769FF0520C1E770BD9C480068418A70
:10D15000408BC900B1FBF0F09749404388607EE7FF
:10D160002DE9F04FDFF85892099C0225D9F820707C
:10D170000326C8464FF0000C4FF0010A4FF0040B95
:10D1800043448F4203D8022C01D0012A06D0D9F89B
:10D190002480884513D9022C24D110E090F8E410A3
:10D1A000032902D190F8CA1021B103F801AC80F82C
:10D1B000E4B02DE003F8015C80F8E4602FE08AB170
:10D1C000884531D88F422FD9022C2FD080F8CAC081
:10D1D00013F8011C032903D103F8015C80F8E46013
:10D1E000BDE8F08F90F8E410042902D0022908D09D
:10D1F0000AE090F8CA1039B903F801AC80F8E4B03D
:10D200000DE090F8CA1031B103F8015C80F8E460D9
:10D2100080F8CAC0E4E703F8016C80F8E45010F825
:10D22000CA1F491C0170DBE7022CD9D103F8016C3D
:10D2300080F8E450D4E7624B03EB400003898B4253
:10D2400002D203EB020102E002D9A3EB0201018149
:10D2500070472DE9F041044605F0DAFB584A0546CF
:10D260001019918D138ED78D568E10F8012C5448BD
:10D27000022A00EB440008D0012A16D0032A10D15C
:10D280000289B24221D211440DE0048903EB43022A
:10D29000944202D9AC7B04B9028102899A42F2D34A
:10D2A00014D8BDE8F0810181FBE702899A4208D9D0
:10D2B000D11AA2EB6101090A4FF6FF7202EA0121BD
:10D2C000F1E7BA42DFD301D8EBE7EAD9A2EB0101DB
:10D2D000E9E72DE9FE4F99460E46044605F098FB16
:10D2E00005F0B6FB0746354894F80C2194F85150E8
:10D2F0000068314B418A408BC1EB0111890091FBE1
:10D30000F0F149432E48022A13D0A0F1500202EB5B
:10D31000C50252F808BC52F804AC328802927288F6
:10D32000019294F85020022A94F8E52014D042B3D8
:10D3300035E0002200EB050CB6F800B0B6F802A00C
:10D340000CF8012C00EB4508B0F834C0A8F808C070
:10D35000012DE2D11A70E0E70AB394F85320C2EB32
:10D36000C20202EB820207EBC20292F8E520B2B9D8
:10D3700000EB4502078EB2F808C0BC450FD91781F3
:10D380000DE089450BD394F80C21032A07D100EB5B
:10D390004507028EB7F808C0944500D93A81227932
:10D3A0004F46022A0ED0032A0CD094F8E5204AB941
:10D3B000894507D2828E06E07807002028080020E1
:10D3C000AC800020428E428694F8E520BC4642B9EB
:10D3D0008C4594F80C1102D203290BD101E00229EB
:10D3E00008D017468046806A604500D90227187821
:10D3F00010B10FE00227F5E7012D0BD1032A09D167
:10D4000001201870FE484189B8F83000814201D9E6
:10D41000FB4948812B460097494620460C9AFFF766
:10D420009FFE49462846FFF714FF08EB4500008998
:10D4300058B301464FF48073FF2801D81A4600E024
:10D440000A4600D81846EF49022F16D094F85150DA
:10D4500000236B54A2F58071029B01FB0BF101EBE1
:10D460000321B1FBF2F1A0F58072019B02FB0AF2ED
:10D4700002EB0322B2FBF0F009E094F851305D5C5E
:10D48000FA2DE7D26D1C5D54E4E700210846DC4A22
:10D4900014F8513F503A02EBC30343F8081C2378B9
:10D4A00002EBC30242F8040CB180F080BDE8FE8FAD
:10D4B0000288438862F30F01808863F31F419A4218
:10D4C00003D963F30F0162F31F410A0C824201D9B1
:10D4D00060F31F4188B20A0C904203D962F30F0136
:10D4E00060F31F41080C704770B5164615885188C7
:10D4F00090F80C21C34B90F851000B3300EB400027
:10D5000003EB8000022A1ED030F80A2C20F8082CE9
:10D5100030F80C2C20F80A2C20F80C5C30F8042C85
:10D5200020F8022C30F8062C20F8042C044620F8B1
:10D53000061C0C38FFF7BCFF0546A01FFFF7B8FF1D
:10D54000B580F08070BD20F8085C20F80A5C20F8F7
:10D550000C5D41810181C1800846F1E770B500256D
:10D5600088B02C4601EB001101EB4400641C30F83C
:10D57000100CA4B20544082CF6D3ED081D6000235E
:10D5800018466E4601EB400434F8104C641B6443AB
:10D5900046F82040401C80B223440828F2D3D80823
:10D5A00031F80A3C31F8101C591A4943116008B08F
:10D5B00070BD954A0021024402F8011C924A921E55
:10D5C000024402F8011C904A921C024402F8011C19
:10D5D0008D4A213202EB800242F8041C8A4A293229
:10D5E00002EB800242F8041C874A093202EB8002F7
:10D5F00042F8041C844A113202EB800242F8041CF7
:10D60000814A193202EB400020F8021C4180704729
:10D610002DE9F04FAFB009B2DDE938560F460124CD
:10D62000EE46E8B332F811002990701E10D4A146DE
:10D63000744604EB800844F8209032F811C0491E6B
:10D6400009B2C8F850C0002900DA691E401EF0D5A2
:10D650000021084689463946721E12D433F811C09B
:10D660005EF82240491E04FB0CF44FEAE47C14EB04
:10D67000090909B24CEB0000002900DA691E521EAC
:10D68000ECD500210C468A46711E5ED40EEB810259
:10D6900033F817C0126D7F1E02FB0CF23FB200E0A0
:10D6A0000BE04FEAE27C12EB0A0A4CEB0404002F79
:10D6B00000DA6F1E491EE9D547E033F811002990C2
:10D6C000701E10D4A146744604EB800844F82090E4
:10D6D00033F811C0491E09B2C8F850C0002900DA59
:10D6E000691E401EF0D50021084689463946731E42
:10D6F00012D432F811C05EF82340491E04FB0CF42A
:10D700004FEAE47C14EB090909B24CEB0000002954
:10D7100000DA691E5B1EECD500210C468A46711E9C
:10D7200013D40EEB810332F817C01B6D7F1E03FB71
:10D730000CF34FEAE37C13EB0A0A3FB24CEB040410
:10D74000002F00DA6F1E491EEBD5002293461146CA
:10D75000774628920BE057F82120DDF8A0C052430D
:10D76000D31712EB0C0243EB0B0B491C2892B1426E
:10D77000F1DB00229046964611460BE007EB810351
:10D7800057F821201B6D01F101015A4312EB0808E3
:10D790004EEBE27EB142F1DB00210D462A910DE015
:10D7A00007EB810257F82130126DDDF8A8C05A430B
:10D7B000D31712EB0C025D41491C2A92B142EFDBF8
:10D7C00000231A46194609E06F4607EB810701F16D
:10D7D00001013F6D7F43FB1842EBE772B142F3DB7F
:10D7E00028992E93A1FB037C0BFB03C301FB02339F
:10D7F0002B9276462A9AC646A8FB02C806E000008D
:10D80000AC800020BF8100207B07002006FB028245
:10D810000EFB0522B7EB0C0163EB02032C9198463B
:10D82000194333D02E9B2B9FA3FB092C07FB09C167
:10D8300003FB00115746AEFB073C06FB07C62B90C7
:10D84000D01A0EFB046661EB060143462C9A0BF0DE
:10D8500082FD3A9908602898A0FB07320BFB07214C
:10D8600000FB0414DDE92A20A2FB096705FB09710E
:10D8700002FB0011981B64EB0104210441EA1041F2
:10D88000000443462C9A0BF066FD02E03A99002012
:10D8900008603A9948603A982999D0E900204843AD
:10D8A00012EB204000D500202FB099E42DE9F04F75
:10D8B0008FB08A46DDE91865DDE91A8783461C4684
:10D8C0009146202103A80BF00BFE002016B1A5F114
:10D8D0000A0300E0631C052B66D94FFA84FC0CF1A7
:10D8E000010080B252464946A84200D30020E6B368
:10D8F00032F81060039631F810000490ACEB55003C
:10D9000000B2002801DA284400B23AF8102005924B
:10D9100039F810000690D8B20BA90095CDE90101A5
:10D9200021464B4652465846FFF772FE0790B8F81C
:10D9300000000D9038880E90FB480068418A428BA9
:10D94000C1EB0111B1FBF2F10891418A428BC1EBAD
:10D950000111B1FBF2F10991418A408B01EB810188
:10D960004900B1FBF0F00A9000E008E0BBF1000FC5
:10D9700003AA10D00EA90BA801F057F80FE01688E3
:10D9800003960E8820F0010004963AF800200592D4
:10D9900039F80000BEE70DA90BA801F06EF80D994B
:10D9A000A8F800100E9939800FB019E4F0B50128DD
:10D9B00008D00425032001240027DC4E002908DDBF
:10D9C000284607E04FF002054FF001004FF0000439
:10D9D000F2E708DA04EB840106EB810101EB420176
:10D9E00021F8027CF0BDD14804EB8401A0F12800AD
:10D9F00000EB410006EB810101EB4201104431F8DC
:10DA0000022C10F8010C642AECD2521C21F8022CD2
:10DA100001211970F0BDF0B50128DDE9057601D0CE
:10DA2000012000E00020C14C00EB8000283C04EB0A
:10DA300040040C4414F8014C002C28D0DFF8ECE230
:10DA40000025AEF1140E0EF13C0C944220D1B74AE1
:10DA500002EB800202EB410232F8022C9A4202D918
:10DA60000EEB400010E00EEB4002531813F8012CAF
:10DA7000642A0CD2002E0AD1521CD2B203F8012C17
:10DA80000A2A04D30CEB4000084400F8015CF0BD06
:10DA90000EEB40020A440CEB400012F8013C052B4F
:10DAA0000AD2014411F8010C642808D20A2F06DBBF
:10DAB000401C01F8010C02E0084400F8015C02F887
:10DAC000015CF0BD2DE9F04F8BB0994692468B4634
:10DAD000054604F09DFF90F85F1219B11E200290D8
:10DAE000022007E03C220292807D022801D303201D
:10DAF00000E00F200690287995F851408A4A0228C4
:10DB00000DD003280BD001290ED08948876887499A
:10DB100095F80C013239002602280ED037E0106843
:10DB20006423418A594303E01068418AC1EB011123
:10DB3000408BB1FBF0F77F43E9E7081900F8016C6F
:10DB40007A481438204400F8016C46727748283827
:10DB5000204400F8016C4672744800EB440020F841
:10DB6000026C4682714885F8E5602830204400F850
:10DB7000016C46726D483C30204400F8016C6D48E1
:10DB8000204400F8016CA5F8B8A0A5F8BA9069483F
:10DB900001EB04088C3000EB041318F8010C03EBC4
:10DBA000400121F810ACA1F8909095F80C110329D0
:10DBB00044D1C01D00F0070003EB40008DF8106059
:10DBC0008DF8146030F8101CB0F89000AAEB010337
:10DBD000A9EB00011068028B5A43038A92FBF3FC05
:10DBE000428B408A4A4392FBF0F904AB22466146DD
:10DBF0000120FFF7DBFE824605AB224649460220A4
:10DC0000FFF7D4FE03909DF810005246CDE900C006
:10DC100021460120029BFFF7FEFE9DF81410DDE96E
:10DC20000232CDE9009121460220FFF7F4FE3F4881
:10DC30002838204400F801AC0399417218F8010C0F
:10DC40004FF00109401CC0B208F8010C082807D3A6
:10DC500008F8016C9BF8E50028B98BF8E59002E024
:10DC60009BF8E50018B195F85000022802D085F81D
:10DC7000E56038E02F4909AB07AA8C312046FFF751
:10DC80006DFC2A4980460AAB08AAD2392046FFF724
:10DC900065FC0322B84501D8B8420BD9234885F862
:10DCA000E5203C30204400F8016C2248204400F874
:10DCB000019C14E01D481438204410F8011C082968
:10DCC00002D8407A082817D918481A493C3020440D
:10DCD00085F8E520214400F8016C01F8019C95F8D5
:10DCE000E500032805D011482830204400F8016CD5
:10DCF00046720BB0BDE8F08F0C483C30204410F861
:10DD0000011CC82902D2491C00F8011C0949214400
:10DD100011F8011C01290FD110F8011C069881424D
:10DD20000AD885F8E520E4E728080020B48300201D
:10DD300078070020B6810020022085F8E500D2E7B0
:10DD40002DE9F74F88B0814609980088ADF810009A
:10DD500009984088ADF8140004F05AFE99F80C01B7
:10DD600099F85140022802D12046FFF722FCFA48D8
:10DD7000F94A2044069010F8015CF748DFF8DC838C
:10DD8000801C204400F8015CF348001D00EB040AED
:10DD90000B321AF8010C02F1080EB8B1681CC0B2BF
:10DDA00014281DD304EB840108EBC10000EB4501EE
:10DDB00030F828CC31F8283CACEB030302EB840CA0
:10DDC0004CF8043C098D008D411A1BE002EB8401E4
:10DDD000002041F8040C0EEB840141F8040C15E01E
:10DDE00004EB840308EBC30101EB400030F8281C6E
:10DDF00030F82A3CC91A02EB840343F8041C018D55
:10DE0000C08C091A0EEB840040F8041C04EB840358
:10DE100008EBC30B0BEB4500BDF8101020F8281CD5
:10DE2000BDF814300385132D02D101200AF8010C2E
:10DE300099F80C0103287AD115B1681EC0B204E02C
:10DE40001AF8010C012815D028460BEB400030F8D9
:10DE5000286C008D891B181A1AF8013C00935BB1DD
:10DE6000BD4B233303EB8406002956F8047C1EDAED
:10DE70004B421DE01320E8E7B74A233202EB84024D
:10DE8000002952F8046C01DA4B4200E00B4633449F
:10DE900042F8043CB04A2B3202EB8403002853F8CA
:10DEA000046C01DA424200E00246324425E00B46AF
:10DEB00007EB030CA84B46F804CC2B3303EB84038D
:10DEC000002853F8048C01DA474200E00746474433
:10DED00002EB840243F8047C52F8042C002A00DA96
:10DEE0005242ACEB020246F8042C0EEB840252F8CC
:10DEF000042C002A00DA5242BA1A43F8042C984A39
:10DF00001268138B4B43118A93FBF1F6518B4143FB
:10DF1000508A91FBF0F7009848B98F481B3000EB0E
:10DF20004400002E30F8022C02DA714201E017E0C2
:10DF300031468A4206DA002E01DA714200E03146AB
:10DF400020F8021C4288002F01DA794200E03946AD
:10DF50008A4205DA002F01DA794200E03946418031
:10DF60007E48022114382044079000F8011C7B48A9
:10DF70000A3800EB040808F8011C99F8E5000328AA
:10DF800002D104F0DDFD58B12046FFF712FB0998DD
:10DF9000BDF8101081800998BDF81410C180A8E662
:10DFA0001AF8010C012803D0E8BB691C07293DD3EE
:10DFB000282E0CDC282F0ADC67491B3101EB4401B9
:10DFC00031F8022C282A02D84988282905D999F83D
:10DFD000040101282AD1032021E05F4900262331D2
:10DFE00001EB840151F8042C5B492B3101EB8401D6
:10DFF00051F8041C8A4200DD012605A904AA142355
:10E00000CDE90221CDE900030BF12802ABF1280193
:10E010002B463046FFF74AFC012800D00020079924
:10E0200001F8010C00E001E008F8010C06980699DF
:10E0300010F8010C401CC0B201F8010C1428A6D342
:10E040000699002001F8010CA1E72DE9F0410C46EA
:10E05000054604F0DDFC94F85110837B01220BB9D6
:10E06000837E0BB180F85F22837D0026032B05D9C8
:10E0700094F87830022B24D0032B22D090F85F3212
:10E08000012B3ED084F805616E712A71EE7090F814
:10E090007C223348022A02D094F8042182B3026819
:10E0A000926DC2F3C0422A700268926DC2F3404280
:10E0B0006A7000682246806DC0F38040A87002201C
:10E0C00036E090F85F32012B1BD094F80531012B1C
:10E0D00017D090F86532012B13D0B4F90230F02B31
:10E0E0000FDBA37B277BDB1B072B04DAE37B677B40
:10E0F000DB1B072BC8DB84F8042184F80521C3E768
:10E1000002E084F80421BFE7026892F85820C2F3C5
:10E11000C0022A70026892F85820C2F340026A7066
:10E120000068224690F85800C0F38000A8700020D4
:10E13000BDE8F041FEF7A8BF10B58A42029C02D1AB
:10E140004FF0FF3010BDE41A401A4443501A94FBBC
:10E15000F0F0184410BD000079070020F88000207E
:10E16000280800202DE9F84F93460AAA0F460646D4
:10E1700092E8030300EBD0709A4601294FEA60044D
:10E1800019D03D1B4FF0000C334652463946284605
:10E19000CDF800B0FFF7D0FF0246B11A4943781B13
:10E1A00000FB0010484532DA04EBD4704FEA6004FB
:10E1B000A5EB040530E0A6EB04054FF0000C3B4650
:10E1C0005A4631462846CDF800A0FFF7B5FF024673
:10E1D000711B4943B81A00FB0010484506DA04EBEE
:10E1E000D4704FEA6004A5EB040505E00BDD04EBF9
:10E1F000D4704FEA600425440CF1010C0CF0FF0CC4
:10E20000BCF1050FDBD3C8E90052BDE8F88F0ADD89
:10E2100004EBD470441025440CF1010C0CF0FF0CFD
:10E22000BCF1050FB0D3C8E90025EEE72DE9F04FAA
:10E2300088B00023069307930D4690F8511090F88C
:10E240000C71491ECCB2DFF814C52E886988ACF178
:10E250002802022F08D0B0F902700C23962F0BDB96
:10E260000779022F08D010E002EB840022F8246026
:10E2700041800CF8043080E01CF804700A2F03D2AF
:10E280007F1C0CF8047000E03C2303FB03F790F8BC
:10E29000C8C07F1CBCF1000F1BD1B0F8A8C032F879
:10E2A0002480ACEB080C02EB84080FFA8CF9B0F870
:10E2B000AAC0B8F80280ACEB080C0FFA8CF809FB86
:10E2C00009FC08FB08CCBC4503DD4FF0010C80F8CD
:10E2D000C8C0DFF888C4ACF1280C3CF824008246A2
:10E2E000301A02B20CEB84000590B0F8029002FBE9
:10E2F00002FCA1EB090000B200FB00CCBC453ADDFA
:10E30000BB465F42002A02DAC2F1000C00E09446EC
:10E31000002802DAC0F1000800E080460DF1180E76
:10E32000C4450ADD934201DA1A4602E0974200DD55
:10E330003A4673460127009209E0834201DA184603
:10E3400002E0874200DD3846734602270090CDF890
:10E350000CB0CDE901734B4652463046FFF702FF41
:10E36000FE490698283921F8240005990798488025
:10E37000DDE9066101E056464946AE80E98008B015
:10E38000B8E410B58A42029C02D14FF0FF30E1E6BA
:10E39000E41A401A4443501A94FBF0F01844D9E6AA
:10E3A000108051800120704710B5401AD11A029C8C
:10E3B0000A2300FB04F292FBF3F2024401FB04F097
:10E3C00090FBF3F00844524300FB0020C2E62DE925
:10E3D000F84F8B46E2498246174609680B981E465D
:10E3E0000D8A4C8A6D1E641EAAEB0701ABEB060278
:10E3F000002839DD414307EB8703C1EB43030A21C2
:10E40000424306EB860093FBF1FCC2EB400090FB1D
:10E41000F1F8BCF1000F0FDBAC4510DDA9465B46FF
:10E420003A46514648460096FFF7ABFF010006D436
:10E43000A14204DC484615E04FF00009EFE7B8F1CF
:10E44000000F02DBA04501DC10E0002453463246F9
:10E45000594620460097FFF794FF002806DBA842A4
:10E4600004DC21460A9A04E0BC4698460A9A4146D2
:10E470006046BDE8F84F93E72DE9F04F90F85170F2
:10E480008DB0064600207F1E0C901546FCB2182168
:10E4900002A80BF025F828880B904FF00008688838
:10E4A0004146CDF820800A90092F77D896F80C01C4
:10E4B000DFF8B0B202280BF5257A02D0032809D084
:10E4C0009BE0A8480BF804100A30015501210A30DE
:10E4D000015592E000910AEB8407D4467B88B6F898
:10E4E000AA203AF82410B6F8A800FFF75DFF00262E
:10E4F000E246099006F1010908A9CDE900196B88E7
:10E500002A8879883AF82400FFF761FF00200090FC
:10E51000BDF822307A88BDF820103AF82400FFF7C1
:10E5200043FF02AA42F826000FFA89F6062EE1DB25
:10E5300009984FF4C851884200DB0146052052F883
:10E5400020308B4202DA00F1010803E0401E00B2E5
:10E550000028F4DA079841F658318842814901F1E0
:10E560000A01085D0BDA0A2801D2401C0855C0B226
:10E570000A2807D11BF80400D8B1401E0BE008B1EF
:10E58000401E08550C98A0B91BF80400404506DA57
:10E5900006280ED2401C0BF804000AE034E008DD27
:10E5A000A0EB0801032902DD0BF8048001E0022939
:10E5B000E3DC6C4E1436305D0A2803D200210BF8E0
:10E5C000041004E01BF8040008B1401C00E0002027
:10E5D00008A9CDE900106B882A8879883AF82400C8
:10E5E000FFF7F5FEBDF82000A880BDF82200E88006
:10E5F000305D0A2801D2401C30550B992AF82410AE
:10E600000AEB84000A9941800DB0BDE8F08F2DE936
:10E61000F04F87B0044600F064FA804600F064FAD8
:10E6200007464FF0000904F013FA064604F0F0F92B
:10E63000059094F85150214603A8FFF706FDFEF718
:10E64000C5FC012806D034F8A80FA0806088E080BF
:10E6500007B0DAE794F85320B4F8A810ADF8041026
:10E66000B4F8AA00ADF80810ADF80600ADF80A003D
:10E67000C2EBC20000EB800006EBC00601AA3146E7
:10E680002046FEF731FF5FEA09008DF80C0007D045
:10E69000BDF80800ADF80400BDF80A00ADF80600AA
:10E6A000BDF80A30BDF8082031462046FFF70AFAC7
:10E6B00094F8500002282DD00020C4F8CC00B4F803
:10E6C000A820B6F8A810DFF89C90511AC4F8D01012
:10E6D000B4F8AA20B6F8AA10A9F1B409511A8346D1
:10E6E00009F10A0AC4F8D410022D03D89DF80F00CE
:10E6F000012821D009EB0501022001F8010C0AEBE9
:10E70000050101F8010C09EB0501002011F8011CBD
:10E7100061B341E0B4F8A820B6F8A800111A00D5FA
:10E72000811AB4F8AA30B6F8AA20981A00D5D01ADF
:10E73000494300FB0010C0E75A4601A92046FFF7F5
:10E74000FFFA94F804010028DDD10748284410F8A6
:10E75000010C012812D00028D5D108E02284002025
:10E7600028080020988100207D0700200FE0D7486E
:10E77000284410F8010C401C1428C4D9BDF8080026
:10E78000ADF80400BDF80A00ADF80600BBE70AEBDF
:10E79000050111F8011C01B10120009005985B46AC
:10E7A00001A9827D2046FEF794FD9DF80D00012809
:10E7B0005ED0BDF80400A4F8AC00BDF80600A4F8D3
:10E7C000AE00314601AA2046FFF756FE94F85100EC
:10E7D000BF4ABDF8081002EBC00040F8081C94F8CE
:10E7E0005130BDF80A0002EBC30242F8040CADF848
:10E7F0000410ADF8060001A92046FFF717FDBDF88B
:10E800000800ADF80400BDF80A10ADF80610A4F831
:10E81000AC00BDF80A10A4F8AE10BDF806104246D0
:10E82000404500DA1046B94200DA3946A94A136871
:10E83000B3F91050A5EB0802551E854200DA501EB0
:10E84000B3F91220D21B531E8B4200DA511E82B242
:10E8500024F8AC2F88B2608036F8AC1F511A2163BF
:10E860007288801A4943606300FB0010E062EFE6A3
:10E87000BDF80800ADF80400BDF80A10ADF80610A8
:10E88000A4F8AC00BDF80A0099E770B5914A156884
:10E8900095F85420530702D50126964301E002F073
:10E8A0000106B0F90040B1F900301EB1EE8AF31A4A
:10E8B0005B1E1BB2960703D5AD8A2C1B641E24B2C7
:10E8C000520702D503800C8070BD04800B8070BDA0
:10E8D00070B5804A1268B2F8983013F0FF024FEA20
:10E8E000132300D1642203B96423058864265543A9
:10E8F000B5FBF6F20C8802805C43B4FBF6F00880AE
:10E9000070BD2DE9FC47044672480068B0F818A0B5
:10E91000B0F81A90868AC58AB0F81080478A00201D
:10E92000ADF80000ADF8040004F072F8B4F8AC00E3
:10E93000B4F8AE1000FB0AF393FBF8F2A4F8B02091
:10E9400001FB09F292FBF7F2704390FBF8F0A4F898
:10E95000B220ADF80000694391FBF7F0ADF8040078
:10E9600001A96846FFF791FFBDF80000BDF804104B
:10E97000401C491C00B209B2A5F10109ADF8000024
:10E98000ADF80410484500DB681E00B2A6F1010C8A
:10E99000ADF80000614500DB711E09B2ADF804104E
:10E9A000002800DC0020ADF80000002900DC002178
:10E9B000A4F8B400A4F8B610B4F8BC00B4F8BE10C3
:10E9C000704390FBF8F0ADF80000694391FBF7F05D
:10E9D000ADF8040001A96846FFF757FFBDF8000035
:10E9E000BDF80410401C491C00B209B2ADF800008B
:10E9F000ADF80410484500DB681E00B2ADF8000019
:10EA0000614500DB711E09B2ADF80410002800DC7E
:10EA10000020ADF80000002900DC0021ADF8041052
:10EA200024F8BC0F6180BDE8FC87F0B5034615688B
:10EA30005C681F68654356680020D2F814C007EB75
:10EA400025439D1B00D5F51A654515D29368D568F9
:10EA50005C4307EB244396695C1B00D5EC1AB44277
:10EA60000AD2D5690C681269A31A00D5131BAB42F0
:10EA700002D290B208600120F0BDF0B5034655689F
:10EA80005C681F68654316680020D2F814C007EB65
:10EA900025439D1B00D5F51A654515D2D3689568A9
:10EAA0005C4307EB244396695C1B00D5EC1AB44227
:10EAB0000AD2D5690C681269A31A00D5131BAB42A0
:10EAC00002D290B208600120F0BD00007B07002058
:10EAD0005C80002028080020FE487047FD489030E8
:10EAE0007047FD4800787047FB4840787047034600
:10EAF00010B50020024603E053F82240521C204487
:10EB00008A42F9DB10BD2DE9F05F0D46064603F0A1
:10EB1000ADFF044603F0A6FF290291FBF0F5310298
:10EB200091FBF4F3DFF8B0E3DFF8A8836F125E1215
:10EB300008F19008BEF804A0BEF806B0002108F560
:10EB4000907909E001FB03F206EB222248F821202C
:10EB500049F82120491C09B2A142F3DBDD4E002116
:10EB600006F5907C09E001FB05F207EB222246F84E
:10EB700021204CF82120491C09B28142F3DB03FB20
:10EB80000BF3D8F800705A13BF1AC8F8007008EBDE
:10EB9000840705FB0AF557F8048C6913904447F87D
:10EBA000048C37686D135B137F1A376006EB8006A1
:10EBB00056F8047D0F4437609EF80260BEB1D9F864
:10EBC000005009EB8403AD1AC9F8005053F8044D06
:10EBD0000CEB800022441A60DCF80020521ACCF8BA
:10EBE000002050F8042D11440160BDE8F09FD9F8D1
:10EBF00000700CEB8000BA1AC9F8002009EB8402FF
:10EC000052F8044D23441360DCF80020511ACCF86C
:10EC1000001050F8041D2944E6E70346AF4830B41D
:10EC20000168AD4A0224488A098A0C259480D5805F
:10EC300030BC68E7A8488078012800D000207047E1
:10EC400030B40400A548A44B0268508A118A0ED043
:10EC500092F85440528BE4084443B4FBF2F21A7029
:10EC60005A7002229A800C22DA8030BC4BE70022D4
:10EC7000F5E79A48026892F85430508A118ADB0806
:10EC8000528B4343B3FBF2F3934A13705370022346
:10EC900093800C23D3800023937034E72DE9F04F49
:10ECA000B3B00D460446CC228D4968460AF0BCFB41
:10ECB0008A480168487991F804B0B1F812900F8A37
:10ECC000697801FB00F216B2B5F90220012A00DCD6
:10ECD00001222B78EE4683B1A0F1010C1E4463455E
:10ECE00004EB460612D136F9026C012E00DC012637
:10ECF000F602764296FBF2F63BE004EB4606B6F9E6
:10ED00000260012E00DC0126F602F3E736F902CCA0
:10ED1000BCF1010F01DC4FF0010CB6F90260012ECD
:10ED200000DC01264FF064080CFB08FC0CEB620CC5
:10ED30009CFBF2FC3EF91CA0C44606FB0CF606EB5D
:10ED4000620696FBF2F63EF91660B24513D0DFF884
:10ED500094810AEB060CC44505DBBCF5004F03DBD0
:10ED600047F6FF7C00E0C446AAEB0606F60296FBD7
:10ED7000FCF636B200E00026A1B1ABF1010C614512
:10ED8000A1F1010C0CFB00FC0FFA8CFC9C4412D18D
:10ED900034F91C40012C00DC0124E402644294FBA1
:10EDA000F2F243E003EB000C34F91C40012C00DCD0
:10EDB0000124E402F3E734F91CC0BCF1010F01DCCB
:10EDC0004FF0010C01F1010808FB00F80FFA88F878
:10EDD000984434F91880B8F1010F01DC4FF00108B4
:10EDE00064240CFB04FC0CEB620494FBF2FC3EF983
:10EDF0001C404FF0640C08FB0CF808EB620C9CFB09
:10EE0000F2FC3EF91C20944212D0DFF8D88004EBCB
:10EE1000020CC44505DBBCF5004F03DB47F6FF7C65
:10EE200000E0C446A21AD20292FBFCF212B200E049
:10EE3000002209041B0403EB061301EB021103F586
:10EE4000004301F5004193FBF0F091FBFBF17843A7
:10EE500001FB09F100144FEA214101D5002200E035
:10EE60000246BA4201DD384602E0002800DA0020FE
:10EE7000002901DA002200E00A464B464A4501DD3E
:10EE8000194602E0002900DA002125F8A80F698060
:10EE900033B0BDE8F08F70B5A4B00C4605461646F9
:10EEA000902168460AF01CFB00206A4607E054F8EF
:10EEB000201056F82030594342F82010401CA84238
:10EEC000F5DB29461046FFF712FE06462946204686
:10EED0000AE0000054840020AC070020280800202D
:10EEE00084AD11000080FFFFFFF701FE96FBF0F0FC
:10EEF00024B070BD2DE9F04F8946ADF5117D03EBCF
:10EF00008906934605461C46DDF868A256F8048C2F
:10EF1000CC22FE4934A81F680AF086FAFB49D022A9
:10EF2000CC3168460AF080FAA422F94967A80AF0B1
:10EF30007BFABAF1000F0ED066688F982246301A1D
:10EF4000606059464846FFF7A6FF054666602846BA
:10EF50000DF5117D9DE7B5F5D57F1ADADD2D01DCC4
:10EF6000332007E0A5F2A9104042C11700EB9170D1
:10EF700080100ED45DF820002246391A216056F820
:10EF8000041C084446F8040C59464846FFF783FF22
:10EF9000054642F6346085421DDB42F698608542A4
:10EFA00001DB322006E0A5F53850343800EBD07094
:10EFB000401010D434A9226851F82000111A2160A1
:10EFC00056F8041C2246084446F8040C59464846A4
:10EFD000FFF761FF0546276046F8048CB7E72DE987
:10EFE000FF4FD1B00F461446902101A80AF078FADD
:10EFF000902125A80AF074FA03F00AFD03F01BFD26
:10F0000003F038FD00200646009003F02BFD054676
:10F0100003F02CFDDFF8FCB24990BF4ADBF800009A
:10F02000418A4A91008A4B90607821784C92903ABC
:10F030004D9200FB05120129BA5C02F03F0A01D093
:10F0400039B10EE008280CD309280AD80120009015
:10F0500007E00A2802D0072802D002E0012600E0DB
:10F060000226207B4F90627B94F80E90E07B4E90BE
:10F070002DE002FB05F01FFA80F80DF1040E4F9908
:10F0800020E0519808EB010CB4F93E3030F91C0037
:10F09000322B04DAC01A00B2002800DA012017F877
:10F0A0000C3003F03F0CD4450AD15EF82130034404
:10F0B0004EF8213025AB53F822C0604443F82200BB
:10F0C000491C89B24945DCD9521C4E9892B2824201
:10F0D000CFD9294601A8FFF70AFD00287EDD25A823
:10F0E0004999FFF704FD002878DD01A928464D9ACB
:10F0F000FFF7D1FE894F0446B87830B901AA2946F6
:10F1000020464D9BFFF7F6FE0446387838B1B4F53B
:10F11000FA7F13DCDBF80000018A890007E042F681
:10F120003460844208DBDBF80000018A4900008B70
:10F13000B1FBF0F0044409E0C82C07DCDBF8000068
:10F14000018A008B4900B1FBF0F0241A25A94C9AE2
:10F150004998FFF7A0FEB97829B9009625AA4C9BDB
:10F16000499900F052FADBF800104A8A498B920064
:10F17000B2FBF1F1401AB4F57A7F23DC04EB840191
:10F1800049004FF4C87291FBF2F1C1F119010A294B
:10F1900000DD0A210A23B0F5616F04DB890191FBD0
:10F1A000F3F108440EE040F6944290420ADB8201FB
:10F1B0004FF4BE7592FBF5F2A2F21E224A4392FB77
:10F1C000F3F10844002C00DA0024002800DA0020C3
:10F1D0004B99491E8C4203DD4B9C00E007E0641E06
:10F1E0004A99491E884204DD4A98401E01E00024E5
:10F1F000204654990C805E99088055B049E630B598
:10F2000093B004462422464968460AF00DF9444961
:10F210002422243109A80AF007F92579B4F8A810A6
:10F2200060786A4609AB012D05D0B4F93A50B5F5BE
:10F23000E17F0FDC04E0B4F93850B5F52F7F09DC2D
:10F240002578142D06D933F810000844A4F8A80036
:10F2500013B030BD32F81000F7E72DE9F74F2D4815
:10F260008B4684B00168144691F8560091F8551009
:10F2700000F07F0901F07F0A4FEAD018CF0903F0B0
:10F28000C7FB03F0D8FB03F0E3FB94F85310C1EB8A
:10F29000C10101EB810100EBC10503F0E7FB06466C
:10F2A00094F80B0102210122022802D0032803D086
:10F2B0001AE084F80D210AE084F80D2195F80D017B
:10F2C000012804D002280AD0032808D00CE094F8C2
:10F2D000E80048B984F80D1184F80C1104E003200B
:10F2E00084F80D0184F80C0102A8009001AB2246BD
:10F2F00059460498FFF773FE09EB89000AEB8A016F
:10F30000C0B2C9B2B8F1000F0ED00BE050AE110080
:10F31000ECAF11002808002004860020AC07002074
:10F3200094B211004042C0B20FB14942C9B2BDF817
:10F3300004201044A4F8A800BDF808000844A4F86C
:10F34000AA0095F8E80001280AD1287840B9687821
:10F3500030B1761EB04203DA94F8E900012807D0F4
:10F3600095F80701012809D1E088E988884205D38A
:10F3700035F8A80F24F8A80F6888608007B088E5E2
:10F380002DE9F84F044603F043FB03F061FB01460F
:10F3900094F8530094F85120C0EBC000521E00EBCB
:10F3A0008000D5B201EBC00BC02603F05BFB0090E0
:10F3B00003F05CFB0123074684F80C3194F80D013F
:10F3C000DFF814C3022802D003280AD032E0B4F8D0
:10F3D000A8002CF825000CEB8501B4F8AA004880A1
:10F3E00028E03CF82520B4F8A800111A00D5811AAD
:10F3F0000CEB8509E246B9F80280B4F8AAC08AB2DB
:10F40000B8EB0C0101D5ACEB080189B2AA2A01D8EE
:10F41000AA2901D984F8C8304FF4C87C624501D8C4
:10F42000614501D984F8C9302AF82500B4F8AA103A
:10F43000A9F80210B4F8A800A4F8BC00B4F8AA1007
:10F44000DFF894E2A4F8BE1094F80D21AEF1840E1A
:10F45000AEF128084FF0020A4FF0000C08F17809CD
:10F46000022A04D0032A2CD0012A7DD09FE02078E4
:10F47000032811D90099091F88420DDA6078032802
:10F480000AD93F1FB84207DAB4F90200962803DD13
:10F4900084F802C184F80CA109F80530B4F8A8106A
:10F4A00028F8251008EB8500B4F8AA104180B4F8BC
:10F4B000A8104EF835100EEBC500B4F8AA10416044
:10F4C00075E09BF80C21022A1DD0032A1BD038F8C6
:10F4D0002520C346131A00D5831AB34209DC0BEB6F
:10F4E00085077B88B3EB010801D5A1EB0308B04584
:10F4F0000DDD09F805C00BEB8500A4F8A8204088B5
:10F50000A4F8AA0044E0032084F80C014FE05EF860
:10F51000351001444EF835100EEBC5008846B4F89E
:10F52000AA6041680E44466019F80500401CC0B24C
:10F53000B8FBF0F109F805000090B6FBF0F0664E5C
:10F5400089B2283E80B256F8256006EB460808EBE3
:10F55000C608B4F9386006EB8606B8EB460F04DA45
:10F560002BF82510788022E015E0561A00D58E1A67
:10F57000042EF5DC1A1A00D5C21A042AF0DC009A0F
:10F58000042AEDD3A4F8A810A4F8AA0009F805C02D
:10F5900084F80CA10BE0504809F805C0283840F861
:10F5A00025C008EB850028F825C0A0F802C04A4A0B
:10F5B000B4F93800283A494642F8250019F8050000
:10F5C0000A2814D95EF83560B6FBF0F024F8A80FCD
:10F5D0000EEBC5004B5D4068B0FBF3F0608009F8AE
:10F5E00005C042F825C084F864A0BDE8F88F94F8FF
:10F5F0000C010328F9D194F8ED000128F5D184F825
:10F600000CA184F8EDC0F0E727E62DE9F04F8A461B
:10F61000ADF5017D03EB8A05934606461C468A9F9D
:10F6200055F8049CF4222D4931A8D3F8008009F044
:10F63000FBFE2A49C422F431684609F0F5FE4C224B
:10F6400027496EA809F0F0FE27B1012F28D0022F1C
:10F6500032D03CE041F2B15086421CDB41F21160F5
:10F66000864201DB302106E0A6F5A850B13800EB58
:10F67000D07041100FD45DF821002246A8EB0001A4
:10F68000216055F8041C084445F8040C59465046BE
:10F69000FFF701FC0646C4F8008045F8049C16E01C
:10F6A000256B59982246281A206359465046FFF781
:10F6B000F2FB064625630AE065695998224628440C
:10F6C000606159465046FFF7E6FB064665610DF559
:10F6D000017D3046BDE8F08F4087002090B01100DA
:10F6E00048B211002DE9F04114460E46054603F0DC
:10F6F000B9F90746D6E90902F16A58B102EB82026C
:10F700009200400001EB81018900B2FBF0F3B1FBF4
:10F71000F0F101E0002319460A20B3FBF0F2B1FB3F
:10F72000F0F000FB07202380618035F81000A080F6
:10F73000BDE8F0812DE9F0410DF11808044698E884
:10F74000C1000D4620B1002081F841000020EFE704
:10F7500055F8020B20606888A0806868E060A8689F
:10F7600020611068C4F80600908860812C22194638
:10F7700004F1240009F058FEE86860612869A0617E
:10F780006869E061A8692062D5F82200A062E88B70
:10F79000A08495F8300084F84800D5F83200E06481
:10F7A00095F83C0084F84900288CE08795F84100E2
:10F7B00084F8510095F83E0084F8F70095F8400071
:10F7C00084F8F80095F8450084F80E01012084F8CB
:10F7D000F60095F8430084F8150184F8F97095F85F
:10F7E000460084F814013078401CC0B230700A28FA
:10F7F000ACD301209CE710B5002801DC002010BD2F
:10F8000004024FF4807100200B1294FBF3F30A46BC
:10F81000991801EBD1714910531A00D58B1A802B1E
:10F8200002DB401C6428EFD3081210BD2DE9FF4F06
:10F8300087B00024C4201D4617460E460090FE489F
:10F84000019003F00FF98346B7F900000290B7F971
:10F8500002E0B0790590307A0490F279707A002352
:10F860001E461F46039027E0059820E002FB0B0C84
:10F87000079931F91C103C2917DDDDF808C000EBB1
:10F880008008CCEB480A012102EB8208CEEB480845
:10F8900008FB08FC0AFB0AF908FB0AF809FB01331C
:10F8A0000CFB016608FB1177641C401C00B2049934
:10F8B0008842DBDD521C12B203988242D4DD642000
:10F8C00093FBF0F196FBF0F297FBF0F0002801DAE1
:10F8D000434200E003460A2B08DC881800EBD07096
:10F8E0004110881800EBD070421000204CB1090282
:10F8F0001202000291FBF4F192FBF4F290FBF4F09F
:10F9000002E000210A46084601FB02F300FB10302A
:10F910008C1807126642B90006FB06F0C1EB2020E6
:10F92000FFF769FF000101193044C0F1000001EB4D
:10F93000D17100EBD0704C104FEA600601D56142E6
:10F9400000E02146002E01DA704200E0304681429C
:10F9500005DD002C01DA604206E0204604E0002EBE
:10F9600001DA704200E03046002C01DA614200E02A
:10F970002146002E01DA724200E03246914205DD56
:10F98000002E01DA714206E0314604E0002C01DA73
:10F99000614200E021468846FFF72DFF4FEA001C38
:10F9A0004046FFF728FF01010CEBCC0001EBC10141
:10F9B000C0F3D610C1F3D6132F61002C00DA6442D5
:10F9C000AC60002E00DA764204EB44018900192273
:10F9D00091FBF2F10C22091D02EB4102EE60FF2ABD
:10F9E00000DDFF22DDE90041103104FB001004FBC3
:10F9F000031100124FEA212100D50020002900DA6E
:10FA00000021FF2800DDFF20FF2900DDFF21052860
:10FA100000D2401C00B109B90120014602B90122FF
:10FA200085F8222005F8200F69700BB0BDE8F08F33
:10FA30002DE9FF4F81480E468DB0D0E904121A9C83
:10FA4000CDE90012D0E90612CDE90212D0E9081280
:10FA5000CDE90412D0E90A10CDE9061002F0D8FF72
:10FA60001C30089002F0FEFF054602F0FFFF0990EF
:10FA70000021B6F902E030780B9070788A460F4684
:10FA80008B460B46F1460A460A90002024F81100E6
:10FA90003DF812600B98304402AE00B236F812C046
:10FAA0000A9E66440FFA86FC0CFB050636B2BCF1D2
:10FAB000000F2FDBDDF82480A8F10108C44529DC04
:10FAC000002827DBA5F1010C604523DC0D9830F9F7
:10FAD000160024F81100002802DC012024F811008F
:10FAE00034F911000A2806DD4FEA0E2CBCFBF0FCAD
:10FAF0007F1CE244FFB2584500DD8346DDF820C09C
:10FB00001CF806C0BCF1000F01D05B1CDBB24844FE
:10FB10000FFA80F9491C521CD2B2C9B2042AB4D3DC
:10FB20000020002224F8112004AA32F810600B9A59
:10FB3000324406AE12B236F810C00A9E664436B29F
:10FB400006FB052C0FFA8CFC002E1ADBDDF8248056
:10FB5000A8F10108464514DC002A12DB6E1EB242F1
:10FB60000FDC0D9A32F91C2024F81120002A02DC47
:10FB7000012224F81120089A12F80C200AB15B1C0B
:10FB8000DBB2491C401CC0B2C9B20428C9D31098CA
:10FB900003700EEB0B0001B217B1BAFBF7F000E0F7
:10FBA00000200F9AC009D1820F99C8610F99A1F85E
:10FBB000149011B03AE700B587B001AB009305ABE4
:10FBC000FFF736FF07B000BD2DE9F0411E4617468E
:10FBD0000C46069D02F01CFF1949096891F858105F
:10FBE00009064ED5817C69BB218C3288914215D99A
:10FBF00097F82020B1888A4210D9618E7388994283
:10FC00000CD91144502909D9B4F90210B0F90220D5
:10FC1000B1EB620F02DD2978491C2970218C46293D
:10FC20001BD997F820101E2917D9628E142A14D9CF
:10FC30001144462911D906E0ECFCFFFFDCB21100AB
:10FC4000280800201DE0B4F90210B0F90220B1EB41
:10FC5000620F02DD6978491C6970218C282910D94E
:10FC600097F820101E290CD9618E0F2909D9B4F9F3
:10FC70000210B0F90200B1EB600F02DDA878401C61
:10FC8000A870002054E52DE9F0410D46044602F02D
:10FC9000EDFE064602F0E6FE002285F847206B786E
:10FCA000014613B1761EB34239D12E7803FB016EA3
:10FCB0001FFA8EF023B1431A1FFA83FC01230BE0D5
:10FCC0004318F9E7C718BFB234F91770232F06DDC0
:10FCD000521C5B1CD2B2DBB2F7188F42F2D3012167
:10FCE00009E0431A9BB234F91330232B05DD521C73
:10FCF000491CD2B2C9B2731AF3D5032A0FD934F909
:10FD00001000C8280BDA1FFA8EF034F91C1034F9F1
:10FD10001000B1EB600F02DA012085F8470007E51B
:10FD20002DE9F04F0446A5488A4689B0D0E9001273
:10FD3000CDE90012D0E90210CDE904100020ADF8A1
:10FD40000A00ADF80800ADF80E00ADF81E00ADF8E1
:10FD50001A000646ADF80C00ADF81C00ADF818000E
:10FD6000374602F07FFE054602F080FE9AF801B0A9
:10FD70000021A0F101090DF1100E3DF91120002024
:10FD80000BEB02034B4561DC002B5FDB9AF800C0F4
:10FD90003EF910206244A5F1010C624556DC002AB0
:10FDA00054DB03FB052292B2022909D0022806D0B7
:10FDB000BDF808C034F81280C444ADF808C049B199
:10FDC00030B1BDF80AC034F81280C444ADF80AC09E
:10FDD000022908D030B1BDF80CC034F81280C444F8
:10FDE000ADF80CC041B1022808D0BDF80EC034F8FF
:10FDF0001280C444ADF80EC0012801D0012911D1F0
:10FE000034F912C001290DD1022806DABDF8188094
:10FE10000028E044ADF8188018DDBDF81A80C4440D
:10FE2000ADF81AC0012811D1022908DABDF81CC0AA
:10FE300034F812800029C444ADF81CC006DDBDF8BA
:10FE40001EC034F812206244ADF81E20401C00B2DF
:10FE5000032897DB491C09B203298EDB002002AA84
:10FE600006AB32F91010B94200DD0F4633F910101D
:10FE7000B14200DD0E46401C00B20428F1DB09B09F
:10FE8000D4E52DE9F74F002096B083460446149040
:10FE90000746129010908146119002F0C4FD159013
:10FEA00002F0B6FD804602F0C6FD82463720ADF86E
:10FEB00040002D208DF84C40ADF842001E20189CCB
:10FEC0000026ADF84400641E4BE004EB440000EB58
:10FED0000411179800EB810595F8410001283ED1E7
:10FEE0002C2103A809F0FCFA00200E907F1C0F9033
:10FEF000FFB203AA2946189B1698FFF75CFE03ABD6
:10FF00000EAA29461698FFF7EDFB03AB0EAA294669
:10FF10001698FFF78BFC12A8009010AB03AA294695
:10FF20001698FFF751FE149913AA8DE806089DF85C
:10FF30004C0003ABC0EBC00000EB800115980EAA8B
:10FF400000EBC1002946FFF7F5FB01280BD0288CF8
:10FF5000B04200D90646686A484500DD8146641E05
:10FF600024B2002CB1DA9DF8480070B99DF8490020
:10FF700001280AD818B19DF84A10012905D8072F81
:10FF80000ED99DF84A10C8420AD001208DF82F00E2
:10FF900088F81B0098F81A1051B988F81A0007E081
:10FFA000BAF90200642803DA9AF87B020028F4D038
:10FFB000A8F804609DF84C0019B037E5DCB21100D8
:10FFC0002DE9F04F87B00F46804602F04FFD064600
:10FFD00002F048FD00250446039502F015FD01904E
:10FFE00002F016FD824602F01EFD029002F023FD93
:10FFF000059002F02DFD024698F80000A8B10521F9
:020000021000EC
:10000000284661F3070098F8011081B1B11F61F330
:100010000F20052161F3174098F8031049B1A11F83
:1000200061F31F60814600208FE00221E8E7F11EA6
:10003000EDE7211FF4E7CBEBCB0000EB8003029848
:1000400000EBC30090F8F61001297BD1B0F9021043
:1000500001EB41014FEAE17C01EB9C7189100FFA41
:1000600081FE029911F83330A4F1090106918B4207
:1000700001DD052101E009F0FF0190F80DC05FEA04
:100080000C0826D190F801C0CDF810C08C4520D2C4
:1000900000210091BCF1010F11D9414609E001FB9B
:1000A000043C1FFA8CFC37F91C80F04511DB491C1D
:1000B000C9B2DDF810C08C45F1D8009949B9019951
:1000C000C95CC90705D0012180F80F1161F307054C
:1000D000039106998B4202DDB11FC9B201E0C9F359
:1000E000072190F80FC0A6F10108CDF818C0C4454B
:1000F00028D190F801C0CDF810C08C4522D900213C
:1001000000916146A6F1020C614511DA069909E0F9
:1001100001FB043C1FFA8CFC37F91C80F04511DB15
:10012000491EC9B2DDF810C08C45F1D3009949B918
:100130000199C95C890705D5012180F80F1161F388
:100140000F2503910BF10100C0B29AF815108346F8
:1001500059453FF670AF002071E0CBEBCB0000EBD0
:10016000800302EBC30090F8F610012964D1B0F9C6
:10017000021001EB41014FEAE17C01EB9C71891017
:100180000FFA81FE417B5FEA010825D1417809F031
:10019000FF0C049161451FD20021009104990129AF
:1001A00013D941460BE012F833C001FB04CC1FFA0F
:1001B0008CFC37F91C80F0453EDB491CC9B2DDF8E8
:1001C00010C08C45EFD80099B1BB12F833300199BB
:1001D000C95CC9072DD12FE0C17BA6F1010C88466F
:1001E000614529D14178C9F3072C0491614523D990
:1001F000002100910499A6F1020C614513DA4146F1
:100200000BE012F833C001FB04CC1FFA8CFC37F969
:100210001C80F04510DB491EC9B2DDF810C08C45CA
:10022000EFD3009941B912F833300199C95C8907BD
:1002300002D5012180F80F110BF10100C0B28346F5
:100240000598417D594588D80398FB49012803D07A
:100250009AF8150008B32CE0002001230870761EE0
:1002600016E0C0EBC00101EB8102029901EBC20173
:1002700091F8F620012A09D14A780AB1B24205D193
:10028000B1F90220642A01DA81F80F31401CC0B2B2
:100290009AF815108142E4D80BE00878401CC0B2EF
:1002A0000870052805D9052008702021019809F05B
:1002B000F5F815F0FF0F02D001208AF86902C5F3A6
:1002C000072010B101208AF86A02C5F3074010B177
:1002D00001208AF86B02280E02D001208AF86C02F5
:1002E00007B0BDE8F08F2DE9F34F85B0044602F06A
:1002F000B9FB824602F0BAFB00250646049502F0DF
:1003000083FB761EADF810500AFB06F1ADF8121013
:10031000039501218DF80C1002218DF80D10009528
:10032000019502950021E9460DF10C0B0DF1080E27
:1003300000263546334632462BE004AF37F81170BD
:100340001744BFB234F917C0BCF10F0F07DA10F829
:1003500002C01BF801802CEA080C00F802C034F936
:100360001770282F06DD0EB1134604E0154601264E
:100370002B4600E0002619F801805F1BCC4647455C
:1003800005DD0CF8017001AF7D540EF80130521CF0
:10039000D2B25245D1D319F80120062A10D901AAA8
:1003A0005B46525C764605E0855C5F5C3D43855468
:1003B000521CD2B2755C9542F6D2069B01225A5469
:1003C000491CC9B20229B3D38AE738B504460020D4
:1003D000009002F01DFB90F86502002807D16946E5
:1003E0002046FFF780FF21466846FFF7E9FD38BD4C
:1003F0002DE9F04F04468FB0002083460D9002F0A7
:1004000007FB074602F00FFB824602F02BFB054676
:1004100002F02CFB0C90002009900A900B902421F4
:10042000684609F05DF8002697F815E0B4E0C6EBE1
:10043000C60000EB80014FF0190C1AF831000AEBEE
:10044000C1014A7805FB02031FFA83F9012320B199
:10045000971F052F03D8012801D14FF00F0CB1F9D8
:100460000210282900DA002301216F1E00EB010889
:10047000B84507DA09EB01080FFA88F834F9188053
:10048000E04543DBB0EB010807D4A9EB01080FFA04
:1004900088F834F91880E0457CDB491CC9B204298E
:1004A000E4D39BB3511E36D4092A34D001FB050195
:1004B0001FFA81F9002100EB010CBC4510DA09EBB1
:1004C000010C0FFA8CFC0CEB050834F91CC00FFA78
:1004D00088F8BCF1190F17DC34F91880C44513DC17
:1004E000B0EB010C13D4A9EB010C0FFA8CFC0CEB54
:1004F000050834F91CC00FFA88F8BCF1190F03DCA9
:1005000034F91880C44502DD002304E042E0491CB0
:10051000C9B20429CFD3DDF830C0511C614533DAAC
:10052000082A31D001FB05011FFA81F9002100EBF7
:10053000010CBC4510DA09EB010C0FFA8CFCACEB9A
:10054000050834F91CC00FFA88F8BCF1190F21DC3A
:1005500034F91880C4451DDCB0EB010C10D4A9EBB4
:10056000010C0FFA8CFCACEB050834F91CC00FFA37
:1005700088F8BCF1190F0DDC34F91880C44509DC8A
:10058000491CC9B20429D2D323B109A90120885535
:100590000DF80200761CF6B2B6453FF648AF0020D3
:1005A00069460CE00A5C012A07D10D9A0244D2B2D6
:1005B0000D920BF1010202F0FF0B401CC0B20C9A2D
:1005C0009042EFD30D99501E814214D1BBF1020F1E
:1005D00011D1002009AB0122195C012907D1C0EB20
:1005E000C00101EB81040AEBC40181F81021401C19
:1005F000C0B20A28F0D30FB073E670B5ADF53E6D0A
:100600000E46054602F004FA04464FF43E61684681
:1006100008F066FF6A463146284605F08EFC024621
:10062000207569462846FFF72CFC60752846FFF7C1
:10063000DFFE0DF53E6D70BDB40700202DE9FF4FC4
:10064000ADF2DC6D984691460027012640F28441C8
:10065000684608F045FF4FF411710DF2844008F030
:100660003FFFFE48007801284DD03220CDF8C80663
:1006700002F0F8F9834602F0F9F9CDF8CC068DF8CE
:1006800000908DF801800BFB0891DDF8E00669F31E
:100690000F0468F30F0530F9110069F31F4468F384
:1006A0001F450DF2844ECDF8D40669461DF817207B
:1006B00001EB4700CDF8D00643784FF0FF390BFB34
:1006C000032080B2CDF8D8061DF8172002EB0901EF
:1006D00009B2002955DB594553DA4FF0FF32DDF8F6
:1006E000D0064078104400B2002846DBDDF8CC3656
:1006F000984242DA0BFB00139BB21EF803C0BCF118
:10070000000F02D039E03C20B0E7DDF8E0C6DDF8AC
:10071000C8863CF913A0C24507DADDF8D4C64FF00D
:1007200003089CFBF8F8D04527DCDDF8E0C6DDF8CF
:10073000D8863CF91880D0451FDB4FF001080EF831
:1007400003806B460DF8161003EB4603761C5870B9
:100750002BB2B6B2834201DD60F30F0523B28B42A8
:1007600001DD61F30F042B14834201DA60F31F45AE
:100770002014884201DA61F31F44521C12B2012A8C
:10078000ADDD09F101000FFA80F9B9F1010F9BDD30
:100790007F1CBFB2B7F5107F01D8B74285D1DDF815
:1007A000DC06046045600DF2EC6DBDE8F08F2DE9CC
:1007B000FF4FAB484FF0000BD1B000680E46174614
:1007C000B0F81480C38ADA46D9465D46902168465F
:1007D0004C9308F085FE902124A808F081FE02F0D9
:1007E00049F902F03FF9489002F040F939144B9171
:1007F00031B23CB2CDE94941489C4FEA264E98FBC4
:10080000F4F31BB24D934C9B47F6FF7193FBF0F052
:1008100000B24F90DDE95E0303FB0403519800260C
:100820000A4630F913004E903746499C33E0489809
:100830004A9B604300B24C9029E04C98DDF8388127
:1008400000EB030C519830F91C004FF0030C98FB9F
:10085000FCFC84450CDC5DF823C00CEB00080DF1BA
:10086000900C4DF823805CF8248040444CF8240020
:100870000BDCA14200DD2146A64200DA26469A4260
:1008800000DD1A469F4200DD1F465B1C1BB273450C
:10089000D3DD641C24B24B988442C8DD701A06284C
:1008A00002DCB81A062802DD002055B07DE70522DB
:1008B0000A236E464A980EE056F8201000EB80049A
:1008C0004D9F02EB440489447C43614391FBF3F464
:1008D000401CA34400B27045EEDD24AC49980EE004
:1008E00054F8201000EB80064F9F02EB46060D44A3
:1008F0007E43714391FBF3F6401CB24400B24B9926
:100900008842EDDD0020B9F1000F0AD09BFBF9F120
:10091000549A51800DB19AFBF5F05499088001204A
:10092000C3E754994880F5E72DE9F0478946DDE9AA
:10093000096700244FF00308DDF820A011E04518F6
:10094000ADB233F915C0BCF1280F08DD9CFBF8FCF3
:100950003D4433F91550AC4501DD641CE4B2491C3B
:10096000C9B29142EBD93F4D4FF0000C05EBCA05DF
:10097000B4B1A95D491CC9B2A9551E290ED9494671
:1009800008E04418A4B2491C23F814C03C44C9B27E
:1009900023F814C09142F4D91E20A855BDE8F08771
:1009A00005F806C0FAE72DE9FE4F0646002402F0DE
:1009B0005DF8074602F056F8A04601464046454617
:1009C00005E026F810500844641C80B2E4B2BC4232
:1009D000F7D320270095CDE90157334603220021A4
:1009E0004046FFF7A1FF0124CDE90054334607221A
:1009F000042140460297FFF797FF0220CDE90050FF
:100A000033460B22082102974046FFF78DFF032053
:100A1000CDE9005033460F220C2102974046FFF7E4
:100A200083FF4FF0040ACDE9005A33461322102108
:100A300040460297FFF778FF4FF0050BCDE9005BCA
:100A400033461722142140460297FFF76DFF062018
:100A50001B2233461821029706E00000B60700204B
:100A60002808002068870020CDE900504046FFF7A5
:100A70005BFF4FF00709CDE9005933461F221C21C7
:100A800040460297FFF750FF01F0F0FF471E01F0CC
:100A9000E9FF4743B8B26FF01F078DE8B00080460A
:100AA000334603220021FFF73FFF0094CDE90147C1
:100AB0003346072204214046FFF736FF0220CDE9E6
:100AC000004033460B22082102974046FFF72CFFD7
:100AD0000320CDE9004033460F220C210297404607
:100AE000FFF722FFCDE9004A33461322102140468A
:100AF0000297FFF719FFCDE9004B33461722142167
:100B000040460297FFF710FF0620CDE9004033462C
:100B10001B22182102974046FFF706FFCDE9004946
:100B200033461F221C2140460297FFF7FDFEBDE819
:100B3000FE8F2DE9F34F4FF0000BBFB05E46CDF8AE
:100B400000B0CDF8C8B0CDF8F0B0CDF8CCB0CDF84D
:100B5000D0B0D9465D46CDF8E8B048210EA8CDF812
:100B6000DCB008F0BDFC482120A808F0B9FC00204A
:100B7000019036903D903590FE480068B0F916100F
:100B8000399144790779A0463B973F98FFF70BFFCF
:100B9000F9480078012807D0322038905020864646
:100BA00000200DF1800C2CE03C2038905A20F6E714
:100BB000002122E000FB04123F9B92B233F9122085
:100BC000389B9A4217DD3CF8103001281A442CF863
:100BD000102010D9BA1E90420DDA884500D98846F7
:100BE0003B9A824200D93B90894500D289463A9A85
:100BF000824200D23A90491CC9B2A142DAD3401CC9
:100C0000C0B2B842D4D3A9EB08014FF0FF300A2993
:100C10007EDC01464FF00009484640E03CF91020D8
:100C2000002A2CDDB9F1000F0DD0379B9A4206DD6A
:100C3000379201EB410302AA02EB43029080B9F123
:100C4000010F12D029E0491C09B201EB41030DF15B
:100C500008083A9328F813003A9B379208EB4302AE
:100C60004FF00109908005291BDC7A1E904214D1B7
:100C700001EB410302AA02EB430250800DE0B9F1FF
:100C8000010F0AD101EB410802AB03EB4803421EFE
:100C90005A804FF00009CDF8DC90401CC0B2B84239
:100CA000BCD34FF00009062978DA0020491C2CE05B
:100CB00000EB400302AA02EB4302B2F904203CF924
:100CC0001280F0451FDD012A10DDBB1E9A420DDAAD
:100CD000009A521CD2B20092369A022A13D233AB37
:100CE0009854369A521CD2B236920CE00BF10102A3
:100CF00002F0FF0B019A022A05D234AB9854019AF4
:100D0000521CD2B20192401CC0B28842D0DB00E03B
:100D1000EFE00098022801D903203EE030B10146FF
:100D20000120022916D001291DD037E0BBF1000FA8
:100D300034D0BBF1030F31D29DF8D0008DF8C8003C
:100D4000BBF1020F03D19DF8D1008DF8C9004FFA15
:100D50008BF022E0884948709DF8CC008DF8C800DF
:100D60009DF8CD000EE0BBF1010F03D0BBF1000FE9
:100D70000CD013E0804948709DF8CC008DF8C80075
:100D80009DF8D0008DF8C900022006E07A4948702D
:100D90009DF8CC008DF8C80001208146A9F1010022
:100DA00002285FD200210DF1380C0DF1F00B67E045
:100DB00032A802AB405C00EB400013F8102003EBBC
:100DC0004000B0F9028015E000200FE002FB0403B0
:100DD0003F9F9BB237F91330389FBB4204DD3CF88C
:100DE00010703B442CF81030401CC0B2A042EDD330
:100DF000521CD2B29045E7DA002210462AE03CF9B4
:100E00001030002B17DD32B1AB4201DD1D468246AA
:100E1000012A03D01CE001221D468246631E98422F
:100E200016D1754514DD761C4B1C0BF801A0DBB206
:100E3000F6B235930CE0012A0AD10022754506DD91
:100E4000761C4B1C0BF801A0DBB2F6B235930025E3
:100E5000401CC0B2A042D2D3009820B1012E02D9CA
:100E60004FF0030944E00020024603E02CF8102074
:100E7000401CC0B2A042F9D30025491C2E46C9B27D
:100E8000494595DB3D9898BB359800244FFA80F989
:100E90002BE032A81BF80450005D2A4600EB40010D
:100EA00002A800EB41003F99868868463346FFF769
:100EB000C5FBDDE900124098CDE9005600EB840344
:100EC0003F98FFF774FC60B14098399930F82400DE
:100ED000884201DA081A00E00020409921F8240035
:100EE00001E04FF0FF39641CE4B235988442D0D35E
:100EF000484641B059E42DE9FF4F1F4800256FF0E7
:100F00007847C18B828B891A09B20291418C028C7D
:100F1000891A09B20191B0F836A00321AAF10100A3
:100F200004B20090BAFBF1F000F0FF0CBCF1060F28
:100F300001D94FF0060C0021DFF840B034E0002367
:100F40002EE0AAEB03080BEB88093BF9212039F9C5
:100F5000046C0BEB8100921BB0F9020039F9026CB2
:100F6000801B02FB02F600FB0066BE4216DA374623
:100F7000002A05E028080020B60700207887002016
:100F800000DC524212B20392002800DC4042A8F179
:100F900001080FFA80FE0DB20FFA88F45B1C9BB2B9
:100FA0006345CED3491C89B26145C8D3DFF8F0C48C
:100FB00042F210708742ACF84850ACF84A4072DCFC
:100FC0000299052091FBF0F203998A426BDD0199A9
:100FD00091FBF0F1714566DD00202CE03BF92030FB
:100FE0003BF92520D846991A002901DD0E4600E07C
:100FF000D61ABCF92470BE4204DD002900DCD11AE7
:10100000ACF8241008EB8001B1F902200BEB85014C
:10101000B1F90230D11A002901DD0E4600E09E1A16
:10102000BCF92670BE4204DD002900DC991AACF838
:101030002610401C80B2A842D0DB00982BE03BF980
:1010400020303BF924205D46991A002901DD0E4627
:1010500000E0D61ABCF92870BE4204DD002900DC8D
:10106000D11AACF8281005EB8001B1F902300BEB76
:101070008401B1F90220991A002901DD0D4600E032
:10108000D51ABCF92A60B54204DD002900DCD11A6A
:10109000ACF82A10401E80B2A042D0DC012004B07F
:1010A000BDE8F08FFFE70020F9E7F0B50023024626
:1010B0001FE0FC4F37F8224037F82060A41B25B210
:1010C00007EB820407EB8007B4F802C07F88B4F80E
:1010D00004E0E488ACEB070CE41B24B26543AEEB00
:1010E00006060FFA8CFC36B206FB1C54521C234435
:1010F00092B28A42DDD35810F0BD2DE9F04F0026A0
:10110000E74A42F210778AB03D4639463446B14646
:10111000B246B4463046B2F836B014E0E14A32F98D
:101120002030AB4200DA1D4602EB8002B2F9022009
:101130008A4200DA1146B34200DD1E46A24200DDBB
:101140001446401C80B25845E8D3601A00B200280B
:1011500059DD0A2290FBF2F00FFA80FC00200446D1
:101160006A4642F2107322F8203002EB8003401CE2
:1011700080B296465C800A28F3D3002225E0C94B52
:10118000012003EB8203B3F90270431E03FB0C142E
:10119000BC4214DC00FB0C14BC4210DBC14B0EEB58
:1011A000800434F9048C33F92230984501DD24F8A9
:1011B000043C34F9028C984501DA24F8023C401CC6
:1011C00000B20A28E1DD521C92B25A45D7D3002062
:1011D00042F21074734633F92010A1420BD003EB96
:1011E0008002B2F90220914205D009F10107521A9A
:1011F0000FFA87F99244401C80B20A28EBD3A6EB81
:10120000050C0CFB09FC0AEBCA020CEB8C1102EB7F
:101210000A10B1EB800F02DD01200AB040E7002088
:10122000FBE72DE9F04F002305461A4618464FF01C
:10123000010B4FF0020A8D4201DD002030E7DFF89C
:1012400064E20EEB85063EF925903EF921C00EEBD7
:101250008107B6F90280A9EB0C04B7F902700CFB08
:1012600008FC09FB17C9A7EB0806002C03DD764232
:101270006442C9F10009AFB213E00EEB870C3EF9EE
:101280002780BCF902C008FB06F804FB0C8808EBB9
:10129000090CBCF1000F20DD03F1010307F1010788
:1012A000BFB28F42E9DD642403FB04F6491B4C1CEA
:1012B00096FBF4F54B2D02DACB1A032B01DA40EA48
:1012C0000B006423534393FBF4F34B2B02DA891A8C
:1012D0000329B3DA40EA0A00E2E602F10102DDDBAB
:1012E000DAE72DE9F04F0025DDE90BBEDDF824A09B
:1012F00037E0B2F90060282E72DA0AEBC504B4F9BF
:101300000690B9F11E0F2ADD00EBC60794F900C064
:1013100097F90080E0450BD1B7F806C00CEB090641
:10132000FE80B2F90060A48800EBC606B48016E027
:10133000761C36B2168000F836C0B2F900706688A6
:1013400000EBC7077E80B2F90070A68800EBC707E4
:10135000BE80B2F90060E48800EBC606F4806D1C24
:10136000ADB25D45C5D9002235E0B3F90040282C67
:1013700036DA0A9800EBC200B0F906701E2F28DD9D
:1013800001EBC40590F9006095F900C0B44509D19E
:10139000EC883C44EC80B3F90040808801EBC40445
:1013A000A08016E0641C24B21C8001F83460B3F9FC
:1013B0000050448801EBC5056C80B3F90050848867
:1013C00001EBC505AC80B3F90040C08801EBC40453
:1013D000E080521C92B27245C7D9012060E6FFE757
:1013E00000205DE6F0B52E482F4D5430DFF8B0C038
:1013F000B0F90040B0F904202E68B0F90210B0F93D
:101400000600B6F91650BCF81AE0A71A0B1AB6F97E
:101410001460BEF1030F1ED14FF0000EACF81AE0BD
:10142000102C18DB103DAC4215DC102A13DBAA424D
:1014300011DC10290FDB103EB1420CDC10280ADB56
:10144000B04208DC7F4303FB037041F288318842DD
:1014500001DA0120F0BD0020F0BDF0B5124C0327E9
:101460002468B4F91650B4F9146095FBF7F4B0F998
:101470000E50AC421CDCB1F90EC0BCF1C80F17DA3B
:10148000B2F800C0BCF1010F12D1B3F900C0BCF139
:10149000020F0DDA007A012808D00920F0BD000003
:1014A000B607002078870020280800200820F5E7EC
:1014B000AC4213DD96FBF7F0B1F90E40A0420DDC13
:1014C000188801280AD1B2F90000022806DA087A41
:1014D000012801D00B20E1E70A20DFE70020DDE74B
:1014E0002DE9FF4FDFF84C84002785B0B8F81E10B7
:1014F000B8F81C20B8F82000891A0CB2B8F82210ED
:101500003E46081A05B20397BB46BA46B94601974C
:10151000962C77DB962D75DBFFF7EFFD002871D158
:10152000DFF814C4B8F836000CEB8001BCF90030C9
:1015300031F9042C981A002800DCD01A0290FE48D9
:1015400031F9021CB0F90220501A002800DC881A78
:101550008046FFF7D0FCF74AD071B2F84A0081B25A
:10156000B2F8480080B2FFF7A0FD0799089AB1F9D8
:1015700000100091B2F900209646714500DC11463A
:1015800004910121032294FBF2F395FBF2F21BE09C
:10159000DDF800C08C4509DBDDF814C00CEBC10C94
:1015A000BCF906C0634501DA7F1C3FB28E4509DBFA
:1015B000DDF818C00CEBC10CBCF906C0624501DABD
:1015C000761C36B2491C09B2DDF810C06145DFDD7A
:1015D000012F79DD012E77DD042F75DA042E73DA01
:1015E000002801DD014600E0414242F210739942B9
:1015F0006ADD032204FB05F191FBF2F2002802DD13
:10160000014601E060E041428A425DDA0299B1EBB5
:10161000A40F08DAB8EBA50F05DA0299494308FBD5
:101620000811994221DBC34BD97901291BD1B3F9A8
:101630002410B1EB640F16DAB3F92620B2EB650F74
:1016400011DAC8290FDAC82A0DDAB3F92820B2EB6B
:10165000640F08DAB3F92A10B1EB650F03DAC82A70
:1016600001DAC82901DB039949B1B449002801DD39
:10167000002000E001208876062009B010E5B3F9CB
:101680004800B3F94A401DE0AB4A019D32F92010F1
:10169000A94202DD0191A3F84E0002EB8002B2F9EB
:1016A0000220524502DD9246A3F85200594502DA63
:1016B0008B46A3F84C004A4502DA9146A3F8500045
:1016C000401C00B2A042DFDB0020D6E72DE9FF4F2F
:1016D000DFF860C28A468AB0BCF81E20BCF81C3015
:1016E000BCF82010D21A14B2BCF822200027511ADC
:1016F0000C9A049709B2B2F900303D4647F6FF7BD9
:10170000282B7CDA0D9AB2F90020282AF9DA962CD7
:1017100075DB9629FCDB934201DD1E4600E0164690
:10172000012117E08B4207DB00EBC104B4F906404E
:10173000462C01DD07B98FB28A4207DB0AEBC104F0
:10174000B4F90640462C01DD05B98DB207B11DB9CB
:10175000491C09B2B142E5DD00EBC7060AEBC5043E
:10176000B3880693A38874480593069B028830F8D3
:1017700023309646D11A0FFA81F86E49CDF80080D1
:10178000C98E039100EB8108B0F802C038F8041C40
:10179000CA1A069B0FFA82F900EB83025288ACEB5F
:1017A00002031BB2029338F8028CA8EB020213B2B8
:1017B0000193059B30F82330AEEB0302C91A059B59
:1017C00012B200EB830009B24088ACEB00030FFAC1
:1017D00083FCA8EB0000DDE9008308FB03F8029B13
:1017E0000FFA80FE09FB1380002805DC09FB03F0DB
:1017F000DDE9003803FB18004010079000E09FE28D
:1018000002FB0EF001FB1C00002803DC01FB0CF1C5
:1018100002FB1E104FEA60090398401E81B20020AF
:10182000FFF743FC00284348C08EA0F1010081B2BD
:101830004FF0000002DDFFF738FC02E0FFF735FC57
:101840004042B4F90230DFF8F08038F923C0CDF817
:1018500000C0B4F9042038F922100191ACEB010169
:10186000002902DC0199A1EB0C0108EB830308EBD2
:101870008202B3F90230B2F902C0A3EB0C02002AD3
:1018800001DCACEB030211440891B4F90A3038F9D9
:1018900023C0CDF808C0B4F90C2038F92210039108
:1018A000ACEB0101002902DC0399A1EB0C0108EB70
:1018B000830308EB8202B3F90230B2F902C0A3EB52
:1018C0000C02002A01DCACEB0302DFF86CC0B6F9B5
:1018D00002E0B6F9043011443CF92E203CF9238093
:1018E000A2EB080CBCF1000F01DCA8EB020CDFF846
:1018F000488008EB8E0208EB8303B2F902E0B3F9EB
:101900000230AEEB0302002A01DCA3EB0E020CEB6B
:10191000020EB6F90A30084A0993B6F90C8032F97A
:10192000233032F928C0A3EB0C02002A01DCACEB17
:10193000030205E0B6070020788700203CCB00209A
:10194000DFF858C4099B0CEB83030CEB880CB3F94C
:101950000230BCF902C0A3EB0C08B8F1000F01DCA7
:10196000ACEB03089044022D5DD80D9AB2F900202B
:10197000521B012A05D0022A55D1B4F91620322A69
:1019800051DA0C9AB2F90020022A4CDC089AC82AD3
:1019900049DDC82947DDB1EB420F44DAB2EB410F14
:1019A00041DADDE90023FD499A4203DADDE9022349
:1019B0009A4207DBDDE900239A4234DDDDE90223A8
:1019C0009A4230DDF64BB1F90020B3F836C001EB96
:1019D0008C0131F9041C511A3231642923D949464A
:1019E000484501DD024600E00A46A0EB0901002956
:1019F00001DCA9EB000102EBD272B1EB620F12DA4B
:101A00000599998594F90010012903D194F90820CA
:101A1000521C02D0491C03D005E002200EB00DE498
:101A2000217A01290AD0022F7AD80C99B1F9001035
:101A3000C91B012908D0022902D071E00320EDE77B
:101A4000B6F9161032296BDA0D99B1F90010022996
:101A500066DCBEF1C80F63DDB8F1C80F60DDB8EB1E
:101A60004E0F5DDABEEB480F5ADAB6F90210CB4BD7
:101A700003EB8101B1F90220B6F9041003EB8101F7
:101A8000B1F902108A420DDAB6F90A70B6F90CC043
:101A900003EB870703EB8C0CB7F90270BCF902C0AB
:101AA00067450FDB8A423BDDB6F90A10B6F90C2018
:101AB00003EB810103EB8202B1F90210B2F90220BB
:101AC00091422DDDB64FB3F90210FA8E03EB82027C
:101AD00032F9022C891A3231642921D907998842B6
:101AE00001DD024600E00A46411A002901DC07999F
:101AF000091A02EBD270B1EB600F11DA0698B885C3
:101B000096F90000012803D196F90810491C02D06B
:101B1000401C02D004E0042080E7307A012805D080
:101B200094F90090B9F1FF3F02D084E0052075E7F9
:101B3000207A01287FD194F91000401C7BD1207EAF
:101B4000012878D10123DFF8548200216A180AEBBA
:101B5000C200B0F90260B0F9042038F926C038F9A3
:101B60002270ACEB0700002801DCA7EB0C0008EBAF
:101B7000860608EB8202B6F90260B2F90270F21B27
:101B8000002A00DCBA1B1044642800DA0023049AFF
:101B9000904200DD0490584500DA8346491C09B2A2
:101BA0000429D3DB0498B0EB4B0F00DD0023B4F91C
:101BB0002220B4F92410464638F9227038F921C0A1
:101BC000A7EB0C00002801DCACEB070006EB82025F
:101BD00006EB8101B2F90270B1F90220B91A0029AD
:101BE00000DCD11B0844642825DC012B23D1B4F987
:101BF000020036F92010B4F9120036F920008142B3
:101C000019DAB4F91C1036F92110884213DAB4F944
